:0200000460009A
:10000000464346420004015600000000010303007D
:100010000101000001040000400000000000000099
:1000200000000000000000000000000000000000D0
:1000300000000000000000000000000000000000C0
:1000400000000000010406000000000000000000A5
:100050000000800000000000000000000000000020
:100060000000000000000000000000000000000090
:100070000000000000000000000000000000000080
:10008000EB04180A063204260000000000000000FD
:100090000504012400000000000000000000000032
:1000A0006B0418080832042600000000000000005D
:1000B0000604000000000000000000000000000036
:1000C0008104042400000000000000000000000083
:1000D00020041808000000000000000000000000DC
:1000E00001040420000000000000000000000000E7
:1000F0003204180804220000000000000000000084
:1001000090041830002400000000000000000000EF
:100110000204180800200000000000000000000099
:100120003504000000000000000000000000000096
:10013000600400000000000000000000000000005B
:10014000F5060000000000000000000000000000B4
:10015000000000000000000000000000000000009F
:10016000000000000000000000000000000000008F
:10017000000000000000000000000000000000007F
:10018000000000000000000000000000000000006F
:10019000000000000000000000000000000000005F
:1001A000000000000000000000000000000000004F
:1001B000000000000000000000000000000000003F
:1001C000000100000010000000000000000000001E
:1001D000000001000000000000000000000000001E
:1001E000000000000000000000000000000000000F
:1001F00000000000000000000000000000000000FF
:10100000D10020410020006000000000000000002E
:1010100020100060001000600000000000000000D0
:10102000000000600000800000000000FFFFFFFFE4
:1020000000000220451E0360615000006550000082
:102010005D5000005D5000005D50000000000000B9
:1020200000000000000000000000000069500000F7
:102030005D50000000000000998702605D9D026015
:1020400075500000795000007D5000008150000064
:1020500085500000895000008D5000009150000014
:1020600095500000995000009D500000A1500000C4
:10207000A5500000A9500000AD500000B150000074
:10208000B55000005D5000005D5000005D50000044
:10209000B9500000BD500000C1500000C550000004
:1020A000C9500000CD500000D1500000D5500000B4
:1020B000D9500000DD500000E1500000E550000064
:1020C000E9500000ED500000F1500000F550000014
:1020D000F9500000FD5000005D5000005D50000010
:1020E0005D5000005D5000005D5000005D5000003C
:1020F0005D5000005D5000005D5000005D5000002C
:102100005D5000005D5000005D5000005D5000001B
:102110005D5000005D5000005D5000005D5000000B
:102120000151000005510000095100000D5100004F
:10213000115100005D5000005D5000005D50000036
:102140005D5000005D5000005D5000005D500000DB
:102150005D5000005D5000005D5000005D500000CB
:102160005D5000005D5000005D5000005D500000BB
:102170005D5000005D5000005D5000005D500000AB
:102180003D0100004D0100005D0100006D010000F7
:102190007D0100008D0100009D010000AD010000E7
:1021A000BD010000CD0100001551000019510000D3
:1021B0005D5000005D5000005D5000005D5000006B
:1021C0005D5000005D5000005D5000005D5000005B
:1021D0005D5000002D9E02605D5000005D500000CB
:1021E0005D5000005D5000005D5000001D5100007A
:1021F000215100005D5000002551000029510000D0
:10220000B13C0260A13C02602D5100003151000040
:102210005D5000005D5000005D5000005D5000000A
:102220005D5000005D500000310200005D50000074
:102230005D5000005D5000005D5000005D500000EA
:102240005D500000190200001F020000250200007E
:102250002B0200005D5000005D5000005D5000004A
:102260005D5000005D5000005D5000005D500000BA
:102270005D5000005D5000005D5000005D500000AA
:102280005D5000005D5000005D5000005D5000009A
:102290005D5000005D5000005D5000005D5000008A
:1022A00035510000395100003D5100005D500000E3
:1022B000415100005D5000005D5000005D50000085
:1022C0005D5000005D5000005D5000005D5000005A
:1022D0005D5000005D5000005D5000005D5000004A
:1022E0005D5000005D5000005D5000005D5000003A
:1022F0005D5000005D5000005D5000005D5000002A
:102300005D5000005D5000005D5000005D50000019
:102310005D5000005D5000005D5000005D50000009
:102320005D5000005D5000005D5000005D500000F9
:102330005D5000005D5000005D5000005D500000E9
:102340005D5000005D5000005D5000005D500000D9
:102350005D5000005D5000005D5000005D500000C9
:102360005D5000005D5000005D5000005D500000B9
:102370005D5000005D5000005D5000005D500000A9
:102380005D5000005D5000005D5000005D50000099
:102390005D5000005D5000005D5000005D50000089
:1023A0005D5000005D5000005D5000005D50000079
:1023B0005D5000005D5000005D5000005D50000069
:1023C0005D5000005D5000005D5000005D50000059
:1023D0005D5000005D5000005D5000005D50000049
:1023E0005D5000005D5000005D5000005D50000039
:1023F0005D5000005D5000005D500000FFFFFFFFDA
:10240000024B5A690260586100207047B0270020D3
:10241000024B5A6912685A61704700BFB02700200A
:10242000C460056146618761C0F81C80C0F82090D7
:10243000C0F824A0C0F828B0C0F82CD080ED0C8BD8
:1024400080ED0E9B80ED10ABC0F808E0FFF7D8BF21
:10245000104908B54B690BB925F02FFD1A68586073
:102460004A611846C468056946698769D0F81C80C6
:10247000D0F82090D0F824A0D0F828B0D0F82CD0F4
:1024800090ED0C8B90ED0E9B90ED10ABD0F808E02A
:1024900001207047B027002010B5002104464AF003
:1024A000BBFF18B914B120464BF00EF810BD002147
:1024B0004AF0B2BF10B5012104464AF0ADFF18B989
:1024C00014B120464BF000F810BDFFF7E5BF10B582
:1024D00001220C464BF01CF818B914B120464AF002
:1024E000F3FF10BD4BF014B84BF03AB8484308B5B1
:1024F0000830FFF7DCFF40B1044B5A6A02B11060AC
:102500000021C0E900125862083008BDB027002041
:10251000034678B153F8042C083812B153F8081C5C
:10252000116053F8083C13B15A604BF019B8024BD4
:102530005A62FAE7704700BFB02700200346054AF9
:10254000106A1A6841688A4202D3521A1A607047A8
:102550000068F7E7B0270020014441F205538842A4
:1025600004D398B2012838BF0120704703EB43130E
:1025700010F8012B5340F2E7034B044A1A62002281
:10258000C3F83823704700BFB027002014C105608E
:102590002DE9F04780460E46FFF7DEFF124B074657
:1025A0001C6A0CB920461AE0D4F80C90002504F1FE
:1025B000180A4D4501D12468F3E7236933F8153033
:1025C000BB420ED163695B5DB3420AD132464146DC
:1025D0005AF8250026F032FD18B960682844BDE895
:1025E000F0870135E5E700BFB02700202DE9F8436B
:1025F00081460E46FFF7CCFF0246002840F08B8054
:10260000FF2E03D9454946484AF0C6FF454C751C84
:10261000D4F8380390B1D4E9CF132B448B4229D995
:102620002944FFF75FFF0746D8B90246D4F84013A4
:10263000D4F83803FFF756FFC4F83873802D2F46BF
:1026400038BF80273846FFF732FFC4F83803D0BBC5
:102650002846FFF72CFFC4F8380398BB28464AF0F9
:1026600033FFD4F83C332B44C4F83C33D4F838332C
:10267000002BE3D0D4F840333146D4F838734846C1
:102680001D441F44C4F84053FFF766FF49464FF00E
:10269000000980463246384626F06EFC07F8069060
:1026A000236AD3E90253AB4225D36D000A2D38BF0C
:1026B0000A25C5EBC5001830FFF7F9FE48B9C4F884
:1026C0003803CBE72F460023C4F83C73C4F84033EB
:1026D000D0E700F11803226A03EB8503026003616F
:1026E00003EB450343615368D268C0F80C90134470
:1026F000C0E901352062236AD3E903215B6921F82F
:102700001280911D9E54236A43F821705868D9683D
:1027100002440131D9601046BDE8F8830FD7046048
:102720004C4B0560B027002010B5044626F098FCFD
:1027300001462046BDE81040FFF758BF07B501909D
:1027400001A8FFF7FBFE019A036933F8120003B0FA
:102750005DF804FB07B5019001A8FFF7EFFE019BB0
:102760004269D05C03B05DF804FB07B5019001A895
:10277000FFF7E4FE019B063350F8230003B05DF839
:1027800004FB13B5019001A80C46FFF7D7FE019B8F
:102790004269D25C063350F82300226002B010BDBB
:1027A0002DE9F8431D460023074688460360164678
:1027B0000B6013602B60154BDFF854901C6A0CB152
:1027C0004C4505D12B68326813442B60BDE8F88373
:1027D0003B6801333B60E268D8F80030134462691B
:1027E000C8F80030E368D1188A4207D320464AF07F
:1027F000EFFE2B68246818442860E0E7336812F87D
:10280000010B013303443360EEE700BFB027002023
:1028100014C105602DE9F8430D4B0E4F1C6ADFF81B
:102820003880DFF838900CB1BC4201D1BDE8F883A4
:1028300004F11805E36805EB8306B54201D324686B
:10284000F1E755F8042B4146484600F0CFFCF4E789
:10285000B027002014C105601DD704601024056056
:1028600038B54468054603682144994211D9037B71
:10287000DB0703D5002107484AF08EFE01F1100462
:10288000806824F0070408342146FFF720FE2C60FE
:10289000A86038BD4C4B056070B504460E46114625
:1028A0001546FFF7DDFF31462A46D4E901301844CA
:1028B00026F08AFB62682A44626070BD70B5466883
:1028C0000446B14228BF31460D460121FFF7C8FF3B
:1028D000A368681C721B5919184426F075FB6368BD
:1028E000A06801332844636070BD012938B538BF42
:1028F000012104460025084621606560FFF7CCFDF4
:10290000237BA06065F30003237338BD38B505460B
:102910000C460131FFF7E9FF6C6038BD0023016010
:10292000C0E90132037B43F00103037370470000E9
:1029300038B514460546FFF7D8FF024B25606360A3
:1029400038BD00BF99280060037BDB0710B5044643
:1029500002D48068FFF7C8FD0023A36010BD13B543
:1029600001901020FFF798FD04460199FFF7BDFF85
:10297000204602B010BD10B5044650B1037BDB0702
:1029800002D48068FFF7B0FD2046BDE81040FFF795
:10299000ABBD10BD38B5037B04460D46DB0703D540
:1029A000002107484AF0F8FD016880682944FFF7D4
:1029B0008EFD2368A0601D441844256038BD00BF0B
:1029C0004C4B056038B504460D46FFF749FFD4E986
:1029D00001301D441844656038BDD0E9002310B5AE
:1029E0009A42044602D10121FFF7D4FF0021D4E925
:1029F0000132D154A06810BD10B50C460121FFF77B
:102A0000E1FF047010BD7F29F8B50C46CEB204D8A2
:102A10000121FFF7D7FF0670F8BD06F03F06B1F5BC
:102A2000006FC1F3871546F0800607D265F03F05B9
:102A30000221FFF7C7FF46700570EDE705F03F057F
:102A4000B1F5803FC1F3073745F0800508D267F044
:102A50001F070321FFF7B6FF457007708670DBE79D
:102A6000A40C07F03F07042164F00F0467F07F0710
:102A7000FFF7A8FF857004704770C670CCE713B5E8
:102A800004460846019126F0EBFA019902462046D9
:102A900002B0BDE81040FFF7FFBE10B51446FFF7C7
:102AA0000DFF047010BD10B51446FFF707FF04704A
:102AB00010BD43688B422CBF591A002141607047FA
:102AC00038B504461546084662688A4203D9294447
:102AD0008A4201D8606038BDA368521A184419446C
:102AE00026F072FA6268521B6260F4E708461146EB
:102AF0004AF05EBC37B505460846019126F0B0FAAB
:102B0000044620B102466B68019928689847204620
:102B100003B030BD2DE9F74F89469DF830101746B8
:102B20000D9A11F0DF0F0646A2EB07023DD03029C7
:102B30000CA8254913BF80464FF0100A88464FF075
:102B4000010A13F0800535D002EBD2746510A2EBB8
:102B50006404002D35DDAB46DA45524673684146C4
:102B6000A8BF5A46306801929847019AABEB020B16
:102B7000BBF1000FF0DC2FB13D4473683A46494683
:102B800030689847002C0CDD2544A24557467368F1
:102B90004146A8BF27463068E41B3A469847002CB8
:102BA000F3DC284603B0BDE8F08FDFF820804FF05B
:102BB000100AC6E713F0010401D11546C9E714460F
:102BC000D9E70025D7E700BF292405601824056050
:102BD0002DE9F043064689B00020119D9DF84880FC
:102BE000139F8DF80F000AB381421ADA2D22494251
:102BF0008DF80F20109A08AC0DF11009A2F10A000F
:102C00008E46B1FBF3FC03FB1C126146092A8CBF04
:102C10001218303204F8012D4C450ED07345EFD90F
:102C20000BE0A80727D52B228DF80F200029E1D132
:102C300030230DF11F048DF81F3015F040099DF869
:102C40000F301CD023B301222B460DF10F0130466B
:102C5000013FCDE90082FFF75DFF814608AA2B46C0
:102C600021463046121BCDE90087FFF753FF484449
:102C700009B0BDE8F0836A07D8D52022D4E7002B3D
:102C8000ECD004AA9442E9D904F8013C013CE5E700
:102C90009946E3E72DE9F04F93B081461D46C807FA
:102CA0009DF874300C4690461C9E0693DDE91E7A12
:102CB0000BD4A10703D122687A4B9A4205D0204653
:102CC0000AF0B6FE400040F0010416F0810306D180
:102CD000069A302A03D15745B8BF57469A46204630
:102CE0000DF1280B0DF090FF002818DBB20712D56C
:102CF0002B230DF129028DF82830F006EDB21DD5F9
:102D0000B8F1020F0DD13021134603F8021B691CE4
:102D100051701A4612E0730701D52023E9E75A469D
:102D2000EBE7B8F1080F61D1B1054FF03003137034
:102D300049BF05F10E03013253700232A2EB0B03BF
:102D4000002116F0200F11700EAA05930CBF0B4640
:102D50002C23BAF1010F0B924FF01002C8BF46F0BE
:102D600040068DF82710CDE90C2116F04002CDE980
:102D70000253079244D023460DAA0BA8CDE9008147
:102D80000CA90DF021FE037880462D2B06D18DF87D
:102D9000273000F101080D9B013B0D93BAF1010FA3
:102DA0003CDD0D9D079B5545B8BF55462BB19DF8A1
:102DB000273003B10135059B1D44AF422BDD16F0D2
:102DC0000103A7EB050527D12C461D4626F0010679
:102DD0004CB12023019434494846009300231A46FD
:102DE000FFF798FE04463023069319E0B8F1100F60
:102DF000A4D13021134603F8021B05F1170187E720
:102E00000AAB0DAA0CA90BA8CDE9008323460DF04F
:102E1000DBFD8046C2E700250024D7E700252C46CD
:102E2000079BDBB19DF8273053B1002301220DF140
:102E300027014846013FCDE90032FFF76BFE04440D
:102E4000059B5BB10023012259464846CDE900327B
:102E5000059AFFF75FFE059B0444FF1A069BBAF133
:102E6000010FC8BF57460D9A414600934846334666
:102E70000197FFF74FFE04444DB120230A4948460D
:102E80000195009300231A46FFF744FE04440B9873
:102E90000EAB984201D0FFF727FB204613B0BDE8E8
:102EA000F08F00BF9C520560CC3B06602DE9F043DB
:102EB00016468BB007469846B207DDF848903DD4D9
:102EC00016F0040F0CBF002320230A460093202194
:102ED000139B02A809F054FBF30504460DD5431CCF
:102EE0001F2B0AD80AAA00211444252204F8202CFA
:102EF0000AAA1C461A4402F8201C16F040051FD0EE
:102F00009DF808302F2B4FF000031BD8012202A997
:102F1000384609F1FF39013CCDE90032FFF7FAFDEF
:102F20000DF109010546334622463846CDE90089B0
:102F3000FFF7F0FD28440BB0BDE8F0832B23C4E776
:102F400002A9F0E702A91D46EDE700002DE9F04FC8
:102F5000074689B014460025DFF88C820B461E46D2
:102F600013F8012B92B9B14213D30B78002B00F068
:102F70003481013120234FF0000A084610F8012B5C
:102F800082B94FF000094FF00A0C2AE0252AE6D159
:102F9000E9E7A6EB01097B6838684A464D44984743
:102FA0003146E2E72D2A03D14AF0010A0146E4E75F
:102FB0002B2A02D14AF0020AF8E7202A02D14AF06D
:102FC000040AF3E7212A02D14AF0080AEEE7302A80
:102FD000D7D14AF0400A1346E8E70CFB0929A9F1CA
:102FE00030090E4611F8012BA2F130000928F4D95E
:102FF0002E2A33D172782A2A0FD00A464FF00A0CB3
:103000000021164612F801BBABF13000092807D8A1
:103010000CFB01BBABF13001F3E7023654F8041BA3
:1030200021EAE17B32786C2A08BF01363178002929
:1030300000F0D38078295FD8572912D8472959D86A
:10304000442959D907345246384624F00704CDE9BB
:10305000009BB4EC020BFFF729FF5FE04FF0FF3B52
:10306000E0E7A1F15802202A46D801A050F822F04A
:10307000AB310060F9300060F9300060F930006079
:10308000F9300060F9300060F9300060F93000601C
:10309000F9300060F93000600731006029310060CC
:1030A0008F31006045300060453000604530006081
:1030B000F9300060F9300060F9300060F9300060EC
:1030C000F9300060F9300060F9300060F9300060DC
:1030D000CB3100603D310060F93000606731006045
:1030E000F9300060AB310060F9300060F930006009
:1030F000AB310060502968D07B68012231463868C6
:10310000013598470BE054F8042BCDE900395346BC
:103110003AB1042233493846FFF7FCFC0544711CE0
:103120001CE705224146F6E754F8042B07A98DF861
:103130001C200122CDE900395346ECE707A954F8D9
:10314000040B0493FFF71DFBBBF1FF3F0146049BFB
:1031500004D0079A934538BFCDF81CB0079ACDE943
:1031600000395346D7E754F8041B059308460491E9
:1031700025F076FFBBF1FF3F0246DDE9041302D0E4
:10318000584528BF5A46CDE900395346C3E7CDE933
:10319000023961230122CDF804A000930A2354F8D8
:1031A000041B3846FFF714FDB8E74A1C21F00F0155
:1031B000CDF804A002F006020F39CDE90239C9B2F8
:1031C000C2F1100300910022E9E7CDE90239612341
:1031D000CDF804A000931023F5E7284609B0BDE818
:1031E000F08F00BF04240560092405600EB403B508
:1031F00003AA52F8041B0192FFF7A8FE02B05DF883
:1032000004EB03B0704790F90010024603780029E0
:1032100001DB1846704703F07F004023184206D1B7
:1032200012F8013F03F0C001802904D0704720EA62
:1032300003005B08F2E703F03F0343EA8010EFE787
:10324000431C18460133027802F0C002802AF8D0ED
:10325000704703460020994200D8704711F8012DAD
:1032600002F0C002802A18BF0130F4E7014403468F
:10327000002099421A4600D870471278013302F0B4
:10328000C002802A18BF0130F3E700007F289DBFED
:10329000024B185CC0F34000002070473A240560E0
:1032A0007F289DBF024B185CC0F3C0000020704710
:1032B0003A2405607F289DBF024B185CC0F3800054
:1032C000002070473A2405607F289DBF024B185CA0
:1032D000C0F38010002070473A2405607F2809D889
:1032E000064B1B5C13F00C0F06D1A0F15F03584294
:1032F0005841704700207047012070473A2405600C
:103300007F289DBF024B185CC0F30010002070475F
:103310003A2405607F289DBF024B185CC0F3401023
:10332000002070473A24056008B50246FFF7E8FF21
:1033300000B12032104608BD08B50246FFF7EAFF8B
:1033400000B1203A104608BD3038092884BF20F06B
:1033500020000738704701440246002010B5E524DC
:10336000914203D8B0FA80F0400917E012F8013B0F
:1033700030B103F0C003802B11D1431ED8B2EFE768
:10338000BF2B09D9F72B09D8DB0803F0060344FA51
:1033900003F303F00300E3E71B06E1D510BD0020B3
:1033A000FCE7023981420B4603D20233181A40105F
:1033B00070471A880239002AF4D0F6E7B2EB131FDF
:1033C00070B54FEA131416D9121B03F00F0301EB6B
:1033D000440115460E46012D31F8024B18BF3468E2
:1033E000013D24FA03F4A4B220F8024BF2D104B94F
:1033F000013A104670BD0022FBE7F0B5059F00249E
:10340000D21B2646A74210D100EB470C002401EB4B
:103410004701A24214D10CEB42031EB10121023339
:103420002CF81210181A4010F0BD31F8145033F86F
:1034300014C06544354420F814502E0C0134E1E7E3
:1034400031F8145035442CF814502E0C0134E0E7B8
:10345000F0B4049F0025D21B2C46AF420BD100EBE9
:103460004706002301EB47059A420FD106EB4201C4
:10347000F0BCFFF796BF31F81560344433F815609F
:10348000A41B20F8154024140135E6E735F8131085
:103490000C4426F8134024140133E5E7022938B51B
:1034A00038BF0221044680680D4618B12368B1EB8D
:1034B000930F07D96900FFF70AF82368A06065F346
:1034C0009F03236038BD38B504460C20FEF7E4FFA7
:1034D000054623682278C3F39D0023F0030302F01E
:1034E0000102400013432B6063686B60FEF7D4FF5A
:1034F000A8602268A168C2F39D02520025F03CFD3D
:10350000284638BD00EB410002EB410210B509B975
:10351000084610BD30F8023D32F8024D1B1B002B4F
:1035200002DB04D10139F2E74FF0FF30F1E701206F
:10353000EFE710B5044638B18068FEF7D5FF2046A6
:10354000BDE81040FEF7D0BF10BD38B50C460221D3
:103550000546FFF7A3FF002C2B78B5BF0122002200
:103560006142214662F3000301222B70AB68023BEB
:1035700023F8021F090C104602F10102F8D168601D
:1035800038BD0023C0E900338360704728B1037859
:103590009B0702D48068FEF7A7BF704738B5054681
:1035A0000C464968FFF77AFF22782B78A86862F307
:1035B00000032B706368A1686B606268BDE83840E7
:1035C000520025F0D9BC0A4629B90178426062F35D
:1035D000000101707047FFF7B8BF08B5FFF7D1FFD2
:1035E000BDE80840FFF7EFBF920042F00202026020
:1035F000002210B4C0E901215DF8044B1946FFF721
:10360000E2BF2DE9F843914698469DF820700421C9
:1036100006464C464546FFF741FF3FB1002C78F186
:1036200000030EDAD9F1000468EB4805337867F33C
:10363000000333700023736054EA050303D1BDE82F
:10364000F8830027F2E7D6E90132591C716022F8AD
:103650001340230C2A0C43EA054315461C46EBE7AE
:103660002DE9F84353EC102B1E460378074610EE65
:10367000105AF20F62F30003037047F6F07313EA77
:10368000164207D13B786FF300033B7000237B6049
:10369000BDE8F8839A42F5D0C6F30A52A2F2FF348D
:1036A000002CEFDB04D10121BDE8F843FFF74DBF4B
:1036B000A2F2EF38C6F31306B8F1000F46F48016F5
:1036C000B8BFA2F57878332C4FEA28183FDCC4F154
:1036D0003402A4F11403C4F1140406FA03F3D54030
:1036E00026FA04F4D6401D4325430024A146414652
:1036F0003846FFF7D3FEC7F80480B9F1000F05D0B4
:103700004FEA49020021B86825F076FC9CB105FA21
:1037100004F2BB6823F81920C4F11003103409F136
:103720000109A3F12002DD4006FA04F426FA02F2B0
:10373000DE40254315434B469845A9D0BA6822F888
:1037400013502D0C013345EA0645360CF4E7A2F27E
:1037500033430C34002B04F00F04B8BFA2F224430F
:103760004FEA2319C3E72DE9F8438F18C2F35B0230
:1037700004460D46511C9846089EFFF78FFE23789D
:1037800029461FFA86FC68F3000323700023636058
:10379000B942084602D3401BBDE8F88302780131E4
:1037A000A2F13003092B05D9A2F14103192B14D83A
:1037B000A2F13703B342EED2D4E901E0F0468146EC
:1037C000B8F1000F10D100EB4E0213B1023220F815
:1037D0001E30121A52106260DAE7A2F16103192B4F
:1037E000D9D8A2F15703E5E7B9F8002008F1FF386E
:1037F00002FB0C3329F8023B1B0CE1E7F8B5044649
:1038000015461E46C1B1531E4FF0FF371E44E90056
:1038100020460F310909FFF741FE237800216FF39D
:103820000003616023704DB9D4E9011000EB410140
:10383000FFF7B7FD6060F8BD0127E8E700230F2917
:103840000ADC3278013D3E4402FA01F201F108013E
:1038500043EA02039BB2F2D162681039501C6060E7
:10386000A06820F81230DEE738B50B7804460578FA
:1038700003F0010305F00100181A0CD163684A68CF
:10388000934209D30BD88A681946A068FFF73AFE1D
:10389000EB0748BF404238BD4FF0FF30F8E701204A
:1038A000F6E7884210B5044601D0FFF777FE23788B
:1038B0006FF30003237010BD884210B5044601D099
:1038C000FFF76CFE63683BB12378C3F30002C2F1DB
:1038D000010262F30003237010BD88421FB5044645
:1038E00001D0FFF75BFE626862B901212046FFF755
:1038F000D5FD0123A26813806360237843F00103A0
:10390000237010E02378D9070FD56FF30003A16867
:10391000237001230846ADF80E3000930DF10E031D
:10392000FFF796FD606004B010BD511C2046FFF704
:10393000B5FD0123D4E90121ADF80E30009308460E
:103940000DF10E03FFF759FD6060D6E72DE9F8434E
:103950004B6805460E46144603B12AB9314628463F
:10396000BDE8F843FFF71ABE02F10F014FEA111844
:1039700003EB1111FFF792FD14F00F04AB6808BFC1
:103980001024D6E90102C4F1100408EB000702EB91
:10399000400E002207F10041013903EB41030146CB
:1039A000994601BB6FF0010C22FA04F408F1FF32D2
:1039B0000CFB00FC520003EB0C0023F80C40C8F198
:1039C000010300EB4303184625F016FB831E17B1D5
:1039D00033F8172092B12B786F60327862F30003CE
:1039E0002B70BDE8F8833EF802CD01394CEA0202A3
:1039F00022FA04FC120429F802C9D2E7013FE6E7E3
:103A0000F0B50E46496885B00546144601B12AB99D
:103A100031462846FFF7C2FD05B0F0BDFFF73EFD79
:103A20002346A868D6E90121FFF7C8FC2B78686017
:103A3000327862F300032B70DB07EDD500232209F7
:103A40007168ADF80E30994201D093420FD1914286
:103A5000E2D9B36804F00F0433F81220012303FA0B
:103A600004F4013C224213D0ADF80E3008E0B768F0
:103A700037F8137057B101239142ADF80E30E8D8F2
:103A8000A968012348B90B806B60C5E70133DAE709
:103A9000BDF80E30002BBFD0F2E702460093084677
:103AA0000DF10E03FFF7A9FC6860B5E773B5536825
:103AB0000C46496806461546994206D308D89268CE
:103AC000A068FFF71FFD002802DA23462C461D469A
:103AD00023782A7861685340DB071BD401313046D4
:103AE000FFF7DCFC6B68B0680093AB68D4E9012198
:103AF000FFF783FC706023787268C3F30003002A29
:103B00000CBF002303F00103327863F3000232702C
:103B100002B070BD3046FFF7C1FC6B68B06800931F
:103B2000AB68D4E90121FFF793FCE3E7F7B55368ED
:103B30000C46496805461646994206D324D8926831
:103B4000A068FFF7DFFC00281EDA23460127344671
:103B50001E462378327861685340DB0716D5013161
:103B60002846FFF79BFC7368A8680093B368D4E904
:103B70000121FFF742FC68606A682B7892B962F312
:103B800000032B7003B0F0BD0027E2E72846FFF7E3
:103B900085FC7368A8680093B368D4E90121FFF736
:103BA00057FCE8E7227802F00102002FE7D0C2F1CB
:103BB0000102E4E72DE9F04F16464A680C4685B04D
:103BC000736805469A423EBF34460B461E4623782C
:103BD0006168DA0756BF3378012303F00103194403
:103BE000FFF75CFCB368726836780093A868D4E984
:103BF00001E824788246A2EB0E02A8F1020884EACA
:103C0000060106F001060392CB07C6F10009B4468F
:103C100054BF04F0010B4FF0000B04F001041FFA35
:103C200089F9CBF10001274689B20191614289B23D
:103C30000291714699B900EB4E01BBF1000F03D020
:103C40000123023120F81E30FFF7ABFB34402B7804
:103C5000686064F300032B7005B0BDE8F08F38F89E
:103C6000022F0139029B5A40039B17445A18914274
:103C700029BF009B4A4633F8022B82EA090228BF7B
:103C80000093019B944407EA0C024FEA1C4C3F0C42
:103C90005A401BFA82F24FEA124B2AF8022BC9E76C
:103CA0002DE9F04F16464A680C4685B07368054604
:103CB0009A423EBF34460B461E4623786168DB07B6
:103CC00056BF3378012303F001031944FFF7E6FBE5
:103CD000A868D4E901A72478A7F10208574614F090
:103CE000010F04F00104009018BF0122A446D6E998
:103CF00001B3367808BF06F0010206F00106514212
:103D0000C6F10009B64689B21FFA89F901916142EC
:103D100089B20291ABEB0A01039167B900EB4A014A
:103D20003443FFF73EFB2B78686064F300032B708D
:103D300005B0BDE8F08F38F802BF013F02998BEA69
:103D4000010B0399DC4401EB070B01995F452ABF86
:103D500033F802BBCB468BEA090BDE444CEA0E0B70
:103D60004FEA1E4E4FEA1C4C8BEA010B009912FAE7
:103D70008BF221F8022B120C0091CEE72DE9F74FC0
:103D800015464A680C4606466B684FF6FF7B9A421A
:103D90003EBF2C460B461D4623786168DB0756BFA5
:103DA0002B78012303F001031944FFF777FB2378F5
:103DB0002A78A16883EA020CD4F80480B068DB4357
:103DC000D243A1F1020A69680CF0010CAF6803F05C
:103DD0000103A1EB080102F00102C64681460191F0
:103DE000BEF1000F19D100EB4801BCF1000F03D068
:103DF0000123023120F81830FFF7D3FA70602378DE
:103E00002A78C3F30003C2F300025340327863F30D
:103E10000002327003B0BDE8F08F3AF8021F0EF1D5
:103E2000FF3E59440B44019971448E452ABF37F82F
:103E3000021B4FF6FF7159440A4483EA0201120C37
:103E40001B0C1CFA81FC29F802CB4FEA1C4CC7E77B
:103E50004B682DE9F04F044685B00E4615460BB170
:103E6000536843B923786FF3000323700023636022
:103E700005B0BDE8F08F81422ED1FFF724FBA542AB
:103E80000646074600D105466B682046716819440E
:103E9000FFF704FB22680021A068C2F39D025200D4
:103EA00025F0AAF8B368D4F808E00022D6F804A0F8
:103EB0000193F446AB680EEB4A08114602936B6817
:103EC0000393039B934231D0ACF10200DDF804B0C0
:103ED0000023CDF800A018E0824204D1FFF7F3FAE6
:103EE00005460746D0E70027CEE730F8029F994401
:103EF0003BF8023B1946029B33F8123003FB019357
:103F00000099038001391B0C009100990029ECD124
:103F10004146881C13B10146A8F80030A1EB0E0100
:103F20000CF1020C013280464910CAE76160384644
:103F30002A7833785340227863F30002227005B068
:103F4000BDE8F04FFFF7F5BA4B6870B5054614466B
:103F500013B11378DA0706D52B786FF300032B70B3
:103F600000236B6070BD636823B90121BDE8704018
:103F7000FFF7EBBA0846FFF7A6FA06462046FFF71A
:103F8000A2FA012104462846FFF7DFFA636883B1ED
:103F9000A3681B88DB0704D5324629462846FFF76D
:103FA00057FF0123D4E901210846FFF707FA6060B3
:103FB00038B93046FFF7BDFA2046BDE87040FFF73C
:103FC000B8BA324631463046FFF742FFDEE72DE908
:103FD000F04F0C4651688FB01746013105460293E9
:103FE000FFF75CFA7A680021A8680132520025F0D8
:103FF00003F82B7820466FF300032B7000236B60CF
:1040000079680131FFF74AFA39462046FFF7C6FAC8
:10401000029BD4F804905B684B45019342D8029B05
:10402000A668D3F80880AB6803933DD3424649465F
:104030003046FFF767FA002832D10123039A606007
:1040400013806B6023786168C3F3000200290CBF02
:10405000002202F0010262F30003029A23703B780F
:1040600012785340DB0718D56B682A78003B18BFDD
:10407000012363F300022A70636873B14FF0FF31CC
:104080000BA8FFF7AAFA0BAA29462846FFF70EFD50
:10409000029A21462046FFF709FD0FB0BDE8F08FD8
:1040A000013001D10023CCE7019B4FF0000E03F15A
:1040B0000042013A5300049338F8123018040EF10C
:1040C000010156D54FEA490300201FFA8EFA09F183
:1040D000010103F1020C0593CAF1100B26F8190037
:1040E00006EB0C03B44661600693069B9C4544D3E3
:1040F000019B38F81220012B02FA0AFB09D9049B14
:10410000CAF1100008EB030232F8022CC2404BEA5D
:10411000020B019A059B891A039A3344696001F1E5
:104120000041013902EB41020592049A02320992E0
:10413000A8F102020892626804920499019A8A42E4
:1041400027D301F1004BCAF1100000210BF1FF3B16
:1041500006EB4B0B5E4570D96FF000416B682BB1DD
:104160005A18039830F81220002A70D06FF00041DE
:1041700072E05B008E469BB2A0E7BCF800E00EFA4E
:104180000AF949EA00002CF8020B2EFA0BF080B273
:10419000ABE71988002033F8022C804642EA01423E
:1041A0000999591AB2FBFBF20691DDF818C008997B
:1041B000079163450BD819880844B8BB0599023BA1
:1041C00021F80229049A0591013A6260B3E7079940
:1041D000BCF8009031F802EF19FA80F907910EFA55
:1041E0000AF141EA18481FFA88F151431FFA81FE8B
:1041F000090CA9EB0E0EC1EB20412CF802EB01EBF0
:104200002E40D6E739F802EF0EFA0AFE4EEA1848B9
:10421000B1F800E01CFA88FCF44421F802CB4FEA24
:104220001C4C8B42EED86044013AC6E74FF0000CBC
:10423000DDF820900699E046F3E7BBF8003043FA3A
:104240000AF283400A4399B22BF8022982E7013B24
:104250006B6083E7013B63606368002B3FF4F2AE61
:104260005A1836F81220002AF4D0EBE6F0B51F46B3
:104270004B6885B004460D4616464BB11378DA07F5
:1042800006D47B68012B0BD1BB681B88012B07D19F
:1042900023786FF3000323700023636005B0F0BD43
:1042A00001212046FFF751F97368002BF6D028460C
:1042B000FFF709F905463046FFF705F9064601A85C
:1042C000FFF75FF97368B3B1B3681B88DB070AD5E2
:1042D0002A4621462046FFF7BBFD3B4622462146A3
:1042E00001A8FFF774FE0123D6E901210846FFF774
:1042F00065F8706048B901A8FFF748F92846FFF74C
:1043000018F93046FFF715F9C8E72A462946284626
:10431000FFF79EFD3B462A46294601A8FFF757FEB8
:10432000D0E7D0E901210346002001EB420210B59D
:10433000914204D31B78DB0748BF404210BD32F8DE
:10434000024D44EA0040F3E730B5D0E901240023F0
:1043500004EB4202944206D302780120D20748BF00
:104360005B420B6030BDB3F5004F04D232F8025D02
:1043700045EA0343EEE70020F4E72DE9F047054660
:10438000D1B1981800264FF0010C03EB0209374613
:10439000D5E90184A4F1020EB8F1000F0ED1B9B332
:1043A000C21A18462B7813F0010FBDE8F04714BF6E
:1043B000FF21002124F020BE1846E3E73EF8024F1B
:1043C000103744EA064695F800A0072F0AF0010AC4
:1043D00002DC08F1FF38DFE7B4B2BAF1000F06D013
:1043E000E4435CFA84FC1FFA8CF4CCF3072CE4B2AF
:1043F00049B100F1FF3A00F8014C53450BD0083F9A
:10440000360A5046DFE782460AF8014BCA45F5E70F
:104410001A44121AC6E7BDE8F08700000000000049
:10442000D0E901329FED0C0B9FED0D6B02EB4303C6
:104430009A4205D30378DB0748BFB1EE400B7047C3
:1044400033F8021D07EE101AB8EEC77B00EE067BAC
:10445000B0EE470BECE700BF0000000000000000DA
:10446000000000000000F0402DE9F84F446881464C
:104470008A4615461E469DF828B00B9F9CB982B10E
:10448000551E3B4615F8011F184639B930230370F5
:10449000002300F8013FC01BBDE8F88F03F8011BA3
:1044A000F0E73846F2E764002046FDF7F5FF804666
:1044B0002246D9F8081024F05FFD3846394608EB4B
:1044C0000402A6F13A03A2F1020C0026E04564467C
:1044D00039D930360C46392E88BFF61804F8016BEE
:1044E0004646B242B44638D8BBF1000F0AD0012686
:1044F000A4EB000CBCF1030F02BF8C1C81F801B0CF
:104500002046F6B14046FDF7EFFF5DB1284624F0A6
:10451000A7FD2A18611E1346AB4229D8954288BFD1
:104520000020044499F80030DB0744BF2D2304F831
:10453000013B3B46621E9A421FD80023E01B2370BA
:10454000AAE72146BFE7248844EA0646B6FBFAF408
:104550000AFB14662CF80249B8E7BCF800C0023622
:10456000BCF1000FBDD0BBF1000FEAD00026BFE7C1
:1045700013F8016D01F8016FCEE71978107803F890
:10458000010B02F80119D6E7D0E9023293423DBF90
:104590005A1C826018784FF0FF307047036810B5DE
:1045A000044613B14068FDF79FFF2046BDE8104068
:1045B000FDF79ABFF8B50C461F4616460546102073
:1045C000FDF76AFF054B8460C0E900743444C460A1
:1045D0006B60034B2860AB60F8BD00BF894500608D
:1045E0009D45006002690A2A10B5044635D1836AE8
:1045F000013383620123A269E36263696261226F0E
:104600002361002A31D0616E8A423BBF501CA16EEB
:104610000022206738BF8A5CA2613BB9E269636609
:104620002261226A23676261626AA26163690D2B5B
:1046300008D10A22A3699342626103D1D4E901033C
:104640009847A061A369013306D163695A1C03D05E
:104650000A2B1CBF0A23A36110BDC36A092A04BF29
:10466000073323F007030133C5E7D4E90103984773
:10467000A061DBE770B504460D4600262069431CA7
:1046800001D1304670BD0A2808D115B1636B002BEB
:10469000F7D020460126FFF7A5FFEFE7FEF7F6FD6E
:1046A00018B12046FFF79EFFE8E72369232B08D1C6
:1046B0002046FFF797FF23695A1CDFD00A2BF7D15A
:1046C000DCE75C2BDDD163690A2BDAD12046FFF7EA
:1046D00089FFE6E70369272B2BD0222B29D0A3F1F2
:1046E000620113291ED8174ACA40D2071AD5426957
:1046F000272A1ED0222A1CD0722B1CD1662A06D152
:104700008269272A15D0222A13D0722B15D143692A
:10471000622B0CD1806927280BD0A0F122035842CC
:1047200058417047662BF0D14269722AE8D00020C8
:10473000704701207047662BF6D0622BF7D1436992
:10474000722BE6E711000900436E2DE9F04F044695
:104750002DED028B85B0A3B1036F93B92921603091
:10476000FEF74AF92369E36163692362A36963621F
:10477000A36E1A7822615A7862619B78A361032341
:104780002367002120466165FFF774FFA36A256B4C
:104790006364002DE36AA36409DA0823013584F811
:1047A0004C30256305B0BDEC028BBDE8F08F04D022
:1047B0000723013D84F84C30F3E7002834D0626BC6
:1047C00092BB06225D1E6FF0004384F84C20D4E9B2
:1047D0000F20D11830F811108D42E3D019D9A16BF8
:1047E0008A4207D308314900FDF771FEA36B2064AC
:1047F0000833A363D4E90F32591CE16322F8135044
:10480000236B01332363CDE7013AE263226B013A64
:104810002263E26BD11830F811108D42F4D3C1D06D
:10482000022384F84C30BDE72669771C01D10023B0
:10483000F7E72046FFF74EFF8146002800F0C481CD
:10484000002384F84C302369752B51D0622B07D19B
:104850006369722B51D1C84602270D23002612E04E
:10486000722B06D16369622BF5D0662B49D10523E3
:10487000D7E7662B49D16369722BF8D04E460127E2
:104880000C234FF0000894F84C20002A3FD184F804
:104890004C303FB12046FFF7A5FE022F02D1204643
:1048A000FFF7A0FE23692046222B14BF4FF0270BF1
:1048B0004FF0220BFFF796FE23695B452AD163690F
:1048C0009B4527D120464FF0030AFFF78BFE204679
:1048D000FFF788FE26B1BA4904F16000FEF7CFF871
:1048E00004F16002002304F1500708EE102A23E0CF
:1048F000012700260C23B046C5E701270D2300261B
:10490000BFE7C84601270C23A8E72F46F1E79A42E4
:10491000BFD047E74FF0010ADCE7934538D10133B8
:1049200059463846CDE90133FEF76DF8019B204624
:104930000193FFF757FE019B2269511C00F03A8159
:10494000BAF1010F02D10A2A00F034815345E4D3B1
:10495000194604F15000FEF7ACF801212046FFF79C
:1049600089FE2046FFF7B6FE00287FF46CAF19E7FA
:104970002046FFF737FE21697B2920D13846FEF714
:104980003BF82046FFF72EFE7B213846FEF734F831
:1049900021690EB17B29EBD05C2940F006812046CD
:1049A0000191FFF71FFE23690199B8F1000F3CD078
:1049B00001933846FEF727F8019B1946D1E0636E54
:1049C00000222169481C04D0C2B93A2901D07D29AE
:1049D00014D1D4E91921881810F8010C3D2807D109
:1049E000D21A19443846FDF757FF636E013B6366E0
:1049F0002C2118EE100AFDF7FFFFC5E721F020007B
:104A00005B280DD10132C9B218EE100ACDE901328E
:104A1000FDF7F2FF2046FFF7E5FDDDE90132D0E7C3
:104A20005D2808BF02F1FF32EDE7782B06D85B2B3B
:104A30000BD8222B74D053D80A2B4FD0A3F13001BE
:104A4000072900F2AB800323A1E0A3F15C021C2A3A
:104A5000F4D801A151F822F0214B00603D4A0060DA
:104A60003D4A00603D4A00603D4A0060CD4A00601A
:104A7000F94A00603D4A00603D4A00603D4A0060DE
:104A8000094B00603D4A00603D4A00603D4A0060BD
:104A90003D4A00603D4A00603D4A00603D4A00607A
:104AA000014B00603D4A00603D4A00603D4A0060A5
:104AB000F54A00603D4A0060FD4A00600D4B006011
:104AC000054B00603D4A0060754B0060072194F87B
:104AD0004C300C2B65D13846FDF795FF002326E7B7
:104AE000552B13D0AAD8272B1AD04E2BA6D1354838
:104AF00048F07EFC0D21EAE70821E8E70921E6E716
:104B00000A21E4E70B21E2E70C21E0E794F84C20CE
:104B10000D2A07D15C2138460193FDF774FF019BF4
:104B20001946D4E7752B0CBF04230823002116E097
:104B3000204603930191FFF755FD2269104602922A
:104B4000FEF7C2FB002800F04B810199029A09018F
:104B500010460191FEF7F8FB0199039B0144013BCC
:104B6000E6D2481CBAD0B1F5881FB0D3012384F82F
:104B70004C30B3E70223D9E72046CDE90113FFF714
:104B800031FD22690199303A029B02EBC101626951
:104B9000303A072AE5D8013BEED1E2E75C210193E8
:104BA00007E7FF29E2D80D2BE0D1C9B23846FDF75F
:104BB00023FF93E753453CBF032284F84C20C7E60C
:104BC000FF240560082505603046FEF769FB0646B0
:104BD00020691EB95F2801D07F283ED9092304F13E
:104BE0005005C1B284F84C302846FDF705FF204639
:104BF000FFF7F8FC2069421C1BD128467B4FFDF7CC
:104C0000ECFE0025064657F8041B304624F02FFA28
:104C100000281CD10F35EDB2122D84F84C507FF4D2
:104C2000C1AD734BD3F84433002B0CBF11230F23BA
:104C3000F7E5FEF735FB40B920695F2805D07F28EE
:104C400003D8FEF737FB0028D7D0217CCCE7FFF64E
:104C5000A9AD0135242DD6D1A4E5FEF72BFB68B311
:104C600021692E2935D10B2384F84C3004F15005ED
:104C70000B272846FDF7C7FE2046FFF7B3FC206947
:104C8000431C3FF48FAD002E35D120F02003452B7F
:104C900031D16521284684F84C70FDF7B4FE2046DA
:104CA000FFF7A0FC21692B2901D02D29E7D1284647
:104CB000FDF7A9FE2046FFF795FCE0E723692E2BC0
:104CC00004D16069FEF7F6FA0028C9D10026494DE3
:104CD00031E00A23302984F84C30C7D1636943F0AE
:104CE0002003623B162B9EBF434DDD4005F00105BE
:104CF00005F00106BAE7FEF7D3FA28B121692E299B
:104D00000DD184F84C70D2E72069FEF7D3FA002861
:104D1000F4D123692E2BF1D05F2BCBD042E521F0CB
:104D200020034A2BC3D1ECE7652F01D0632F00D1BC
:104D30000135013601352F7817B12369BB42F3D114
:104D40002046FFF74FFC0FB901236AE5212F07D159
:104D500023693D2BF8D12046FFF744FC3A2360E558
:104D60002E2F0FD123692E2B02D163692E2B01D058
:104D70005D2356E52046FFF735FC2046FFF732FC61
:104D80000E234EE50335334615F8027C632F0FD012
:104D9000652F0DD0194AD35C03F0FD0284F84C3026
:104DA000552A01D0592B13D1636B01336363F9E4A6
:104DB00015F8012C01362169914207D12046FFF7F1
:104DC00011FC3346652FE5D00235DDE7632FFAE7A6
:104DD000562B02D0582A7FF4E5AC636B013BE5E724
:104DE0000123014684F84C3071E600BFC8250560F8
:104DF000B0270020BA2405600120400099250560F5
:104E00007FB501AD0646742085E80E00FDF744FB32
:104E10000446034695E8070043F8046B002583E841
:104E2000070001236FF001021420C4E90A320A22AC
:104E3000C4E90C55C4E90E23FDF72EFB20212064A4
:104E400004F15000FDF751FD294604F16000FDF723
:104E50004CFD236C20461D802561C4E90555FFF7F4
:104E6000C1FB2046FFF7BEFB2046FFF7BBFB2046F9
:104E7000FFF76AFCA36C2046012B1CBF072384F8B4
:104E80004C3004B070BD30B585B0054601AC20464D
:104E9000FFF790FB284694E80E00FFF7B1FF05B03E
:104EA00030BD30B585B00546014601AC20461AF04C
:104EB00065FA2846FDF738FC94E80E00FFF7A0FFDE
:104EC00005B030BD10B5044690B1C368406898473E
:104ED00004F15000FDF738FD04F16000FDF734FDEA
:104EE000206CFDF701FB2046BDE81040FDF7FCBA41
:104EF00010BD0000F8B5054630200E461746FDF7F8
:104F0000E4FA072D04460570C66001D0012D0FD1CB
:104F1000B368C3F30F13A38207F090FF042320614B
:104F200020202783E384FDF7B7FAE0622046F8BD2E
:104F3000014B5B5DEFE700BFE02B056010B5044659
:104F4000C06AFDF7D1FA2046BDE81040FDF7CCBAA3
:104F500030B500220446058D954201D8002030BDB1
:104F6000E36A03EBC20043688B42F8D00132F3E7F7
:104F700070B504460D461646FFF7EAFFC0B9E38C4C
:104F8000228D9A4208D30633E06AD900FDF79FFAD2
:104F9000E38CE0620633E384238DE26A591C02EB62
:104FA000C300218502F833600023456043704380CD
:104FB00070BD034618465B68002BFBD1FFF7C8BFE6
:104FC000F8B544680E462CB9F8BD042BFCD1052376
:104FD0000370F9E7254628466D68002DF4D0776800
:104FE0003946FFF7B5FF0028F5D00378043B022BC4
:104FF000EAD806231D463370002239462046FFF7C3
:10500000B7FF0378002BE0D105706468F4E7036A0A
:105010001B8B012B1EBFC368C918C1607047836A10
:1050200010B50446DB6F406A9847238B226A013330
:10503000918C9BB29942238338BF938410BD038B1C
:10504000013B10B503830446836A406AD3F8843079
:10505000984720460121BDE81040FFF7D8BFF7B5BB
:105060001E4659B111F0030511D14F68FCB29442AC
:105070000DD13F0A01F10804BD4201DB03B0F0BDD0
:1050800054F8041B01350190B0470198F4E733460A
:1050900003B0BDE8F04018472DE9F04F04460D4637
:1050A00098462DED028B08EE102A83B01BB1CB8AF7
:1050B00043F00803CB8218EE103AEB83236ADA8AB6
:1050C00042F03002DA821B78002B4CD1A36A18EE32
:1050D000102A2946606AD3F8B4604346B44603B048
:1050E000BDEC028BBDE8F04F6047DB6A03EBC60BFB
:1050F00013F83630053B012B1DD84FF0000917E09F
:10510000EB6A03EBC90213F83930062B0ED1DBF83A
:1051100004105368994209D1A36A0AF1010ABBF845
:1051200002205B69606A1F460023B84709F1010944
:105130002B8D4B45E4DC0136236A1A8DB242D4DC58
:10514000BAF1000FC2D0A36A5246CDF800802946BA
:10515000D3F8B86018EE103A606AB04703B0BDECFF
:10516000028BBDE8F08F0026B246E5E7F8B50E46A3
:1051700011461A4600230446857807698370036147
:105180000E4BFFF76CFF6368BBB9618A51B1228A8D
:1051900042B9A36A606AD3F8A0309847A36A606AEC
:1051A0005B6C9847238A3146628A2046FFF774FF7A
:1051B000003D276118BF0125A570F8BD255E006080
:1051C000024B9D228968FFF74ABF00BF297A006021
:1051D000024B6B228968FFF742BF00BF3577006042
:1051E000836A002110B50446D3F88830406A984796
:1051F000A36A606A10215B6B9847A36A606A012109
:10520000D3F8CC30984720460321BDE81040FFF783
:10521000FEBE38B5836A04460022406A9B6C9847FC
:10522000A36A606AD3F8C05000231A461946A847FB
:105230002046BDE83840FFF7D3BF836A0022896863
:105240005B6D0909406A1847836A89681B6C406A6C
:10525000184710B50446084611461A46FFF74AFE9D
:10526000236A436000238360E3690BB9E06110BDEA
:105270001A469B68002BFBD19060F8E770B5437825
:1052800005460C46012B06D1036A0A4602211B8BF8
:10529000FFF7DFFF2061A268284621694C23BDE8A3
:1052A0007040FFF763BF70B51346427805460C4661
:1052B000012A04D10A460721FFF7CBFFA061A669A6
:1052C00028464623E2683146FFF750FFB08A70BD9A
:1052D0002DE9F04F85B005460C4600AF11B901210C
:1052E000116015E011F003081BD10B79682B07D171
:1052F000CB681B0913608C68002CF0D04FF00108BC
:1053000004F00F03022B0FD12109B8F1000FE7D0F1
:10531000AB6A0022686A1B6B98471437BD46BDE82C
:10532000F08F4FF00008EBE7B8F1000F02D1A3684F
:105330001B091360666804F1080A360AD14606F1B3
:10534000FF3B0AEB860659F8040B0009FDF702FA49
:10535000B1458344F7D10BF1070323F00703ADEB0D
:10536000030D6B4699465AF8040B07F10C013B609C
:105370000009FDF706FAFA68014648467A6023F00C
:10538000FBFD7A68B2453B68914418D159461846EE
:10539000FDF72CF9AB6A014600221B6B686A98473F
:1053A000B8F1000FB9D00C34A642B6D054F8041BA3
:1053B0000022AB6A0909686A5B6D9847F4E74FF011
:1053C0002E0209F8012BCEE731B101F00303026888
:1053D000134304BF0B6803607047000038B543688F
:1053E0000D460446114653B905480AF077FA294696
:1053F000606004F10800BDE83840FFF7E5BF38BD44
:10540000004C05602DE9F04F0E460162002142700C
:105410008DB00446C16015463378072B05D0814A0C
:10542000FFF7DCFF0DB0BDE8F08F012A05D0036B5C
:10543000021D2946C06A1B6898476378D6F80C900D
:10544000032B10D10BAA462109F10C0048F0C4F837
:10545000236B01460B9A9B68E06A984763687083E8
:10546000002B40F0AE80D9F81010B9B101F00F0652
:10547000022E0FD10B09752B3CD006D83E2B3BD00A
:105480005E2B0CD0684A2046CAE7B3F59D6FF9D170
:10549000032604E0654A2046FFF7A0FF0226D9F85C
:1054A00014304FF0000A0AAA192109A8099348F0FC
:1054B00093F80690069B9A4520D16378012B15D965
:1054C000236B3146E06A5B6898476378042B0DD103
:1054D000206A05210396438BE26A02930023CDE9FB
:1054E0000033D2E90232006907F0C2FC6368002B86
:1054F00067D197E70026D2E70126D0E70A9B4FEA5B
:105500008A0B53F82A100B79082B02D10AF1010AF1
:10551000D0E7052B01D0464AB5E7CB68002BFAD17E
:105520008B681A792C2AF6D19F6807F00F02022A9D
:10553000F1D1DB680593002BEDD09807EBD11B79F7
:10554000302BE8D1059B0BAAA4213F0903F10800E9
:1055500048F042F840F2034380469F421BD10128A5
:1055600005D10B9A136803F00F03022B04D0314AC4
:105570000A9B53F80B1086E7E168012D01F1010346
:10558000E36019D01268236B1209E06ADB68984760
:1055900090B9294AECE7B7F5547F16D1012803D119
:1055A0000B9B1968CA0701D4244AE1E7012D03D0F7
:1055B0004910E06A03F071FA6368002BA6D0DDF8A9
:1055C0001490D9F80030A3602CE740F28F339F424B
:1055D0001CD1012804D90B9B196811F0010701D1D6
:1055E000174AC5E7012DE7D049100B9B53F8272038
:1055F000D30701D4134ABBE701375210E06A079181
:1056000003F052FAB8450799EFD1D5E7012DD3D071
:10561000236B02463946E06AD3F810B00B9BD8479B
:10562000CAE700BFE72B05600B2C0560182C05604E
:10563000402C0560632C05607F2C05608F2C056075
:10564000AB2C0560D02C0560014AFFF7C7BE00BF38
:10565000F22C05600B79092B4FF6FF7370B508BF6C
:10566000858A044618BFC58A9D4202D1064AFFF7C3
:10567000B5FE218B628BA36A8A1A606A29469B6FEA
:10568000BDE87040184700BF0F2D056013B50446F4
:10569000B9B101F00F03022B0FD10A091046019294
:1056A00008F04CF80028019A05DA074907480AF083
:1056B0009FF96060002002B010BD054AFFF78EFE22
:1056C000F8E70846F7E700BF2F2D05602C4D056071
:1056D0001F2C05602DE9F8430646006A0F469046E8
:1056E000C48A14F0020506D0334A39463046BDE874
:1056F000F843FFF773BE01F00F02022A17D1B37807
:1057000009097BB1828B013282834FF001090029A4
:105710004FD00022FFF72CFC03780446002B34D036
:10572000264AE2E7428B1D4601324283EDE70A79C1
:105730000D4642450BD18968B37809091BB1838BAB
:1057400001338383E1E7438B01334383DDE79A42EF
:1057500013D1B578002DC7D10123B370896841B347
:1057600001F00F0244F004044FF00309022AC4823E
:105770001CBF0D46A9680909C9E7896844F00204FD
:105780004FF005090909C482C1E7042380F801909C
:105790000370336A1B8B032B0BD1B8F1480F08D170
:1057A0003DB1E9683046FFF771FF637843EA0013C3
:1057B0006370BDE8F88300BFDA260560412D0560FF
:1057C0004F234E22FFF786BF49234822FFF782BFAF
:1057D00010B404460B46006A6278012A03D15DF8D2
:1057E000044BFFF7C5BBA16A0246606A14315DF83D
:1057F000044B02F04FBC000070B505460C46002972
:105800002DD0CA0706D5836A49109B6B686ABDE82C
:10581000704018478B0716D004F00F040909022CBA
:105820000AD0062C0CD0062919D0836AC9B2406A66
:105830005B6BBDE870401847BDE87040FFF7C8BF1C
:10584000836ADB6BE2E7836A09681B69406A9847F1
:105850002279034B2146284653F82230D7E770BD02
:10586000EC2F05602DE9F74F04460D4616461F46FE
:10587000284647F045FE20B1CEB9A36A3946DB6E13
:105880004CE0284647F00CFE08B186B1F5E7002D44
:1058900055D0AB0753D16B684FEA132BDBB21E2BED
:1058A0001BD1F6B1083505EB8B0B5D450DD103B06F
:1058B000BDE8F08F43465AF8041B2046019209F1D7
:1058C0000109FFF7CFFF019A19E03B46324655F830
:1058D000041B2046FFF7C6FFE7E71F2B23D1002E4E
:1058E000E0D0D4F80C8005F1080A4FF0000986F0EA
:1058F000010208F10103E3600BF1FF330093009B09
:105900004B45D7DC0BF101013B463246204655F8AA
:105910002110FFF7A7FFA36A4146DB6A606A03B064
:10592000BDE8F04F1847202B03D1AD6886F0010683
:105930009EE72D2B03D1AB68002BA6D19CE729460F
:105940002046FFF759FFA36A3A4631461B6F606A4B
:1059500003B0BDE8F04F1847026A38B51278044624
:105960000B46072A06D0022A04D0154ABDE8384063
:10597000FFF734BD9D6885B9A36A1021606A5B6B2F
:105980009847A36A0021606AD3F8CC309847204634
:105990000121BDE83840FFF73ABBAB070BD12B79AB
:1059A000AF2B08D12046A968FFF726FF2046BDE8A7
:1059B0003840FFF715BC29462046FFF71DFFE0E7FA
:1059C000562D056070B5437804461546CE68012B08
:1059D00006D1036A0A4629461B8BFFF73AFC706121
:1059E0000023716920461A46FFF756FBF1682046EE
:1059F000FFF702FF062D05D1A36A0021606AD3F8E4
:105A000088309847A36A0121606AD3F8BC5000230C
:105A1000AC461A46BDE87040604738B505460C46AE
:105A2000C968FFF7E9FEA1682846BDE83840FFF7DE
:105A3000E3BE0B79342B70B504460D4610D189684E
:105A4000FFF7DAFEED68AD6885B9A36A1021606AD8
:105A50005B6B9847A36A04220221D3F8A0301AE0B6
:105A6000836A1021406A5B6B9847ECE7AB071FD154
:105A70002B799A2B13D1A36A1021606A5B6B98472C
:105A8000A9680029E6D02046FFF7B6FEA36A0422E3
:105A90000321D3F8A030606ABDE8704018479B2B03
:105AA00006D1A9682046FFF7A7FEEB689968E8E7EA
:105AB00029462046FFF7A0FECCE710B504468968CA
:105AC000FFF79AFE0021A36A606A1B6DBDE81040D3
:105AD000184700002DE9F7438D680446164645B97E
:105AE000FAB1836A02222946D3F8A030606A984747
:105AF00017E015F0030740F084802B79372B13D182
:105B000032B1836A02220121406AD3F8A03098475B
:105B100020462946FFF770FEA36A606AD3F8A430D6
:105B2000984703B0BDE8F0839F2B6AD1EB681A79E0
:105B3000A12A56D1A22101AA03F1080047F04CFD89
:105B4000A968804611B38B0720D10B79372B1DD163
:105B500036B1A36A411C0222606AD3F8A03098478C
:105B6000A9682046FFF748FEA36A4FF00109606A62
:105B7000D3F8A430984747450ED1B9F1000FD0D1E2
:105B8000A36A0322791CD3F8A030AFE720464FF078
:105B90000009FFF731FEEEE7019B53F8271099B19A
:105BA0008E0711D10E79A6F13700464246412046B4
:105BB000FFF722FEB9F1000F0FD03EB9164A294671
:105BC0002046FFF70BFCACE70026F0E7A36A606A0B
:105BD000D3F8A43098470137CDE7002EFBD00F4A09
:105BE000EDE7AB684BB19A0707D11B79372B04D18E
:105BF00004222946FFF7E6FE93E7052229462046C0
:105C0000F8E729462046FFF7F7FDA36A03220121A2
:105C1000D3F8A0306AE700BF6F2D05608C2D0560BA
:105C20000122FFF757BF70B50D46C9680446FFF75C
:105C3000E3FDA968A36AC1F30711606AD3F898303D
:105C4000342916BF40390221C9B2BDE87040184757
:105C5000F8B54F680C46002689683F0A0C340546A3
:105C6000FFF7CAFD02360834B74200DCF8BD54F82D
:105C7000041C2846FFF7C0FD54F8081CAB6A09094C
:105C8000686AD3F89C302539C9B29847EAE72DE90C
:105C9000F0414E680C4601278968A6F10D080C34C6
:105CA000360A05465FFA88F8FFF7A6FDB74201DB22
:105CB000BDE8F08154F8041B2846FFF79DFDAB6A50
:105CC0004146686AD3F89C3001379847EEE72DE9E2
:105CD000F0414E680D4689680446360A0127FFF7F1
:105CE0008BFD032E89BFD4F80C804FF0000808F11B
:105CF0000103E3607B1C9E4222DC032E55DDE56838
:105D0000606A6B1C2946E360A36ADB6E9847A36A4E
:105D10004146606ADB6A9847A36A0121606ADB68D2
:105D20009847A36A606A5B6E9847A36A606A1B6EB5
:105D30009847A36A2946606ADB6ABDE8F0411847C4
:105D4000023729692046FFF757FDB74207DAA36AF1
:105D5000606A9B6D9847A36A606A9B6E9847EB6880
:105D6000A26A03F00F01606AD2F89C200A2911D1BF
:105D7000C3F30713262B16BF353B0621D9B2904734
:105D8000B74205DAA36A42460021606A5B6F984712
:105D90000835AFE71979852901D13221EFE79B68F2
:105DA0000BB90721EBE73321E9E7BDE8F08110B536
:105DB00004468968FFF720FD0321A36A606AD3F8CF
:105DC0009830BDE8104018472DE9F0474E6804466A
:105DD000D0F80C8001F108055FFA86F90027360A31
:105DE000A9F11E03D3F1000949EB030908F10103EE
:105DF000C360B74206DBA36A4146606ADB6ABDE85E
:105E0000F0471847013755F8041B2046FFF7F4FC0C
:105E1000B742F0DAA36A42464946606A5B6F984728
:105E2000E7E7000001F00F03022B70B504460FD026
:105E30000B79492B01D04F2B02D10123A37070BDE8
:105E40004A2BFCD0502BFAD0482B0DD10D696DB9DF
:105E5000A378002BF3D1638A002BF0D020461D4A93
:105E6000BDE87040FFF7BABACD68F0E7A37843B356
:105E7000238A8E6801339BB2012B23820ED1618A63
:105E8000D4E90903D1B1D3F8A03000229847A36A1E
:105E900002220021606AD3F8A030984729462046A4
:105EA000FFF7AAFCA36A606A3109DB6B9847A36A13
:105EB000606AD3F8A430BDE8704018475B6C98471F
:105EC000E5E7638A2946204601336382BDE87040D6
:105ED000FFF792BCAB2D05602DE9F041C568044683
:105EE000D1F80C800E46AB1C00226F1CC3602B4601
:105EF000D8F80810FFF7B6FCB1682046FFF77CFC25
:105F0000A36A3946606ADB6E9847A36A2946606ACD
:105F1000DB6A9847A36A606A4FF0FF31DB689847F5
:105F2000D8F80C102046FFF767FCA36A3946606A70
:105F3000DB6ABDE8F04118472DE9F047C668044622
:105F4000D0F814A00D46B31C06F10108B0F81A9061
:105F5000C360038B8682A0F816804383886847F06D
:105F6000CFFAF8B9E7687B1CE360A86847F098FAB5
:105F700020B9A36A4146606ADB6E9847A36A394636
:105F8000606ADB6A9847E9682046FFF735FCA36A38
:105F90004146606ADB6A98473B460122A968204671
:105FA000FFF760FC29692046C4F814A0A4F81A90F1
:105FB000FFF722FCA36A3146606ADB6ABDE8F0475E
:105FC00018472DE9F347C66804460D46731CC360A5
:105FD000886847F095FA024610BBE76820467B1CAC
:105FE000E3603B46A968FFF73DFC2046E968FFF700
:105FF00003FCA86847F054FA00BB2B690BB96B6926
:106000004BB1A36A606A9B68984720B9A36A31467E
:10601000606ADB6E9847A36A3946606ADB6A984714
:1060200001AA712105F11000002747F0D5FA814639
:106030004F450BD169692046FFF7DEFBA36A314665
:10604000606ADB6A984702B0BDE8F087019B53F8AD
:106050002780D8F8080047F053FA024620BBD4F84E
:106060000CA020460AF10103E3605346D8F808105B
:10607000FFF7F8FB2046D8F80C10FFF7BDFBD8F867
:10608000080047F00DFA0028D8D1A36A606A9B681F
:10609000984720B9A36A3146606ADB6E9847A36AC5
:1060A0005146606ADB6A98470137C1E770B58D6871
:1060B00004463DB9836A2946D3F8C830606ABDE812
:1060C00070401847AB070ED12B795E2B0BD1A96816
:1060D000FFF792FBE9682046FFF78EFBA36A0221D7
:1060E000D3F8C830EAE729462046FFF785FBA36AC4
:1060F0000121D3F8C830E1E710B504468968FFF7FD
:106100007BFBA36A606A1B6EBDE8104018472DE94F
:10611000F0414E6801F108040546360A04EB860793
:10612000BC4208D1AB6A3146686A0022D3F8A0307D
:10613000BDE8F041184754F8041B2846FFF75CFB04
:10614000EEE74B682DE9F04105460E461F0A01F1C6
:1061500008080024BC4201DBBDE8F08158F8041BAC
:106160002846FFF749FB6B6843B1023405F108008C
:1061700056F82410BDE8F041FFF726B90134E9E7ED
:1061800010B50446FFF7DDFF2221A36A606AD3F849
:106190009C30BDE81040184770B58D68044645B97D
:1061A000836A01222946D3F8A030606ABDE87040B6
:1061B0001847A9071ED16B68DAB2922A1AD11B0AB6
:1061C000022B0CD1EB6853B19A0708D11B79AC2B89
:1061D00005D129460322BDE87040FFF7F3BB2946ED
:1061E0002046FFF7AEFF6968A36A0122090AD3F8C7
:1061F000A030DAE729462046FFF7FEFAA36A01221B
:10620000D3F8A0301146D0E7184B2DE9F041D3F870
:10621000447304460D463FBBC6680122731CC3602D
:1062200033468968FFF71EFBA36A1F2101229B6981
:10623000606A9847E96851B12046FFF7DDFAA36A22
:106240003A460121D3F8BC503B46606AA847A36A8E
:106250000121606AD3F8C8309847A36A3146606A62
:10626000DB6ABDE8F0411847BDE8F081B0270020A7
:10627000026A10B512780446072A04D00A4ABDE81B
:106280001040FFF7ABB8896859B9836A1021406A9A
:106290005B6B9847A36A606AD3F8C430BDE81040CE
:1062A0001847FFF7A9FAF5E7D92D05608968034675
:1062B00010B441B9826A406AD2F8A0400A46234627
:1062C0005DF8044B18474A68120A022A0BD1CA68C3
:1062D0004AB1940707D11279AC2A04D106225DF89D
:1062E000044BFFF76FBB18465DF8044BFFF70FBF79
:1062F00010B4026A044640780B46012804D11046C7
:106300005DF8044B01F0B7BEA16A606A1C315DF80C
:10631000044B01F0BFBE00008B072DE9F14F04468E
:106320000D46164611D001F00F03022B16D1D707E8
:106330004FEA111104D401B0BDE8F04FFFF7D8BF08
:1063400001B0BDE8F04FFFF743BA4968CBB22D2B3F
:106350007BD00BD8062B0DD02C2B12D04E4A2946C1
:10636000204601B0BDE8F04FFFF738B82E2B7FD0A4
:106370009D2BF3D1002EF1D105F10802090A204628
:106380007BE0022A02D0A968FFF736FAEF68002FF7
:10639000E4D017F00309E1D17B68B846DAB28E2A5F
:1063A0000DD1022E4FEA132805D007F1080A08F193
:1063B000FF3BD94511DB08F1010857F8288098F810
:1063C0000430312B24D1022E0FD1A36A606A9B6E58
:1063D0009847A36A1B6D012115E05AF8041B20465B
:1063E00009F10109FFF708FAE3E7D8F80810204699
:1063F000FFF702FA012EA36AECD1DB6D606A9847C1
:10640000A36A00211B6D606A01B0BDE8F04F184718
:10641000322BA3D1012ED4E909030CD19B6D9847EF
:10642000A36AD8F8081000225B6D0909606A01B000
:10643000BDE8F04F1847022E01D15B6E9847A36A62
:106440000122D8F808105B6DEFE7AA68002A85D012
:10645000002E83D15168090A022907D1D3682BB1D4
:10646000980703D11B79AC2B3FF478AF083286E74D
:10647000002A7FF473AFA96821B901B0BDE8F04FDD
:1064800000F074B88E0703D10B790A46922BE1D045
:1064900005F10802012172E7F32D05602DE9F047AF
:1064A000C7681E4604460D46BB1C3946904607F198
:1064B0000109C360836A406ADB6A9847A36A494658
:1064C000606AD3F88C309847A96800222046FFF70D
:1064D00023FF2D69002D2DD141462046FFF78CF971
:1064E000236AA06A197806291DD1D0F8CC30294634
:1064F000606A984720460121FEF789FDA36A606A19
:106500001B6E9847A36A3946606ADB6E9847A36A98
:10651000606A4946DB6A9847A36A606AD3F890309C
:10652000BDE8F0471847B200D0F8A850606A0532BD
:10653000A847E7E72B79AD2B07D1A9683B46002296
:106540002046FFF78FF9ED68C4E7E9682046FFF7BA
:1065500053F9A36A606A0121D3F888309847731C05
:10656000424629462046FFF799FFCBE72DE9F8433D
:106570004FF0FF3704460E469046002501EB070911
:10658000B5420CD17B1C05D1A36A3146606AD3F8B1
:10659000AC3098470025B5421CD1BDE8F88358F8C7
:1065A000251079B18A070DD10B79222B0AD1013739
:1065B0000AD1A36A2F46A9EB05022946D3F8B030C9
:1065C000606A98470135DBE72046084ABDE8F84392
:1065D000FEF704BF58F82510AF424FF000022046E6
:1065E00008BF89680135FFF797FED4E70E2E0560D6
:1065F0002DE9F7430446904699460F4629B91946B6
:1066000003B0BDE8F043FFF7F7B8C668731CC3607A
:1066100015684DB315F0030226D12B797B2B23D1BE
:10662000A9680192FFF7E8F8019A31462046FEF783
:10663000F6FC019AE9682046FFF76EFE08F10402B5
:106640004B46791E2046FFF7D3FFA36A3146606AA6
:10665000D3F88030984703212046FEF7D8FC03B0DA
:10666000BDE8F043FEF7EBBC29462046FFF7C4F82F
:10667000204600223146FEF7D2FCA36A606A1B6EF8
:106680009847DBE737B50C46054601AA7A2104F1A5
:10669000080046F0A1FFE3680146019A2846FFF78B
:1066A000A7FF03B030BD8B6803F00F03022B2DE969
:1066B000F04F04460E462DED028B87B040F0058169
:1066C000CB68002B00F00181980740F0FE801A791A
:1066D0002C2A40F0FA809A6802F00F01022940F05B
:1066E000F48012097C2A40F0F080DB681A79302AA5
:1066F00040F0EB809B6805AAA42104A8049346F00F
:106700006BFF431E022B00F2E080059901280A6806
:1067100000F0CD800228D1F804A000F023818D681C
:10672000E90740F1D2806B0800F0CF8032B19307C7
:1067300004D11179A639022940F2C780BAF1000FBD
:1067400008D01AF0030F05D19AF80410A6390229CF
:1067500040F2BB80B3681AF0010B776908EE103A7B
:106760003369218B08EE903A6369E6680293638B84
:1067700006F10208618306F10401019306F10103A9
:1067800006F10309A6820393E382E16005D1514635
:1067900020460392FFF730F8039A11462046FFF790
:1067A0002BF8A26A4946606AD26E9047A26A4146B7
:1067B000606AD26A9047A26A606A926D904700222E
:1067C00018EE101A2046FFF7A7FD18EE901A204683
:1067D000FFF712F8A26A711C606AD26A90472946D4
:1067E0002046FFF709F8A26A0E21606AD2F89C20C1
:1067F0009047A26A4946606AD26A9047A26ABBF192
:10680000000F58D1D36D606A9847A36A606A5B6EC7
:106810009847002DA36A606AACBF00210121D3F81C
:106820009C309847A36A424601211B6F606A9847D3
:10683000029B6361019B6383002F44D0A36A606A5B
:106840001B6E9847BBF1000F03D1A36A606A1B6EF1
:10685000984739462046FEF7CFFFE568606A6B1C13
:106860002946E360A36ADB6E98478BF00101A36AB7
:106870000131606ADB689847A36A3146606ADB6A67
:106880009847A36A606A1B6E9847BBF1000F03D15B
:10689000A36A606A1B6E984727B1A36A2946606A9B
:1068A000DB6A984707B0BDEC028BBDE8F08F9246DB
:1068B0000325024642E7606A926D904751462046A2
:1068C000FEF79AFFA5E73D46D6E7E5682046238B0D
:1068D000B4F81A906F1C63836FEA4543D4F814A090
:1068E00005F102086FEA5343E782A382EB1CE360E1
:1068F000F168FEF781FFA36A0121606AD3F888304E
:106900009847A36A3946606ADB6A9847A36A41469A
:10691000606AD3F88C3098470022B1682046FFF7B0
:10692000FBFC20463169FEF767FFA36A606A9B683B
:10693000984720B9A36A3946606ADB6E9847A36A14
:106940004146606ADB6A9847A36A606AD3F8903070
:10695000984771692046C4F814A0A4F81A90FEF76D
:106960004BFF9AE70325E1E62DE9F74F04469046F1
:106970000F4629B9194603B0BDE8F04FFEF73CBFFA
:10698000C668321D06F1010A06F1020B06F1030981
:10699000C260D8F80050002D00F0F28015F003021C
:1069A00040F0EE8029797B2940F0EA80A968CDE9A2
:1069B0000032FEF721FFA16A606A896D8847A8212D
:1069C0002046FEF726FC019AE9682046FFF7A4FC62
:1069D000009B3146204602220093FEF720FBA26A6C
:1069E0000321606AD268904708F10402009B791E77
:1069F0002046FFF7B9FFA36A606A6FF00201DB6807
:106A00009847A36A1021606A5B6B9847A36A606A23
:106A10005B6E9847A36A5146606ADB6E9847A36A2B
:106A20003146606ADB6A9847A36A606A9B6D984743
:106A3000A36A0122606A9B6921219847A36A606A60
:106A40000821D3F89C309847A36A5A460021606A0F
:106A50001B6F9847A36A606A9B6D9847A36A606A38
:106A60009B6E9847A36A606A5B6E9847A36A002290
:106A7000A921606A9B6C9847A36A606A9B6E9847DD
:106A8000A36A606A9B6E9847A36A606A9B6D984789
:106A9000A36A00220A21606A5B6D9847A36A606A54
:106AA0005B6E9847A36A606A10215B6B9847A36A84
:106AB0000321606AD3F8C05000231A46A847204635
:106AC000FEF78EFBA36A4A460021606A1B6F984757
:106AD000A36A606A1B6E9847A36A606A10215B6BA9
:106AE0009847A36A4946606ADB6E9847A36A606A62
:106AF0000221DB689847A36A5946606ADB6A9847B7
:106B0000A36A606A9B6E9847A36A606A9B6E984707
:106B1000A36A5146606ADB6A9847A36A0022606AEA
:106B20009B6CA9219847A36A1021606A5B6B984708
:106B3000A36A606A9B6D9847A36A606A9B6D9847D9
:106B4000A36A0321606AD3F8C05000231A46A847FD
:106B50002046FEF745FBA36A606A1B6E9847A36A4E
:106B6000606A4FF0FF31DB689847A36A606A494664
:106B7000DB6A9847204603B0BDE8F04FFEF75FBAE6
:106B8000294620460093FEF737FEA26A606A926D9E
:106B900090472046A821FEF73CFBA26A606A126E6D
:106BA000904715E72DE9F041CD6804460E4635BB08
:106BB0000378BBB1036A1D78A5B9CF21FEF708FEA3
:106BC000B1682046FEF718FEA36A2A460121D3F8D1
:106BD000BC602B46606AB047A36A606A1B6EBDE862
:106BE000F0411847B1688B0700F09A8001F00F035D
:106BF000022B40F09C802046FEF7FEFDECE7AF073D
:106C000040F099806B68DAB25B2A14D1ED68002DF0
:106C100040F08F80006A0378072B40F088808968F5
:106C200001F00F03022B40F082800422BDE8F04106
:106C3000D140FEF79DB9562A13D101228968FFF78A
:106C40006BFBE9682046FEF7D7FDA968A36A09092E
:106C5000606AD3F89C303F39C9B298470222B168C4
:106C600059E0572A65D11B0A5F1E013355F82310DE
:106C7000FEF7C2FD002F03DDA36A606A9B6D984793
:106C8000B1680835002600222046FFF745FBBE42CA
:106C90004DDA0136BE4203DAA36A606A9B6D9847FB
:106CA000002255F8041B2046FFF736FBEFE76B6820
:106CB000DAB2062A3FD1B768002F3CD0B8073AD1E4
:106CC0007A68D1B2062936D11B0AB3EB122F32D122
:106CD000022B30D1BB6823B1990702D11B79222B3B
:106CE00029D0FB6823B19A0702D11B79222B22D02D
:106CF000A9682046FEF780FDE9682046FEF77CFD86
:106D0000A36A606A5B6E98470022B9682046FFF765
:106D100003FB0022F9682046BDE8F041FFF7FCBA0A
:106D200000293FF468AF0B793A2B7FF464AFBDE8DC
:106D3000F081AB07BBD029462046FEF75DFD00225F
:106D40008DE700000023032A2DE9F04104460D469B
:106D5000164642700162C36080F8342002D1C08EB2
:106D600028BBA0634FF00008A36A31462A461B687F
:106D7000606AA4F83680984706212046FEF747F956
:106D80006778EE68012F04BFA5F82280A5F824805B
:106D90008EB1B2070FD133793F2B0CD1B168FEF71A
:106DA0002BFDA36A606AD3F8C430984730E08000B6
:106DB000FBF78BFBD5E72B784BB931462046FEF726
:106DC0001BFDA36A5B6B1021606A9847E9E7072BFC
:106DD00024D1012F12D1002346222046A3705E4BFE
:106DE000F168FEF73CF92B8B032B07D13169204664
:106DF000FEF74CFCEB8A43EA8010E882204671697A
:106E0000FEF7FAFCA36A606A9B6898470028D8D00E
:106E1000A36A606A5B68BDE8F0411847022B1BD18A
:106E2000A36A31681B69606A98476378012B07D1B0
:106E300000234C222046A370484BB168FEF70FF99F
:106E4000F1682046FEF7D8FCEB8ADB07A9D5A36AD8
:106E5000606A1B6E9847B4E7033B032B4FD8012FA2
:106E6000D6F80C8005D104223946206AFEF780F856
:106E70006F83A36A31681B69606A98472B78032B7C
:106E800024D1A36A0122D3F8A0300021606A984778
:106E90002B78062B28D1A36A606A5B6C9847012186
:106EA0002046FEF795FCA36A606A5B6C9847A36A6C
:106EB000606A5B6C98470023B26841462046FFF742
:106EC000EDFA2B78062B7FF46CAF7AE7042B04D114
:106ED000A36A0222D3F8A030D7E7052BD8D1A36A42
:106EE0000322D3F8A030D0E720460121FEF770FC42
:106EF000A36A0121606AD3F888309847DBE7012F45
:106F000004D104220A212846FEF732F81721204630
:106F1000FEF75EFC16212046FFF7EAF9B168A36A86
:106F20000909606ADB6B98471A212046FFF7E0F9F0
:106F300031692046FEF760FC0A212846FEF708F872
:106F40000378042BA36A3FF43DAF5D690A214288B0
:106F50000023606AA84724E7C9570060C157006052
:106F600001F00F03022B70B504460D46164602D001
:106F70000B4AFEF733FA31462046FEF73DFCA36A82
:106F8000606A9B6D9847266A290920463378033B3F
:106F9000032B9CBF73682362FFF7AAF9266270BDBA
:106FA000F32D05602DE9F04F002787B04FF0010B5E
:106FB0000446B9463E46B84603A81D46CDE902211F
:106FC00005AAA42146F008FB0190019B9F4211D124
:106FD00026B1A36A4946606A9B6B9847029AD4E936
:106FE0000903002A73D0D3F8C040334642462946ED
:106FF000A04713E0059B53F827A0BAF1000F5BD020
:107000001AF0030F58D19AF80420A62A19D1B00714
:1070100007D5304A51462046FEF7E0F907B0BDE8F3
:10702000F08F1D2F01D92C4AF4E70BFA07F246F036
:107030000106DAF8081049EA02092046FEF7DCFBEF
:1070400020E0A72A0ED1A26A46F00206606A526CBE
:107050009047DAF8081008F101082046FEF7CCFB4B
:107060000137B2E7A82A27D1DAF80C2072B19107CC
:107070000CD11179AA2907D192682046DAF80810B4
:10708000FFF76EFF0135EBE7AC290FD0DAF80810F7
:1070900001F00F02022A01D0104ABBE7A26A0909D7
:1070A000606AD26B9047DAF80C10D4E7062251469A
:1070B0002046FEF787FCE5E7B30701D5084AA9E7B4
:1070C000B8F1000F01D0074AA4E75146B5E7D3F85D
:1070D000BC408AE7282E0560372E0560452E0560E6
:1070E000662E05607E2E056070B50D46417804461B
:1070F0001346012903D12A46FEF7ABF86861A36A5B
:10710000606ADB6C98476E690023204631461A4658
:10711000FDF7C2FFA36AB18ADB6B606A9847E96832
:1071200029B18B0703D10B79A32B08BF002120467F
:1071300002230022FFF736FFB08A70BD0023896862
:107140001A46FFF72FBF00002DE9F7430C46896868
:107150000546FEF751FBE668002E58D07768296A8D
:10716000FBB209788E2BA36819BF04F10C06012726
:107170003F0A0836072903F00F024DD1022A49D1F0
:107180001A099A2A4AD132681179302946D192686F
:10719000002A43D10A212846FEF71AFB2A6AD36A3D
:1071A000128D3AB9414A2846316803B0BDE8F04330
:1071B000FEF714B95978C9070FD559682846FEF764
:1071C00007FB022FAB6A0BD8D3F8BC400023022187
:1071D000686A1A46A047012417E0013A0833E0E73D
:1071E000726811793229EFD1B46821793029EBD155
:1071F000916801229B6C0909686A9847A168032479
:10720000002301222846FFF7CDFEA74227D803B06E
:10721000BDE8F0830024F8E7022AFBD140F2B62251
:10722000B2EB131FF6D133681A79302AF2D19C6879
:10723000002CEAD014F00302ECD123792F2BE9D1F2
:10724000AB6A1146686AD3F8BC4013460192A04766
:1072500033682846019A9968FEF73CFCBBE704F1C5
:107260000108A30056F82410B8451AD20A79322A28
:1072700017D13344D3F8049099F80430302B10D14F
:1072800089680022AB6A0909686A9B6C98470023E9
:107290000122D9F808102846FFF784FE08F10104FE
:1072A000B3E72846A046FEF7A7FAF7E79F2E05604A
:1072B000026A0B4610B512780446072A06D0022A45
:1072C00004D0074ABDE81040FEF788B820461946AA
:1072D000FFF73AFF2046BDE81040FDF781BF00BF31
:1072E000B72E0560D1E90212FFF73ABE036A10B566
:1072F00004461A8BFFF7F8FE01462046BDE8104011
:10730000FEF7F6BF036A10B504461A8BFDF7CBFFF4
:1073100001462046BDE81040FEF7EABF2DE9F04FD8
:107320008D6887B004462B79032B0AD12946FFF7D5
:10733000E9FFAA69D38A43F00103D38207B0BDE80D
:10734000F08F026AD28AD20704D4614A2946FEF736
:1073500045F8F3E7162B40F0AE80C668EB6806F1FF
:10736000010B06F102094FEA1318331D06F1030A57
:10737000C360E968FEF740FAA36A606A00229B6C6A
:10738000AA219847A36A606AD3F8C07000231A46FE
:107390001946B84741462046FEF7AAFFE7686369E9
:1073A000BA1C606A0293E260638B228B01937B1CA0
:1073B0006283A26A1946E382D26AA7820393904746
:1073C000012259462046FDF72AFE41462046FEF797
:1073D000FFF92046AC21FDF71CFFA96820460022DA
:1073E000FEF79AFFA26A4946606AD2F894800022AA
:1073F000C047A26A5946606AD26A9047A26A606A28
:10740000D2F8D0209047A26A606A926D9047A26A33
:10741000606A40F2E621D2F818800122C047A26AD1
:10742000606A0821D2F89C209047A26A0021606A15
:10743000D2F870805246C047A26A606A126E9047C6
:10744000A26A3146606AD2F894800122C047A26ADB
:107450005146606AD26A9047A26A0121606AD26886
:1074600090472046FDF7EBFDA26A606AD2F8D4206F
:107470009047A26A4946606AD26A904729692046C5
:10748000FEF7BAF9039BA26A1946606AD26E90476A
:10749000029B3146606A6361019B6383A36ADB6A76
:1074A000984769692046FEF7A7F9A36A3946606ADA
:1074B000DB6A984742E705AA7A2105F1080046F001
:1074C0008BF8EB680146059A2046FFF74DFA35E741
:1074D000D02E05602DE9F04F85B004460026DFF878
:1074E0001CA1019102AA019B4221B14603F10800AF
:1074F00046F072F8236A83461D8B5E450AD1019BD4
:10750000D9680B79032B50D12A462046FDF7CBFED4
:10751000054658E0029B03AA6C2153F8263003F17C
:107520000800009346F058F8039B074619680A09BB
:10753000732A0DD04FF001082046FEF75DF9B845DB
:1075400027D3009BD96859B12046FEF755F907E0CB
:10755000022807D052462046FDF740FF09F10109F5
:107560000136CAE759680B09412B0CD040F2414261
:1075700093420AD040F20752934208D0B3F5567FA7
:10758000E8D10425EAE70125E8E70546E6E7032513
:10759000E4E7039B0022606A53F8281008F1010811
:1075A000A36A09095B6D9847C9E7442B17D18E6818
:1075B0002A4620463146FDF776FEB2690546D38A53
:1075C00043F00103D3820026ABEB0909B1450BD888
:1075D00029462046FEF78CFE05B0BDE8F08F2A460E
:1075E0002046FFF781FD93E7A36A0121606A013617
:1075F000D3F8BC7000231A46B847E7E7F62E0560BB
:10760000F0B58D6885B004460E4605F00F030A2BD1
:1076100006D0002D2FD0AB072DD12B79652B1DD196
:107620000295002503AA652102A845F0D5FF039B1A
:10763000002140F2DA5203EB8000984214D1F26844
:1076400040F22A439A4234D1236A1F78AFB1384AB4
:1076500031462046FDF7C2FE05B0F0BD622B0AD1CF
:10766000AB680293ED68DDE753F8047B97420CBFEB
:1076700001310331E1E70021E1E7A36A606A9B6B16
:107680009847A36A606A0521DB6B9847A36A3A466C
:10769000606AD3F8A0300121984703AA2946204602
:1076A000FDF716FEA36A022239461B6B606A9847F3
:1076B000D2E7A36A0027606A9B6B984706F10C002B
:1076C00002AA6A2145F088FF0646B742D4E90903B9
:1076D00011D1D3F8A0300022314698472946002521
:1076E00003AA2046FDF7F4FDB542D4E909030BD106
:1076F0001B6E9847B0E7029ADB6B52F827200137E0
:10770000916809099847E0E7029A1B6B52F82570C7
:107710000122B968090901919847FB682BB90199C1
:1077200020460135FEF7E4FDDEE71909F8E700BF62
:10773000142F0560836A37B504460D469B6B002104
:10774000406A9847A36A606A10215B6B984701AA58
:1077500029462046FDF7BCFD01992046FEF7C8FDED
:1077600003B030BD10B4026A044640780B460128CD
:1077700004D110465DF8044B00F07DBCA16A606A3C
:1077800024315DF8044B00F085BC00002DE9F04F7A
:107790002DED028B83B0C5681E4604460E9B0F4636
:1077A0000192294608EE103AAB1C012205F1010AAC
:1077B000C360FDF734FC394620460027FEF71CF86D
:1077C000A36A00225146D3F89430606A9847A36AAE
:1077D0002946606ADB6A9847A36A606AD3F8D030AA
:1077E0009847D4F80C8008F10103E360019B9F42A5
:1077F0001BDB2046FDF723FCA36A606AD3F8D43074
:107800009847A36A5146606ADB6A984718EE101AD7
:107810002046FDF7F1FFA36A4146606ADB6A03B0C8
:10782000BDEC028BBDE8F04F18473346D4F80C90FE
:10783000043601371A68009209F10102E260009AE9
:10784000D2F808B0BBF1000F47D1019ABA4237D144
:107850000025A36A606AAB461B6E9847009B2046D2
:10786000D968FDF7C9FFCDB1A26A1021606A526BD9
:107870009047A26A5946606AD26A9047A36A10216B
:10788000606A5B6B984729462046FEF731FD20462B
:107890002946FFF767FF2046FDF7D1FBA36A0122C7
:1078A0004146606AD3F894309847A36A4946606AB3
:1078B000DB6A9847A36A0121606ADB68984795E70D
:1078C00020461F4A1968FDF789FD204603B0BDEC2C
:1078D000028BBDE8F04FFDF7B2BB1BF003052DD1C5
:1078E0009BF804205B46762A03D1DD68DBF808B0FC
:1078F0002D09A36A606A9B6D984759462046FDF79B
:107900007BFFA36A0821606AD3F89C309847A36A7A
:107910004A4600211B6F606A9847002D98D029467F
:107920002046FEF7E5FCD4F80CB020460BF101022E
:107930005946E2600222FDF772FB8FE70025D8E787
:10794000312F05602DE9F043C768164685B00D4616
:107950007A1C394603930446C2600222DDE90C9882
:10796000FDF75DFB039B16BBA36A0321606ADB681E
:10797000984729462046FDF73FFFA36A6FF00201B2
:10798000606ADB689847A36A1021606A5B6B98475E
:10799000A36A3946606ADB6A984720464146FDF78C
:1079A0002BFF204605B0BDE8F043FDF748BB32464B
:1079B00029462046CDF80090FFF7E8FEE3E77FB5C3
:1079C000CD6806460C462B79782B09D1AB6801931C
:1079D000002300931A468968FFF7B4FF04B070BD16
:1079E000742B03AA4FF0770116D105F1080045F07A
:1079F000F3FD2B6902463BB9EB6800933046039BCD
:107A0000A168FFF7C3FEE9E79B683046A1680193D0
:107A1000EB680093039BDFE704F10C0045F0DCFD0D
:107A200000230246E9E7000001F00F03022B2DE9D5
:107A3000F04705460C4604D10909BDE8F047FFF7B9
:107A400091BE002956D011F0030653D10B792C2B8F
:107A500038D18968FDF7D0FEE668002E4AD016F0CE
:107A6000030847D177683346FAB28E2A09D13F0A14
:107A700006F1080907F1FF3AC24510DC013756F854
:107A800027301A79312A12D199682846FDF7B4FEB9
:107A9000AB6A686A02211B6DBDE8F047184759F8C8
:107AA000041B284608F10108FDF7A6FEE4E7322A88
:107AB00020D199680222AB6A686A09095B6DBDE84A
:107AC000F04718472D2B15D18C689CB163681B0AB1
:107AD000022B07D004F108076368B6EB132F10D30D
:107AE000BDE8F087E368002BF4D09A07F2D11B7948
:107AF000AC2BEFD121462846054ABDE8F047FDF7FB
:107B00006DBC57F8041B28460136FFF78DFFE3E7ED
:107B10004F2F05602DE9F04F437885B004460D46A0
:107B2000012B0AD191F80480B8F1100F08D0036A34
:107B30001B782BB9234AFDF751FC05B0BDE8F08F47
:107B400003AA6D2105F10800002645F045FDDFF888
:107B500078900746DFF874A0DFF874B0B742ECD035
:107B6000039B0022206A53F826100909FDF700FA4A
:107B7000B8F1100F0146037813D13BB1032B05D0A8
:107B80005A4629462046FDF729FC08E003230B70DE
:107B90004968206AFDF70DFA08B103230370013626
:107BA000DCE75BB9012301900370206AFDF708FA56
:107BB00001990B78012BF2D15246E2E7062BEED069
:107BC0004A46DEE7672F0560C92F0560AB2F0560C9
:107BD0008C2F05602DE9F04F9BB0AB4D14464FF054
:107BE0000008CDE902011020FAF756FC2B69582253
:107BF00000214360064604A821F0FEF94FF0FF3350
:107C0000012113A809938DF8104045F061FC039BF6
:107C1000012213A8D90041F0020145F04DFC0123D7
:107C20000021436016A809F033FC029A95F8483306
:107C30000021126804A8FDF70CFB054611A800F00E
:107C4000D5FE924B0B9F01900D900E930FB1059CAA
:107C500024B30B9C14B1059B002B3ED041460198E8
:107C600000F0CBFE00270B9CDFF82092DFF820A26B
:107C7000DFF820B2059B002C00F03781002B00F0CC
:107C8000E7800C9B06A8D968FDF79EFB0C9B069A23
:107C90009B8A0399059807F0E7FE29E13B8B0122B7
:107CA000394604A8042B07D1FDF7ACFB079BBF683E
:107CB000984538BF9846C9E7FFF744F83B8D9C428A
:107CC000F4D2FB6A03EBC40113F83430012B02D168
:107CD0003846FDF775F90134F0E7E28A520711D50D
:107CE000218D01390ED3E26A02EBC1025078870779
:107CF00023D53BB1D3E900C792E8030083E8030032
:107D0000C2E900C74FF0000300272384B4F828C05D
:107D1000674518DB00239C454ED1D4F804E0BEF142
:107D2000000F08D00020BEF828B00346584553DBAA
:107D3000002B40F08B80A4688CE7002BD1D1012868
:107D400008BF1346CDE723784FEAC70BD4F82C9031
:107D5000012B09EBC70A05D1DAF804300A2B12D13E
:107D60000137D3E719F837300DD9012B0BD14FF07C
:107D7000030309F80B30238B032B16D0E38A43F05F
:107D80001003E38203E019F80B30032BF3D019F84A
:107D90000B30042B03D09AF80130DB07E0D5238C9D
:107DA0005A1C2284AAF80230DAE7DAF8040005F057
:107DB000C5FC0128EBDCE1E7E26A02EBC30112F843
:107DC0003320052A06D14A78D7075FBF228C4A8024
:107DD0000132228401339EE7DEF82C2002EBC00A38
:107DE00012F83020053A012A15D8002711E0E26A7E
:107DF00002EBC70912F83720062A09D1D9F8042066
:107E00001146DAF804208A4204BFA9F8023001338F
:107E10000137BC45EBD1013088E7E06A00EBC201D5
:107E200010F83200062802D14878C00702D54888E9
:107E30001844488001329445EFD1628B12FA83F2E4
:107E40006283228C12FA83F3238474E70022F2E720
:107E5000238B042B20D10F9B1BB9404604F06AFBF7
:107E60000F9000230322214604A80D93CDF840B0C3
:107E7000FDF7C8FA059B23B90422214604A8FDF7A3
:107E8000C1FAA468F6E600BFB0270020EC30056018
:107E9000E0330560E0360560023B012B21D837B99D
:107EA000434607AA05A911A803F092FC0746CDE9AD
:107EB0000D7A0222214604A8FEF744FF059B002B01
:107EC000DFD10322214604A8FEF73CFF059B002BCF
:107ED000D7D10422214604A8FEF734FF0028F8D0A9
:107EE000CFE7019BCDE90D39E3E7002B7FF4C9AE65
:107EF000DDF81490D5F81080B9F1000F16D0019874
:107F000000F083FD002F41D10F9808B104F027FB4A
:107F1000029845F0B1FA2846AD68FDF70FF8002D3C
:107F2000F9D10598002835D0FAF792FA139C1898E1
:107F3000C4F3DC046400033400EB940024F0030475
:107F40008000FAF7A9FA0444B060F460DDE9144156
:107F500001F1040CA1450BD1189A00239342CED015
:107F6000199951F82300F16841F823000133F5E72E
:107F700051F839303BB1042B1FBF5CF83920DB08C6
:107F8000521020F8123009F10109E3E7384603F0F6
:107F900040FCB9E72A463146404604F0A9FF1BB031
:107FA000BDE8F08F8842F8B505460C4601D10120A6
:107FB000F8BD164B984201D10020F9E79942FBD059
:107FC00005F09EFC0646204605F09AFC8642F3D159
:107FD0000F4B9E4214D16A6863689A42ECD105F156
:107FE0000807083400266B68B342E0D954F8041B34
:107FF00057F8040BFFF7D6FF0028DDD00136F2E773
:1080000021462846BDE8F84005F03CBF643B0560CA
:1080100070650560C900012210B541F002010446F7
:10802000083045F049FA43683BB9A368C3F3DC0361
:10803000013B5B0043F0010343604068C0F34F0025
:1080400010BD37B505460024EB69A34208D805F1F9
:10805000140009F06CF8EC69013C204603B030BD17
:108060002B6A019153F82400FFF79CFF0028F4D1FC
:1080700001340199E8E710B501220446FCF778FFC6
:108080000378012B05D12378012B8CBF0423022315
:10809000037010BD37B504460D46104619460193CE
:1080A000FCF756FF037801995A1E012A06D86B681F
:1080B0000022204603B0BDE830401847032B02D110
:1080C0006B680122F5E7042B2D68428820460CBF1F
:1080D00000230123AC4603B0BDE8304060478079FF
:1080E000003818BF012070474379012B09D08368FD
:1080F000194403695A8C81609142C8BF5984002396
:108100008371704738B50D460021FFF7EDFF4379C5
:10811000012B1EBFC26A036A43F8252038BD6FF0E9
:108120000301FFF7E1BF0421FFF7DEBF6FF002019B
:10813000FFF7DABF4379426A032B11448CBF436BCC
:108140000346416288BF9B18184670474279C36A4C
:10815000032A19448CBF826A0346C16282BFD218C7
:10816000436B9B181846704710B50C460121FFF76A
:10817000EDFF047010BD38B51446FFF7B5FF0121BF
:10818000FFF7E4FF047038BD53220121FFF7F3BF6E
:1081900054220121FFF7EFBF57220121FFF7EBBF68
:1081A00058220221FFF7E7BF59224FF0FF31FFF7B6
:1081B000E2BF5A220021FFF7DEBF5B220021FFF75A
:1081C000DABF5D224FF0FF31FFF7D5BF002915BFA1
:1081D0005F225E2203210021FFF7CDBF3039CAB2F2
:1081E0000021FFF7C8BF62226FF00101FFF7C3BF94
:1081F00010B563224FF0FF310446FFF7BCFF0123A7
:10820000A37110BD01F164024942D2B2FFF7B3BFBE
:1082100001F16702494210B50446D2B2FFF7ABFF45
:108220002269D38A43F00103D38210BD38B50446D6
:108230001D46FFF7A0FF03492A462046BDE8384007
:1082400010F09EBA4D81006037B504460D46C068F7
:1082500019460192FFF7DEFE019A034629462046A1
:1082600003B0BDE83040FFF7E1BF0B46102201210B
:10827000FFF7EABF11320B460121D2B2FFF7E4BF8C
:10828000002A0B464FEA420114BF15221422C1F105
:108290000101FFF7D9BF16320B464FF0FF31D2B2C2
:1082A000FFF7D2BF19320B460021D2B2FFF7CCBF85
:1082B00070B4C4681D4626786388042E04BF6668BF
:1082C00046F823505D1C658070BCFFF7AFBF03F11B
:1082D00028011346CAB20021FFF7A8BF022A02F103
:1082E0002A020B46D2B214BFC1F101010121FFF7EE
:1082F0009DBF03290AD004290BD0002102230A4480
:10830000C94343EA82032F22FFF790BF00210B46A7
:10831000F5E70121FBE70B4630220139FFF786BF65
:1083200010B4144641EA0223312221445DF8044B83
:10833000FFF77CBF012A0B4610B4044608D0022A7E
:108340000ED169224FF0FF315DF8044BFFF713BFE8
:1083500011461B3220465DF8044BD2B2FFF774BFC2
:108360004FF0FF31F5E7F8B51F4605461646FFF713
:10837000BBFE4379022B26D9C46A442E036AC4F19A
:10838000FF2453F8273004F57F0404F1FE041C4455
:1083900012D814F1400F14DB3F2CD4BF0027012763
:1083A000E41BB91C2846FFF7D1FE067077B9442EAE
:1083B00098BF40344470F8BD7F2C94BF002701273C
:1083C000EEE70127ECE700240127EAE7442E6B796A
:1083D00098BF04F58044042B05D1B4F5004F24BFA9
:1083E000012385F8383064F07F03E4114370847012
:1083F000E1E70B4642220021FFF7B5BF002A0B46FA
:1084000002F147020CBF02210021D2B2FFF7ABBF3D
:108410000B464B220121FFF7A6BF0B464A22002143
:10842000FFF7A1BF264BD3F84433022B2DE9F047C9
:10843000044689460ED88669B1420BD9C56A8E1B9F
:10844000436940F2FF77ED1A56EA050304D1E36A67
:10845000C4E90539BDE8F087062E01D90F2D1AD9D8
:108460001F2DAA4628BF4FF01F0A554510D8032ECE
:10847000B04628BF4FF0030801212046FFF75AFEFF
:108480004AEA48130370A5EB0A05A6EB0806DBE7EA
:108490004FF00008F0E7BE42B0464FF00201204620
:1084A00028BFB846FFF746FEAA464FEA181380F8E1
:1084B000018003F070032B4363F07F030370E2E756
:1084C000B027002010B5044631B955224FF0FF31D6
:1084D000BDE81040FFF74FBE022904D1FFF754FE5C
:1084E0002046FFF76AFE56226FF002012046EFE7B2
:1084F000134621B143224FF0FF31FFF734BF44222E
:10850000F9E7134621B145224FF0FF31FFF72BBFAA
:108510004622F9E773B521F4004305460C4616469A
:10852000D2B90A0410D559210193FFF71DFE592134
:108530002846FFF719FE59212846FFF715FE592155
:108540002846FFF711FE019B42220021284602B077
:10855000BDE87040FFF707BF40220021FFF703FF8F
:108560002846210A21F07F013143C9B202B0BDE89B
:108570007040FFF7F9BD322913B513D0332914D158
:108580000124072129390190CAB24FF0FF31FFF7CA
:10859000F2FD01985CB1D322002102B0BDE8104089
:1085A000FFF7E9BD01240621ECE70024EAE702B069
:1085B00010BD23B50B46054611462AB9132202B059
:1085C000BDE82040FFF740BE022A06D10193FFF725
:1085D000DBFD2846FFF7EDFD019B18226FF001013E
:1085E0002846ECE710B41C460B6922435DF8044BA7
:1085F00007BF3222012133224FF0FF31FFF758BE6F
:10860000F8B514461F46D6B2069A05460B693A439A
:108610000BBFC4F10101E14320222122FFF748FEF4
:1086200031462846BDE8F840FFF79EBD10B4044629
:1086300043B90F2A06D8503A01215DF8044BD2B253
:10864000FFF799BD03F12401204613465DF8044B62
:10865000CAB20121FFF7EABD10B404464BB90F2A94
:1086600007D8403A4FF0FF315DF8044BD2B2FFF724
:1086700082BD03F12601204613465DF8044BCAB2C1
:108680004FF0FF31FFF7D2BD70B4DDE90365D2B220
:1086900003EB460443EA062315B101320134D2B29A
:1086A000091B70BCFFF7C2BD07B5CDE900230B461F
:1086B00034220021FFF7E8FF03B05DF804FB07B5A3
:1086C000CDE900230B4636224FF0FF31FFF7DCFFE8
:1086D00003B05DF804FB00000E2910B504460BD171
:1086E0000949C068FFF7ADFC23220346012120465B
:1086F000BDE81040FFF79ABD4131BDE81040CAB255
:108700000121FFF738BD00BF705B056038B5044636
:108710000D461021FFF7E0FF20462946FFF7F2FC47
:1087200002215C22FFF727FD20466FF00301BDE820
:108730003840FFF7D9BC01F110033F2B73B5064653
:108740000C4607D8A1F180020121D2B2FFF713FD38
:1087500002B070BD0DF1050501212222FFF70BFDCE
:10876000294604F07F00E3B2E4112A4605F8010D22
:10877000601C0128F5D8013403F0400312D11BB965
:108780007F2305F8013C951E491B3046FFF7DEFCB0
:1087900001AC01462B46A34208D19DF804205D1B85
:1087A0004255D5E7002BEFD00023EAE713F8012B61
:1087B00062F07F0201F8012BEDE710B50446C068B6
:1087C000FFF73FFC2322034601212046BDE810406D
:1087D000FFF72CBD4379012B70B5044601D1012070
:1087E00034E0C26B0025436A05649B1AC3632069A9
:1087F000038D9D420BD36379032B1AD1606AE36A20
:10880000A06223631844F9F760FE6063E7E7C36A78
:1088100003EBC50213F83530052B08D196780121FA
:108820002046FFF787FC0670236C01332364013573
:10883000DDE7042BD3D1626AD4E90A138A4202D15C
:10884000216B994203D00020A262236370BD94F88B
:1088500038301BB10549064844F09EFEE268C38AE1
:108860005268616B006904F0F3FAB8E7D83005602C
:108870004C4B05602DE9F74F002316460446417125
:10888000378C83608371C362436280F83830B6F8F6
:108890002490B6F81A804FEA8905B6F816A0B6F803
:1088A0001EB04FEA590905F004050AF00F0AC0E9A5
:1088B0000423738C01221F448261B38B974238BF1B
:1088C000174608F003024FEA9808013F1543FA00E3
:1088D0003F0902F07802154347EA090242EA0A0218
:1088E00042EA08021A4352EA0B0234D1012120461F
:1088F000FFF720FC05706379022B17D9D4E90F78B4
:108900007D0008F00103BF09012105F07E054FEA53
:10891000580820461D4358EA070918BF45F080054E
:10892000FFF708FC0570B9F1000FE9D1636A002573
:10893000B18AE363E0682C4FFFF76CFB2A490246DB
:1089400020460FF01DFF738BB28B1344AB4248DD02
:10895000318D002241E065F07F0501212046019321
:10896000FFF7E8FB05703A01019B4FEA8A1502F018
:108970003002BF0805F040054FEA5A0A15430BF0D4
:1089800001024FEA5B0B1543DA005B0802F00802B4
:1089900015434FEA88024FEA580802F004021543D3
:1089A0004FEA49024FEA590902F00202154393E7E0
:1089B000F36A03EBC2035878C0070DD55888A84264
:1089C0000AD15968E0680135FFF724FB39460246B1
:1089D00020460FF0D5FEB6E701329142E8DC0521D2
:1089E000F0E703B0BDE8F08F3581006010B50446B4
:1089F0004420F9F76AFDC46010BD10B50446C1619A
:108A00008800F9F749FD206210BD10B50446006AE0
:108A1000F9F76AFD2046BDE81040F9F765BD10B5CD
:108A2000044601618800F9F737FD606110BD10B59B
:108A3000044611B1C068F9F757FD6069BDE8104000
:108A4000F9F752BD012938B504460D460ADC026922
:108A50004FF0FF314069920020F0CEFA00232560EC
:108A6000636038BD4068F9F717FD6368E060A36094
:108A7000F4E7D0E90032022B11440CBFC368002395
:108A8000416008BF9B18184670470368012BDEBF82
:108A90004268436943F8212070474B1E42684942AF
:108AA000134419404160704738B50C461546FFF72E
:108AB000E0FF10B10444A04200D138BD00F8015BD2
:108AC0002D0AF8E710B50C460221FFF7D2FF10B1CE
:108AD0000470240A447010BD38B50D4604211446B4
:108AE000FFF7C7FF28B105702D0A8470240A45706E
:108AF000C47038BD032994BF144B023970B593BFBD
:108B00005E5CFE2621F00104002446F43541054652
:108B1000FFF7D8FF44B17F2C09D844F430412846F0
:108B200041F08001FFF7CEFFC5E9066470BDA300E8
:108B30004FF2AD21A2012846DBB202F4E0421A4313
:108B400042F45062FFF7C8FFEEE700BFE631056070
:108B5000C16910B5044629B17F290BD841F43041D1
:108B6000FFF7B0FFA169204641F43D41BDE8104048
:108B7000FFF7A8BF8B008A014FF20D21DBB202F490
:108B8000E0421A4342F45062FFF7A6FFEAE71143BE
:108B900041EAC301FFF796BF072A89BF083AD2000E
:108BA000D20042F04002072989BF0839114311431E
:108BB00041F0800141F48C41FFF784BF30B4DCB256
:108BC0001D0144EA02225C10C3F3033305F4E045BF
:108BD00004F480642A43234330BC1943FFF77CBF6D
:108BE00038B54369054653F821404368E41A043C0C
:108BF000C4F34A0141F46041FFF764FF2B68022B84
:108C00000AD124F4FF6020F0070028B110F5006FAE
:108C100014BF0020012038BD0120FCE7F8B54469ED
:108C200006461F4654F822204468121B141F651084
:108C3000B3B9EDB245EA012141F45041FFF742FFDB
:108C40003368022B0AD134F0FF0407D014F5807F7B
:108C500014BF002301231F463846F8BD0123FAE75D
:108C6000A61204F40052C4F38534C5F30B0506F4D0
:108C700080662A43344342F4004244EA811141F4BD
:108C80007041FFF729FFE7E738B54369054653F818
:108C900021404368E41A043CC4F34F02C4F30A3190
:108CA00042F4784241F47041FFF716FF2B68022B23
:108CB00008D1A00D800528B110F5800F14BF002049
:108CC000012038BD0120FCE7F8B504460D461646E4
:108CD000476813460A464FF24021FFF76FFF2046D0
:108CE000330C2A464FF2C021FFF768FF3846F8BD23
:108CF000072910B404460AD832F0FF0307D142EA2C
:108D000001215DF8044B41F40051FFF7DBBE130C69
:108D10001B0443B9134620460A465DF8044B4FF244
:108D20004021FFF74BBF20465DF8044BFFF7CCBF57
:108D300008B50368012B05DD31F0FF0302D00648BA
:108D400044F056FBC9B241EA0221BDE8084041F4B3
:108D50001041FFF7B7BE00BFC431056008B5036816
:108D6000012B05DD32F0FF0302D0064844F040FB42
:108D7000D2B242EA0121BDE8084041F41841FFF7B0
:108D8000A1BE00BFC4310560D2B242EA012141F464
:108D90002841FFF797BE38B543690C46054653F89E
:108DA000223042689B1A0A464FF2402143F00103E9
:108DB0000A3BFFF703FF2346284622464FF4324181
:108DC000FFF7E5FE2846210104F0070401F08001C9
:108DD000214341F48841BDE8384041F07801FFF774
:108DE00071BE072930B4054614460CD8072A0AD8A4
:108DF0001F2B08D841EAC20242EA831130BC41F479
:108E0000D041FFF75FBE9B00284643EA013244F49D
:108E1000784130BC41F0D001FFF75EBE436953F8A2
:108E200021104368CB1A0131A3F1040330B4C3F31A
:108E30004A0204460DD0D91C0BDA23F4FF6525F055
:108E4000070515F5006F04D142F4604130BCFFF70F
:108E500039BEC3F30A33204642F4384243F470412A
:108E600030BCFFF739BE436953F822204368D31A58
:108E70000132A3F1040370B406464FEA63040ED036
:108E8000DA1C0CDA23F0FF0212F5807F07D1E4B27E
:108E900044EA012170BC41F45041FFF713BE9D121A
:108EA00003F40052C3F38533C4F30B0405F4806567
:108EB000304622432B4342F4004243EA811170BC06
:108EC00041F47041FFF708BE38B514460B4607223F
:108ED00005462146FFF785FF2846E100BDE83840FA
:108EE00041F48F41FFF7EEBD90F854007047C36C1A
:108EF00019440369012BC16404DD836D5A8C9142CE
:108F0000C8BF59847047704700224FF0FF3180F886
:108F10005420FFF7ECBFFFF7F7BF00226FF003010B
:108F200080F85420FFF7E3BF4FF0FF31FFF7DFBFBA
:108F300038B5C46C0546036A2144994208D9083102
:108F4000406A21F00304E100F9F7C1FAC5E90840DD
:108F500038BD70B504460E4601211546FFF7E8FFFF
:108F6000E16C626A204602F8316002EBC103012124
:108F70005D605970BDE87040FFF7B9BF70B5044639
:108F80000E4601211546FFF7D3FFE16C626A2046C9
:108F900002F8316002EBC103022201215D605A70C8
:108FA000BDE87040FFF7A3BF0022114680F85420AF
:108FB000FFF7E4BF0A46002180F854100221FFF7B2
:108FC000DDBF38B50D1E044613DDFFF7B1FF626A41
:108FD000E16C002002EBC103294402EBC102012D28
:108FE000587014BF002194F8281003F8081B9A4207
:108FF000F5D129462046BDE83840FFF778BFF8B5DF
:10900000D0E90B5304460E4601331746AB4206D94E
:109010000435406BA900F9F75AFAE5626063C6F3BC
:109020000E01D4E90C305A1C00EB8305226341EA9F
:10903000C732002120F823204FF6FF733246E06D3F
:109040006B80FFF7A8FEE06D00220321BDE8F84029
:10905000FFF76EBE10B4019C41EAC303A40143EACA
:10906000020104F4F86421435DF8044BFFF72ABDC4
:1090700041EAC20242EA831141F4C051FFF722BD26
:10908000D0E90C2310B502F180420446013A03EB0B
:109090008202D0786FF3C710D070043A93420BD895
:1090A00092F903000028F8DA12880021E06DC2F37B
:1090B0000E02FFF770FE07E069B90B460A46E06D45
:1090C00044F24001FFF763FDE06D00220321BDE89B
:1090D0001040FFF72DBE10BD10B504460121FFF76B
:1090E000CFFF0122E06D0021FFF738FE002220466D
:1090F0001146BDE81040FFF72CBF10B4D0E9164070
:109100001346E48AE40704D506225DF8044BFFF712
:1091100068BE5DF8044BFFF721BE70B504460D46EE
:10912000D0E91660F68AF6070AD59200FFF7E0FD4F
:109130002A462946E06D0623BDE87040FFF798BF38
:10914000BDE87040FFF720BE036870B51A7804468A
:109150005D88042A04BF5A6842F825106A1C002161
:109160005A80B0F84820FFF7C8FF0022E06D0223C4
:109170001146FFF736FE00222B46E06D1146BDE892
:109180007040FFF72EBEF8B5C76C0546446A07F17C
:109190000053023B04EBC304D4E9020184E803005A
:1091A000667856B9B5F84A20314628463A44013A1D
:1091B000FFF7A3FF01236660637028464FF0FF317D
:1091C000BDE8F840FFF793BE13B5D0E91630DB8A4F
:1091D000DB0707D5009106234FF4C041FFF73AFFA4
:1091E00002B010BD02B0BDE81040FFF7A1BD70B5E0
:1091F000002405462646EB6CA34200DC70BD6B6A7A
:1092000003EBC4035A78012A07D15E702846B5F8EB
:109210004A105A682144FFF7D7FF0134EBE737B50E
:1092200004460D4601920093FFF7E1FFE06DDDE992
:109230000012FFF75DFD03222946E06D03B0BDE893
:109240003040FFF741BE13B504460191FFF7CFFF51
:1092500003220199E06D02B0BDE81040FFF734BE73
:1092600038B500250446082180F85450FFF7EBFF7D
:109270002A4629462046BDE83840FFF76ABE37B582
:1092800004460D4601920093FFF7B1FFE06DDDE962
:109290000012FFF72DFD03222946E06D03B0BDE863
:1092A0003040FFF711BE10B4002302F129040A4632
:1092B00080F85430E1B25DF8044BFFF7E0BF0023C3
:1092C00070B504460E46154680F8543062B1037DF1
:1092D00053B1084604F032FA021E05DD2046702123
:1092E000BDE87040FFF74ABE0635324620460023EF
:1092F000E9B2FFF7C4FF002220461146BDE87040E6
:10930000FFF727BEF8B51646044600250F46FFF7BF
:109310006EFF31462046FFF70BFEE36C2A46B5424E
:109320000CD1B4F84A20394620461A44FFF7F5FE1E
:1093300029462046BDE8F840FFF7D9BD5819616AB3
:10934000013521F83020EAE773B504461E460D4684
:109350000192FFF74CFF019AE06D0021FFF7C8FC76
:109360003246E06D0121FFF7C3FC03222946E06D80
:1093700002B0BDE87040FFF7A7BD2DE9F041C76C12
:10938000002405460E46BF1AA046EB6CA34201DC42
:10939000BDE8F081BC4211D06B6A03EBC4035A787C
:1093A000012A0BD15A68B24208D183F801803246B3
:1093B000B5F84A1028462144FFF706FF0134E4E7D8
:1093C00070B500250E4604462A46294680F85450BA
:1093D000FFF7D3FF2946F200E06D42F00202FFF7EB
:1093E00087FC2A4629462046BDE87040FFF7B1BDFC
:1093F000F8B5C369044615469E5C602E06D14768E1
:109400000A461448144906F0F3FA38600023022D86
:1094100084F854300DD8A36D9A8C52B9DB8ADB07DF
:1094200007D40E4B5A5D31462046BDE8F840FFF7A1
:1094300090BD00222046ED431146FFF79EFFB4F891
:109440004A20636C002120461A442A44FFF755FE47
:109450000022E8E72C4D0560EA310560D034056054
:1094600070B5002504460E462A46294680F8545019
:10947000FFF783FFA26D31462068D38A43F02003B3
:10948000D382FEF7DEFDB4F8482006462946204682
:10949000FFF733FE2A462946E06D0123FFF7A1FCC2
:1094A0002A462946E06D0323FFF79BFC2A462946FE
:1094B000E06D3346FFF795FC2A4629462046BDE875
:1094C0007040FFF746BD00000E2902D10849FFF7A2
:1094D000C7BF0022102980F8542002D15421FFF781
:1094E0004DBDB1F10F024FF0010118BF0122F6E7A7
:1094F000705B0560037D33B1C36CC9431944436A93
:1095000013F83100704718467047000070B50E46DA
:10951000154643B9037D33B15268C06DFFF7E8FBD0
:109520002C78204670BD2C782CB96A683146C06D05
:10953000FFF7DEFBF5E7012C07D16B68013307224B
:109540003146C06DFFF74DFC0AE0A31E012B09D880
:109550006A683146C06D520042F00102FFF7C8FB55
:109560000024DEE7542C01D10023E8E7014843F052
:109570003FFF00BF0C320560F8B500240546FFF739
:1095800036FE2746EB6CA34200DCF8BD6E6A06EBA4
:10959000C4025378022B0ED10121577000232846B4
:1095A000FFF7B4FF06F83400B5F84A100122284648
:1095B0002144FFF709FE0134E4E7002313B5044614
:1095C00080F854300191FFF7D7FF0199E06D02B0A8
:1095D000BDE81040FFF722BC38B50D4604461146E1
:1095E0007AB10022C06D1146FFF782FB00220121F3
:1095F000E06DFFF79DFB29462046BDE83840FFF7A8
:10960000DCBFFFF73DFDF6E72DE9F04104460E46CD
:10961000A2B300231746D0E90C5C984605F18045BB
:10962000013D0CEB8505284690F9011000290FDA61
:1096300090F9031000290BDAB8F1000F08BF80463B
:109640002BB1B0F800E059886EF30E015980034643
:10965000013FA0F10400E7D16FF00301E06D4A4340
:10966000A918CBB98C4510D91A4644F24001FFF72E
:109670008EFA00220321E06DFFF75AFB26F4004129
:109680002046BDE8F041FFF798BFAA5A1946C2F339
:109690000E02FFF780FBECE75A8847F6FE7161F394
:1096A0000E0239465A8026F40042FFF774FB3A4610
:1096B0001321E06DFFF73CFB3A463946E06DFFF7BA
:1096C00017FB3A460121E06DFFF732FBB8F8006066
:1096D000C6F30E06D2E773B50D4604461946164684
:1096E0002A460193FFF749FEE36C606A5B1B019910
:1096F00000EBC30210F8333033705378012B0DD0D8
:10970000022B14D0C3B9B4F84A202046E36C1A44A3
:10971000521B02B0BDE87040FFF7EFBC52688A42AE
:109720000AD0E06D02B0BDE87040FFF735BA002303
:109730002046FFF7EBFE307002B070BD13460022EA
:1097400010B5044680F854200A460121FFF7C3FFF4
:1097500020464FF0FF31BDE81040FFF7C8BB70B5A1
:10976000049E04461D46FFF7E9FF3246204629467F
:10977000BDE87040FFF7E2BF7FB5012504460DF15B
:109780000F030DF10E0100220095FFF7E8FF9DF891
:109790000F609DF80E1020460022FFF7DAFB2A46E4
:1097A00031462046FFF7D5FB04B070BDF0B501256A
:1097B00085B0002204460DF10F030DF10E01009556
:1097C000FFF7CDFF9DF80F709DF80E602A463946D1
:1097D0002046FFF7BEFB314620460022FFF7B9FBCB
:1097E0002A4639462046FFF7B4FB00223146204680
:1097F000FFF7AFFB05B0F0BD2DE9F04104461D4673
:10980000089FDDE90686FFF799FF29464246204674
:10981000FFF794FF3A4631462046BDE8F041FFF796
:109820008DBF2DE9F04186B00226012504460DF1D9
:1098300017030DF115010022029601930DF1160395
:109840000095FFF7D9FF9DF817809DF81670204608
:109850009DF815100022FFF77CFB3246414620465A
:10986000FFF777FB2A4639462046FFF772FB06B022
:10987000BDE8F08130B587B00025044601220DF126
:1098800017030DF1150102950193022300930DF1C9
:109890001603FFF7B1FF20461921FFF7D4FC2A4633
:1098A00029462046FFF755FB07B030BDF7B5046BDE
:1098B00005460E46D4B104F18044436B013C03EBF2
:1098C000840292F90120002A21DA33F82430C3F30C
:1098D0000E038B421BD100220DF107010124FFF77B
:1098E0002DFF00220121E86DFFF722FA002728460C
:1098F00085F85470FFF740FE3146E86DFFF7C5F874
:109900001CB139462846FFF7BBFB03B0F0BD00246D
:10991000ECE770B5002604460122314680F8546019
:10992000C06DFFF71BFA22212046FFF78CFC47F69B
:10993000FF72D4E90C35013B05EB830523636B888B
:10994000C3F30E03934228D013223146E06DFFF794
:1099500005FA4FF42051E06DFFF7B4F8A3683146E3
:10996000E06D1A68FFF77FFA698847F6FE73C1F366
:109970000E029A420BD14FF48E41E06DFFF7A2F830
:10998000A36820461968BDE87040FFF78FBFC1F398
:109990000E012046FFF711FEF2E770BD2DE9F043FE
:1099A0000446C16887B0FFF781FFA36D9A8CD98AFE
:1099B00012B901F0110373B311F0010117D1B4F81A
:1099C000482020460132FFF798FBA36D9D8C55B9C6
:1099D0004FF42051E06DFFF775F8E2682946E06D1D
:1099E0000132FFF740FA05212046FFF72CFC212128
:1099F0002046FFF728FCA36DDA8AD20706D49B8C99
:109A000023B9E16820460131FFF750FF12220021FF
:109A1000E06DFFF7A3F9E06DFFF79AF8237D002BC7
:109A20005FD1E36D656C5B68013DA3632368EA0069
:109A30002D095B8802F07802E363A36D5E8BDF8AF9
:109A4000B3F81C90B3F81E8006F0030307F00F076D
:109A5000B6081A4345EA0703E06D334343EA0903B6
:109A600053EA08036CD10121FFF71EF8B4F85060E7
:109A7000B4F85270720007F00103B609012102F038
:109A80007E027F08E06D57EA060542EA030218BF2E
:109A900042F08002FFF708F8002DEBD1A36DE76DCF
:109AA000998A20687E68FEF7B5FA024638464C4F20
:109AB0004B490EF065FEA26D538B918B108D0B44BC
:109AC000AB427BDCE36D00259F88BE1BA4F8506091
:109AD000D4E916301A8DAA4272DC4368DB1BA4F865
:109AE00052302369042B27D12268E36D5568227D0B
:109AF000D3E902377AB9A66BE16B3E4400296CD0FA
:109B00000131284605938900F8F7E1FCE26B054630
:109B1000059B40F82260217DA26D00294FF00001D5
:109B20001069CDE90211D28A14BF04210321CDE9C5
:109B300000523A4603F09CF9012007B0BDE8F083DB
:109B400042F080020121FEF7AFFFBA012B0102F0C3
:109B50004002AD0803F030037F081A4308F0010308
:109B60004FEA58081A434FEAC9034FEA590903F06C
:109B700008031A43B300760803F004031A4369E7A5
:109B8000D36A03EBC10393F801C01CF0010F10D09E
:109B9000B3F802C0AC450CD15968D4F85C800135EB
:109BA0002068FEF737FA3946024640460EF0E8FDD7
:109BB00081E701318142E3DB0521EEE70021F9E78E
:109BC000DB6A03EBC50213F83530052B03D152884D
:109BD0000121FEF769FF01357AE735469BE700BFB3
:109BE000738A0060F8B5836804461E68836DC6609A
:109BF000DD8A9B8C05F01102134300F0E28015F022
:109C0000010506F102071BD1B0F848202946FFF7ED
:109C100074FA01232A462946E06DFFF7E2F82A4646
:109C200001232946E06DFFF7DCF805212046FFF708
:109C30000AFBB4F848102A4620460131FFF7C4FA5F
:109C4000D4E916309A8C002A57D1D98A11F001052F
:109C500008D14FF42051FEF735FF3A462946E06D12
:109C6000FFF701F90022E06D1146FFF78DF8202182
:109C70002046FFF7E8FA4FF42051E06DFEF722FF8F
:109C80003A460021E06DFFF7EEF8A36DD98A11F096
:109C900001017DD001220021E06DFFF75FF846F25F
:109CA0007011E06DFEF70EFFE06D02220021FFF75C
:109CB0001FF8E06DFEF74CFF39462046FFF7F6FD32
:109CC000A36DDB8ADB077CD5B4F848202046002151
:109CD0000132FFF712FAE06D4FF48E41FEF7F2FE0B
:109CE000E06D0021012243682364FFF737F8204626
:109CF0002221BDE8F840FFF7A6BA002344F2400154
:109D0000751C03361A46FEF742FF00221321E06D50
:109D1000FFF70EF83A460421E06DFFF73CF82946BC
:109D20002046FFF7C3FD0022E06D1146FFF72CF837
:109D300020212046FFF787FA4FF42051E06DFEF70F
:109D4000C1FE32460121E06DFFF78DF8002344F299
:109D50004001E06D1A46FEF71AFF00220321E06D74
:109D6000FEF7E6FF44F22071E06DFEF7ABFE3146F0
:109D70002046FFF79BFD03220421E06DFEF7EEFF76
:109D80004FF43051E06DFEF79DFE2A46012179E740
:109D9000B4F8482020460132FFF7AFF905212046EC
:109DA000FFF751FAA36DD98A11F001017FF472AF68
:109DB000E06D0122FEF7D2FF22212046FFF743FA91
:109DC0007AE7F8BD138B2DE9F04104460161D81EF6
:109DD0000E46118C15464342A2654341237500236C
:109DE000E36484F85430A3698B4205D2E069F8F744
:109DF0006EFB2B8CE061A361A26D518B938BEA8A81
:109E00000B44510748BF013392074FF0000248BF8F
:109E100001331146934246D1227D002A57D1602159
:109E2000A2699A4255D8226A002360219A4254D1ED
:109E3000042EE06D0CBF02210121FEF703FE00237A
:109E4000A4F84830A36D9A8C002A4BD1DB8A03F02A
:109E5000110313B11323A4F84830A5492068FEF775
:109E6000F0F8277D80462B8CA66D698C002F00F0C2
:109E7000F680CA18B18C6264002935D1F08AC60711
:109E800007D4032BA8BF032319466B8B032B00D9E0
:109E9000013910F0110F28D1E88AB4F84830800653
:109EA00048BF013324E0E06981540132B2E7C86A57
:109EB00000EBC20001324178CF0741BF4788090952
:109EC000E069C155A16D088D9042F0DCA7E7002242
:109ED000F8E7E269D1540133A2E7606A20F8331051
:109EE0000133A3E71423B6E70021B4F84830023366
:109EF000A4F84A30B4F84A30E06D1A44511AFEF71B
:109F0000F9FD012300220721E06DFEF76AFF072219
:109F10000323E06D1146FEF764FF07224346E06D20
:109F20001146FEF75EFFA36D9A8C1AB9DB8A03F027
:109F300030032BB10022B4F84810E06DFEF7F8FEB4
:109F400001220021E06DFEF727FE02220121E06DD3
:109F5000FEF722FE03220621E06DFEF71DFE4FF400
:109F60002451E06DFEF7AEFDA3680121E06D1A6893
:109F7000604E0432FEF777FF6A8B0221E06DFEF738
:109F8000B7FE022300224FF48541E06DFEF7FFFD8E
:109F9000A3680021E06D1A680532FEF764FFA3682C
:109FA000E06D19680431FEF770FD6B8B0221E06DE6
:109FB0005A00002542EA4342FEF79AFE03222C2172
:109FC000E06DFEF781FFA368E06D19680531FEF7CB
:109FD0005CFDA36D5A8BAA4214DC032A0DD99A8C1E
:109FE0005AB9DB8ADB0708D4B4F84A200621636C2F
:109FF000E06D1A44033AFEF7B1FE2046BDE8F04199
:10A00000FFF7F0BD2B4606220021E06DFEF7E9FECA
:10A01000E3695A5D22B1012303212046FFF7FFF8CF
:10A02000022D11DCA36D9A8C72B9DA8AD2070BD497
:10A03000022D02D15B8B032B06D10022715DE06DF6
:10A04000FEF7AAFD0135C4E7B4F84A100022636C9C
:10A05000204619440139491BFFF7B6F8F2E7F68AA2
:10A060001944E06D16F00106616445D0E26B0421ED
:10A07000FEF71AFD226C0421E06DFEF715FDB4F821
:10A080004810E06DFEF736FD4FF4A0233A46062156
:10A09000A364E06DFEF780FD0122E06D1146FEF73E
:10A0A00047FEB4F8483006223946E06DFEF799FEC7
:10A0B00001233A463946E06DFEF793FE03233A4604
:10A0C0003946E06DFEF78DFE43463A460721E06DC6
:10A0D000FEF787FE2046FFF785FDA36D9A8C002AC8
:10A0E00057D0002319462A8D9A4269D8BDE8F081DD
:10A0F000643B0560D0340560B4F8483005339BB24A
:10A100001944A4F84A30FEF7F5FC01233246072132
:10A11000E06DFEF766FE07220323E06D1146FEF7B1
:10A1200060FE07224346E06D1146FEF75AFE3246B6
:10A13000B4F84810E06DFEF7FBFD022332463146CD
:10A14000E06DFEF74EFEE36B23B132463146E06D23
:10A15000FEF747FEB4F84810204600220131FFF711
:10A1600033F8626CE06D0021FEF7C2FDB4F84810D0
:10A17000204600220331FFF727F8B4F84820E06DAD
:10A180000021FEF701FE04222D21E06DFEF79CFE6A
:10A19000A0E7DE8A16F00106A3D10F4F2B8CB34245
:10A1A0009FDDB4F84A20636C17F8011B1A44E06D78
:10A1B000013A921B0136FEF7D1FD032EEED190E756
:10A1C000EA6A02EBC30012F833200133052A02BF0A
:10A1D0004288E069815486E7D03405607FB5044643
:10A1E0000E46154682B90DF10F01FFF7A7FA324668
:10A1F000092120460123FFF742F82A462946204636
:10A20000FEF7A7FE04B070BD012A0FD10223002281
:10A210000DF10E0100930DF10F03FFF7A0FA0123DA
:10A2200032460E212046FFF72AF8EBE70DF10F0129
:10A230000022FFF783FA022344F24001E06D1A4640
:10A24000FEF7A5FCEBE773B504460E4615466AB962
:10A2500001220DF10701FFF771FA0C350023324698
:10A260002046E9B2FFF70BF802B070BD0021FFF7FE
:10A2700041F98DF8070020B901220DF107012046B0
:10A28000E9E70DF1070120460022FFF757FA9DF894
:10A290000720204601230421FEF7C1FF00220121EF
:10A2A000E06DFEF779FCD8E773B516460D4600223F
:10A2B0000DF107010446FFF741FA721C0221204606
:10A2C0002A44FFF71FF8012345EA062228212046E9
:10A2D000FEF7A5FF02B070BD37B504460D4600225B
:10A2E0000DF10701FFF72AFA2A4620460221FFF75F
:10A2F00009F801232A4627212046FEF790FF03B0E4
:10A3000030BD37B50D4600220DF107010446FFF7B9
:10A3100015FA55B1012120460422FEF7F3FF1E2154
:10A320002046FEF790FF03B030BD2A46E06D0121C4
:10A33000FEF7DEFC20461E21FEF785FF2A46294651
:10A340002046FEF706FEEEE737B500220DF10701C5
:10A350000446FFF7F3F99DF807302BB1656805490E
:10A36000054805F045FB286022212046FEF76BFFDB
:10A3700003B030BD213205602C4D056073B501225C
:10A380000D460DF107010446FFF7D8F99DF8076067
:10A3900066B92A46112120463346FEF740FF324671
:10A3A00031462046FEF7D5FD02B070BD20460121A2
:10A3B000FEF79DFD044B64685A5D0449044805F0AE
:10A3C00017FB2060F0E700BF986805603632056033
:10A3D0002C4D05602DE9F3410E4600211746044639
:10A3E0001D46FFF787F802468DF8070048BB0DF1C0
:10A3F00007012046FFF7A2F91DB901212046FEF70B
:10A4000076FD10212046FEF71EFF1DB99DF807308E
:10A4100084F828302046FFF7AFF84FF42051E06D64
:10A4200086B3FEF74FFB3A460121E06DFEF71BFDB8
:10A4300025B94FF0FF312046FEF759FD02B0BDE8C7
:10A44000F08100220DF107012046FFF777F91DB9D1
:10A4500001212046FEF74BFD9DF807305A1E022AC7
:10A46000D3D9072BD4F80480094994BF094A40F294
:10A47000B222094898BF32F8132005F0B9FAC8F89B
:10A480000000C2E7FEF71EFB3A463146CDE700BFAB
:10A4900052320560D03305602C4D05600023FFF774
:10A4A00099BF0123FFF796BF022A7FB504460E46E7
:10A4B000154614D8836D9A8C8AB9DB8ADB070ED4D3
:10A4C0001C4B0DF10F015A5DFFF738F9E1699DF85A
:10A4D0000F204B5D602B13D14A5504B070BD0DF1B8
:10A4E0000F0120460022FFF729F9616CB4F84A30C9
:10A4F000002220460B44E9431944FEF765FEE5E7D8
:10A500009342EAD0072B64680B4896BF0B4940F290
:10A51000B22331F81330072A96BF084940F2B2221D
:10A5200031F8122006490092324605F061FA2060A7
:10A53000D3E700BFD03405602C4D0560D0330560F3
:10A540007A32056070B5164604460D461A465BB968
:10A55000542180F85430FEF711FD3246294620463A
:10A56000BDE87040FFF7A0BF70BD2DE9F0410025A8
:10A57000D0F824C00446DDF8188080F85450C56C2B
:10A58000013D0CEBC5067778012F14D1D6F804E015
:10A590009E4510D0C6450ED01CF835300B70716842
:10A5A00011603A46FEF7E9FE20464FF0FF31BDE864
:10A5B000F041FEF79CBC136820460A460121FFF7D4
:10A5C0008AF8F1E710B5002386B0044605934FF0F2
:10A5D000FF3305AA0DF113010093FFF7C6FF9DF8A5
:10A5E0001310059A2046CDE90212FEF7B2FC204670
:10A5F000DDE90212FEF7ADFC06B010BD70B50446F1
:10A6000086B00D4616461BB9FFF74EFF06B070BD6B
:10A6100000221146FEF7B1FE204600220121FEF77E
:10A62000ACFE324629462046FEF7E2FE002304AA8D
:10A630000DF10F0104934FF0FF3320460093FFF715
:10A6400094FF01230DF10F012046059305AA049BF9
:10A650000093FFF78AFFE06DDDE9043141EAC301B1
:10A6600041F4C04141F04001FEF72CFACEE77FB53E
:10A6700004460D4616461BB9FEF7BAFE04B070BD7F
:10A6800000221146FEF779FE324629462046FEF7A3
:10A69000AFFE4FF0FF33002503AA0DF10B0120465A
:10A6A00000930395FFF761FF039A2946E06D0123AC
:10A6B000FEF797FB2A4629462046FEF74AFCDDE7CF
:10A6C000F0B5044685B00D460121FEF713FF06469E
:10A6D0008DF80A0000212046FEF70CFFB31E8DF80E
:10A6E0000B00012B00F2D080861E012E00F2F680B6
:10A6F000A5F109030C2B9CBF0D35EDB21F2D01D028
:10A70000212D23D1002301220DF10B0120460093BE
:10A710000DF10A03FFF723F89DF80A30022B07D04A
:10A720007D4B66685A5D7D497D4805F061F9306072
:10A730001F2D20460CBF2E212F21FEF784FD002265
:10A7400002212046FEF705FC05B0F0BD01260223DC
:10A7500003AA0DF10B012046039300960023FFF797
:10A7600004FF32460DF10A012046FEF7E7FFA5F18E
:10A770001903B34216D8192DE06D039B08D1324658
:10A780004FF48141FEF703FA01229DF80A10D8E741
:10A790009DF80A20032A32460CBF44F2C0014FF450
:10A7A0008241EFE7162D05D1039B32464FF48641D7
:10A7B000E06DE7E7172D04D1039B324644F24001D8
:10A7C000F6E7182D04D1039B32464FF48041EFE7A2
:10A7D0001B2D06D1039B32463146E06DFEF748FC47
:10A7E000D2E71C2D08D1039941F60923E06D43EA15
:10A7F0008111FEF767F9C7E71D2D04D1039B32468F
:10A8000044F24031D4E7052D31D89DF80A209DF857
:10A810000B309A4205D066684249414805F0E8F895
:10A8200030609DF80A3000222046032B11460CBFF1
:10A8300000260626FEF7A1FD0122039B4FF4854169
:10A84000E06D3544FEF7A3F9374BE06D33F8151092
:10A85000FEF738F942F20101E06DFEF733F94FF4EB
:10A860000051E06DFEF72EF90022012169E7204634
:10A870000121FEF73CFB284B2C495A5D28486468AF
:10A8800005F0B6F820605FE7064327D101270DF1F8
:10A890000A0302220DF10B0120460097FEF75FFF2D
:10A8A000322D17D0332D17D1072500232A46122128
:10A8B0002046FEF7B4FC57B100220121E06DFEF7FF
:10A8C0006BF90023032211212046FEF7A8FC002289
:10A8D000114636E70625E8E73746E6E74FF0FF3151
:10A8E0002046FEF704FB9DF80A300D48072B6468EC
:10A8F00096BF0F4A40F2B22232F813209DF80B3077
:10A90000072B96BF0A4940F2B22331F813300949A8
:10A9100005F06EF8B6E700BF64670560A632056013
:10A920002C4D0560C7320560B8340560E232056021
:10A93000D0330560FF32056003297FB50446164613
:10A9400012D1182501220DF10F01FEF7F7FE0023A9
:10A950000DF10F0231462046FEF7BDFE2946204686
:10A96000FEF771FC04B070BD052906D101220DF17E
:10A970000F011725FEF7E2FEE9E7022301220DF1A0
:10A980000E01192500930DF10F03FEF7E8FEDEE737
:10A99000F0B5044685B00E461546C2B90223077DC0
:10A9A0000DF10E010275012200930DF10F03FEF768
:10A9B000D6FE32462B46232120462775FEF75FFC44
:10A9C0002A4611462046FEF7C4FA05B0F0BD012A1A
:10A9D00010D100270DF10F0229463B4680F8547034
:10A9E000FEF779FE32462B4624212046FEF747FC2F
:10A9F0003A46E6E70DF10F010022FEF79FFE252102
:10AA00002046FEF720FCE0E72DE9F84F002504463C
:10AA10000F469146A846FEF7EAFB4D4510D10026A9
:10AA2000B3464E452BD171422046FEF760FAB4F88A
:10AA30004A20E36C39461A44BDE8F84FFEF76DBB77
:10AA4000E66CD4F824A0013E761B0AEBC6025378CC
:10AA5000022B12D10123394682F801802046FEF7ED
:10AA600055FD0AF83600B4F84A103A46E36C204621
:10AA700019440139491BFEF7A7FB0135CDE7E36C0B
:10AA8000D4F824A003F1FF38A8EB06081AF8382000
:10AA9000BAB1B4F84A50002120461D44013DAD1B17
:10AAA0002A46FEF72AFB01231AF838200421204603
:10AAB000FEF7B5FB002229462046FEF785FB0AF883
:10AAC00038B00136ADE70000037D37B504460D46CA
:10AAD00013B1544842F08CFC826DD38A43F00103D9
:10AAE000D382FEF749FD012D0BD1A36820461968DA
:10AAF0000231FEF762FDA368204619680131FEF7B6
:10AB0000D5FE012200212046FFF77EFF0022022110
:10AB10002046FEF759FB01220021E06DFEF7E8F820
:10AB200000221221E06DFEF703F9A3680021E06D19
:10AB30001A68FEF730F9B4F84810002220460131B7
:10AB4000FEF742FBE168E06DFEF768F9A368E06D8F
:10AB50001968FDF79AFF236BBBB103F18043626B69
:10AB6000013B02EB83039A420FD893F903100029AB
:10AB70001BDA1A880021E06DC2F30E02FEF70BF912
:10AB800000220321E06DFEF7D3F801212046FEF7F5
:10AB900018FA65B92946E06D0122FEF7DFF8222197
:10ABA0002046FEF750FB03B030BD043BDBE7A36853
:10ABB000204619680231FEF779FE0DF107012046A3
:10ABC0000122FEF7BBFD00230DF107022046012103
:10ABD000FEF781FDE06D01220221FEF7BFF820465D
:10ABE00002220021FEF7B5F9012220460221FFF7DB
:10ABF0000BFF20463021FEF726FBE06D4FF420517D
:10AC0000FDF760FFA368E06D01211A680132FEF7CD
:10AC10002AF920460121FEF7D4F92046FEF7B3FABF
:10AC2000C1E700BF28330560F8B5174604460D4656
:10AC3000520093B1CB1C02211A44FFF7E5FE01221A
:10AC400045EA07231D212046FEF77EFB0022204611
:10AC50001146BDE8F840FEF77CB980F854308B1CF3
:10AC600002211A44FFF7D0FE3B462A461C21EAE7A0
:10AC70002DE9F7431646002701EB42020D4680F806
:10AC80005470044611469846FEF734FC70288DF83F
:10AC9000060033D1E26C3946636A204603EBC203F7
:10ACA00013F80C6CFEF726FC072805460DD888B172
:10ACB0002046FEF768FAE36C626A03F10053013B39
:10ACC00002F8336003B0BDE8F0835428F0D01F4889
:10ACD00042F08EFB02460DF107012046FEF72EFDE5
:10ACE0002046FEF711F9324603210123FEF797FAB9
:10ACF0002A4631462046FEF72CF9E3E745EA0629C5
:10AD0000B8F1000F0DD0023202212046FFF77CFE81
:10AD10004B463A461D212046FEF716FB00221146FF
:10AD2000E8E756EA050303D002212046FFF76CFE50
:10AD30000DF1060120460022FEF700FD01234A46E0
:10AD40001B212046FEF76BFAE8E700BF35330560AC
:10AD50002DE9F0411D4600230F46164680F8543079
:10AD60000121B0F848200446DDF81880FEF7C5F947
:10AD70000123E06D1A461946FEF733F855EA080537
:10AD80002CD12046FEF733FA2A460221E06DFDF76A
:10AD9000AFFF39692046FEF7D7F903221A21E06D8B
:10ADA000FEF792F832460121E06DFDF7A1FF324631
:10ADB00002212046FFF728FE25B16FF00101204651
:10ADC000FEF795F8E06D03222B21FEF77DF80022B7
:10ADD00020461146BDE8F041FEF7BBB806F1020877
:10ADE000204602214246FFF70FFE41462046FEF76D
:10ADF0007EF8FEF7FCF9CCE7F7B51E4600231546B2
:10AE00000F46B0F84820012180F854300446FEF780
:10AE100074F90123E06D1A461946FDF7E2FF55EA81
:10AE20000602019218D12046FEF7E1F9019A0221AB
:10AE3000E06DFDF75DFF39692046FEF785F9E06DAD
:10AE400003221A21FEF740F800222046114603B0E3
:10AE5000BDE8F040FEF77DB8022220461146FFF71C
:10AE6000D3FD2046FEF7C3F9E5E7042A70B5044692
:10AE700086B00E4615462AD102294FF0000518D19A
:10AE80000DF1160301220DF117010095FEF767FC85
:10AE90002B4607223146E06DFDF7A3FF2621204611
:10AEA000FEF7D1F9002220461146FEF752F806B00F
:10AEB00070BD0DF1150302220DF1170102950193EA
:10AEC000012300930DF11603FEF796FCE6E700233D
:10AED000012A80F8543001D9032A04D132460121D5
:10AEE0002046FFF791FD1335002332462046E9B294
:10AEF000FEF795F9D6E770B50025044604220E4604
:10AF000080F854502946FFF77FFD20460421FDF7C5
:10AF1000EEFF1F21FEF797F9E06D4FF42051FDF78A
:10AF2000D1FD32462946E06DFDF79DFF2A462946B0
:10AF30002046BDE87040FEF70CB870B50025044609
:10AF40000E4680F854502946FEF79AF820464FF0F6
:10AF5000FF31FDF7CCFFA36819680231FEF7A6FCAC
:10AF60002A4620465421FEF709F82A462046542155
:10AF7000FEF704F82A4620465421FDF7FFFF20463D
:10AF800005220221FFF740FD03222B4620461C210B
:10AF9000FEF7DAF9A36820461968FEF70EFB314682
:10AFA000E06DFDF772FD20460121FEF769F82046AD
:10AFB0000221FEF706F801222946E06DFDF7CEFEDC
:10AFC000E06D4FF42051FDF77DFDA3682946E06D4B
:10AFD0001A680232FDF747FF2B462A46E06D012131
:10AFE000FDF7FFFE294620460122FDF7B2FF2A4663
:10AFF00029462046FDF7ADFF2A4620465421FDF79D
:10B00000BDFF204605220221FFF7FEFC2B4603224E
:10B0100020461C21FEF798F920461021FEF713F96F
:10B02000E06D4FF42051FDF74DFDA3682946E06D1A
:10B030001A680132FDF717FFA36820461968FEF76A
:10B0400035FC2A462946E06DFDF752FEE06D2A46A2
:10B050000121FDF76DFEA36820461968BDE8704028
:10B060000131FEF723BC73B504460E461546002A8F
:10B0700056D1134601210DF10702FEF72CFB0222E7
:10B0800020461146FEF73EF901230D220A212046F3
:10B09000FEF7F5F802220DF107012046FEF74EFB00
:10B0A00001220DF107012046FEF748FB2A460DF16B
:10B0B00007012046FEF742FB01229DF807102046BB
:10B0C000FDF747FF02229DF807102046FDF741FFDC
:10B0D000022220461146FEF715F901230C220A210F
:10B0E0002046FEF7CCF8022220461146FFF78CFCE2
:10B0F0002B462A461C212046FEF726F92A462946D9
:10B100002046FDF726FF2046FEF736FA20460122AC
:10B110003146FDF774FF2046FFF754FA02B070BDC8
:10B12000002380F85430FEF727FAAB1E3146204644
:10B130005A425A41FDF763FFF0E737B504460D4622
:10B1400082B103220121FFF75FFC02220121204688
:10B15000FEF7D8F800232A460B212046FEF78FF889
:10B1600003B030BD0DF10701FEF7E8FA02222046D8
:10B170001146FEF7C7F801232A460A21EDE7000031
:10B180007FB5836D0446DD8A15F0010213D00122DC
:10B190000021FFF739FC002202212046FEF714F8B7
:10B1A0000022E06D1146FDF7A3FD00221221E06DA3
:10B1B000FDF7BEFD1FE0037D002B51D0114601922B
:10B1C000FEF798F95428C5F38715019A28D120462F
:10B1D000FDF79AFE019AC5B92B4607222946E06D74
:10B1E000FDF7FFFDA36D9A8C002ADED1DB8A03F008
:10B1F0001103002BD9D1226B2046E168FEF704FA37
:10B20000012384F8543004B070BD1146E06DFDF7A1
:10B210006FFD01232A4604212046FEF700F8E1E7EE
:10B220000DF10F012046FEF789FA9DF80F30AB4271
:10B2300013D0072D66680D4896BF0D4A40F2B22222
:10B2400032F81520072B96BF094940F2B22331F896
:10B250001330084904F0CCFB3060002DC2D0D8E791
:10B260001A460DF10F01FEF769FABBE72C4D056098
:10B27000D03305603D3305602DE9F04188B00446C8
:10B280000D460DF11C08002940F028810121FEF730
:10B2900031F906468DF8170088BB01462046FEF7B7
:10B2A00029F98DF81C00C0B9012241462046FEF75D
:10B2B00045FA00220DF117012046FEF73FFA04225D
:10B2C0000F2102232046FDF7AAFF00221146204647
:10B2D000FDF73FFE08B0BDE8F0813246414620460A
:10B2E000FEF72CFA9DF81C20204601230421FDF7CF
:10B2F00096FF32460121E06DFDF74EFCD9E7E36C85
:10B30000626A013B02EBC30132F8332040F20223B0
:10B310009A4272D1012620464F68FDF7F5FD33466B
:10B3200042460DF1170100960795FFF71EF92A46D0
:10B3300029462046FEF721F89DF81730062B26D027
:10B34000072B3FD0052B40F0BA80C7B17B1EE06DC4
:10B350001E2B09D8079B2A464FF4F0410097FDF7B2
:10B3600079FE00220221B2E73A463146FDF7C0FCE1
:10B37000079B32463146E06DFDF77AFE0796079946
:10B38000C90041F4F041E06DFDF79CFBE9E7A7B18E
:10B390007B1EE06D1E2B05D8079B2A464FF4084103
:10B3A0000097DCE77A003146FDF7A2FC079B3246A6
:10B3B0003146E06DFDF75CFE07960799C90041F440
:10B3C0000841E0E7A7B17B1EE06D1E2B05D8079B67
:10B3D0002A464FF4D0410097C1E7BA003146FDF745
:10B3E00087FC079B32463146E06DFDF741FE07962C
:10B3F0000799C90041F4D041C5E70123424606A997
:10B40000204607932B460095FFF7AFF82A460DF12B
:10B4100017012046FEF792F92A4629462046FDF7F5
:10B42000ACFF9DF818309A1E012A0DD9072B6568CC
:10B43000BB4994BFBB4A40F2B222BB4898BF32F826
:10B44000132004F0D5FA28609DF81730062B0CD095
:10B45000072B19D0052B32D10022079BE06D114636
:10B46000FDF706FE4FF4F0418DE70022079BE06DEB
:10B470001146FDF7FDFD0022079B1146E06DFDF72B
:10B48000F7FD4FF408417EE70022079BE06D11466F
:10B49000FDF7EEFD0022079B1146E06DFDF7E8FD8C
:10B4A0000022079B1146E06DFDF7E2FD0022079B9D
:10B4B0001146E06DFDF7DCFD4FF4D04163E7072B4B
:10B4C00065689A4994BF974A40F2B222964898BF5D
:10B4D00032F8132004F08CFA286042E7012940F08A
:10B4E0006281FEF707F806468DF8150048BB014655
:10B4F0002046FDF7FFFF02468DF818000221204686
:10B50000FDF7F8FF52EA00038DF81C0008D0314621
:10B5100020460322FFF778FA03212046FDF7E7FCD7
:10B52000022306A920460122CDE9018300230093CE
:10B530000DF11503FEF760F90F212046FDF783FE9C
:10B54000C8E6E36C626A013B02EBC30132F83320C8
:10B5500040F202239A4240F0928020464E68FDF766
:10B56000D3FC022300220DF115010093CDE906233F
:10B570002B4606AAFEF7F9FF069B42460DF117017E
:10B5800020460095FEF7F1FF9DF817305A1E022A5B
:10B590000DD9072B6568664994BF624A40F2B22212
:10B5A000614898BF32F8132004F022FA28609DF811
:10B5B0001530062B27D0072B43D0052B40F0E48015
:10B5C000BEB1731EE06D1E2B07D84FF4E04100960C
:10B5D000DDE90632FDF73EFD7CE632460121FDF74E
:10B5E00087FB0122069B1146E06DFDF741FD01231B
:10B5F0000693DDE9063141EAC30141F4E041E06D23
:10B60000FDF760FA66E6AEB1731EE06D1E2B05D83D
:10B610004FF400410096DDE90632DBE772000121BC
:10B62000FDF766FB0122069B1146E06DFDF720FD4C
:10B6300001230693DDE9063141EAC30141F40041EB
:10B64000DDE7AEB1731EE06D1E2B05D84FF4C0418F
:10B650000096DDE90632BDE7B2000121FDF748FBA7
:10B660000122069B1146E06DFDF702FD01230693C2
:10B67000DDE9063141EAC30141F4C041BFE70223DD
:10B6800006AA0DF1160120460793009300230695A4
:10B69000FEF76BFF00220DF115012046FEF74EF874
:10B6A0009DF816309A1E012A0DD9072B656821498D
:10B6B00094BF1C4A40F2B2221B4898BF32F81320B4
:10B6C00004F096F92860069B42460DF117012046CA
:10B6D00000930023FEF749FF9DF817305A1E022AF7
:10B6E0000DD9072B6568124994BF0E4A40F2B22269
:10B6F0000D4898BF32F8132004F07AF928609DF8BD
:10B700001530062B18D0072B24D0052B3CD1002256
:10B71000069BE06D1146FDF7ABFC07996DE700BF96
:10B7200074330560D03305602C4D05605F330560D0
:10B730008F330560B43305600022069BE06D11462F
:10B74000FDF796FC0022069B1146E06DFDF790FC8C
:10B75000079973E70022069BE06D1146FDF788FC10
:10B760000022069B1146E06DFDF782FC0022069B3D
:10B770001146E06DFDF77CFC0022069B1146E06D52
:10B78000FDF776FC079977E7072B64680D4994BFAE
:10B790000D4A40F2B2220D4898BF32F8132004F04F
:10B7A00027F9206096E50025434606A90122009569
:10B7B000FDF7D5FF02232A460F212046FDF72FFD76
:10B7C00088E500BFA0330560D03305602C4D0560CF
:10B7D000F7B51546074660200E460193F6F775FE4D
:10B7E0008560082504460562C0E900764020F6F72A
:10B7F00053FEE56260622020F6F74EFE6063202073
:10B80000F6F763FE0199E065FDF709F9204603B0FC
:10B81000F0BD10B504460021C06DFDF708F9E06DDC
:10B82000F6F762FE606BF6F75FFEE069F6F75CFE26
:10B83000606AF6F759FE2046BDE81040F6F754BEA0
:10B8400038B50546B2B1940714D110792E2811D11C
:10B8500092687AB190070DD15468E0B2922809D16C
:10B86000240A022C06D1916801201960049BD26839
:10B870001A6038BD0A460448044904F0B9F86B6AF6
:10B8800018600020F5E700BF004C0560D334056068
:10B89000038C032B70B5C46A03D1856A00239D42D3
:10B8A00005D144F82120FDF7F0F8012070BD54F8CF
:10B8B0002360964201D00133F1E70020F6E7FDF75F
:10B8C00047B938B58BB204460D464262032B038458
:10B8D00005D1826A0021C06A92001DF08DFB042D03
:10B8E00020460CBF02210121FDF7ACF820460021C3
:10B8F000BDE83840FDF7FEB802F00F03022B10B58B
:10B90000044608D00A460D490D4804F071F8636AF0
:10B91000186000200FE01209816A0023994204D1C7
:10B92000238C042BF5D10749EEE7E06A50F8230099
:10B93000904201D1184610BD0133EFE7FE34056097
:10B94000004C05601335056000F00F03022B02D197
:10B950000009F6F70ABF0148704700BFCC3B0660FC
:10B9600070B5054610460E46FFF7EEFF0378732BC1
:10B9700019D14378BBB103460A22002013F8014FC6
:10B980005CB91F2808D91F2332460A490A4804F027
:10B990002FF86B6A1860002070BD303C092C02D86B
:10B9A00002FB0040EAE732460449034804F020F86D
:10B9B000EFE700BF2A350560004C056043350560A0
:10B9C000F8B5044610460D461E46FFF7BDFF164A61
:10B9D0000778002194465378BB421BD190F801E0D0
:10B9E00093789E4516D190F802E0D378734511D133
:10B9F0006BB91CF82100B04208D933462A460B49DE
:10BA00000B4803F0F5FF636A18600020F8BDC378A7
:10BA1000002BEED0013104321529DCD12A4605492C
:10BA2000034803F0E5FFEEE7583705602A35056067
:10BA3000004C0560603505602DE9F34706460F466A
:10BA4000002A3CD093073AD113792F2B37D1926833
:10BA500002F00F03022B08D101240F23FFF7B0FFE0
:10BA60008440204602B0BDE8F08742B312F0030ADA
:10BA700025D113799F2B22D1D5682B79A12B1ED1EB
:10BA80004FF001080F239268FFF79AFF01AA08FA06
:10BA900000F4A22105F1080041F09EFD8146CA454F
:10BAA000DFDA019A0F233946304652F82A200AF18C
:10BAB000010AFFF785FF08FA00F31C43EFE73A4657
:10BAC00003490448002403F093FF736A1860C8E731
:10BAD00078350560004C0560F0B585B005460E462A
:10BAE000104603A91F4641F0B3FC48B932460B4942
:10BAF0000B4803F07DFF6B6A1860002005B0F0BDB5
:10BB0000039801F0B3FF30EA0703F7D0034632464B
:10BB100004490097024803F06BFFECE7933505609A
:10BB2000004C0560AB3505602DE9F0470F4688B045
:10BB300004461E4605A938469146F6F722FE0378CC
:10BB40000546762B40F02B81B9F1020F40F0D680EC
:10BB500040F202539F4232D14EF6B4684FF42C6942
:10BB600006E04EF6B168F9E74EF6B1684FF4246985
:10BB7000326829462046FFF7F3FE074672682946D9
:10BB80002046FFF7EDFEFB024201C0F3430003F441
:10BB90007043B90102F0200201F04001134341EA71
:10BBA000080143EA090343EA00022046FCF794FF38
:10BBB00030E24EF6B868D1E74EF6BD68CEE740F207
:10BBC0000D539F42CDD040F20C539F42CCD040F257
:10BBD00003539F42EDD040F204539F42ECD040F219
:10BBE0000B539F421ED13068FFF7AEFEAE491DF0E9
:10BBF0003EFAA8B10F23326829462046FFF7E0FE3F
:10BC000007467068FFF7A0FEA8491DF030FA00282B
:10BC100040F0BC803A034EF6F16142F42162C4E781
:10BC20000F27EEE740F20A539F422ED13068FFF70C
:10BC30008BFE0378722B18D10F23326829462046D9
:10BC4000FFF7BEFE2946804672682046FFF788FE51
:10BC50004EF610610746FA01C7F34307D2B23943E3
:10BC600042EA083242F421629FE7326829462046C0
:10BC7000FFF776FE294607460F2372682046FFF736
:10BC80009FFE4FF46E418046E5E7B7F5A16F2ED1D8
:10BC90004EF69058326829462046FFF761FE07AB02
:10BCA000074629460093204606AB7268FFF7C8FD99
:10BCB000002800F0AF810723069A29462046FFF7A7
:10BCC0007FFE4FF47F730646079A29462046FFF70A
:10BCD00003FFFB02B90103F4704301F0400143EAA2
:10BCE000900041EA080140F4206231435DE740F2F0
:10BCF0000E539F424AD14EF68058CBE7B9F1030F5D
:10BD000044D1DFF8C081002700F1010A0322414637
:10BD100050461DF0C2F9A0BB2B7993BB644B29465A
:10BD20003268204613F82780FFF71AFE726807462C
:10BD300029462046FFF714FEB26881462946204670
:10BD4000FFF70EFE08F0F001FB02420141F46E41E4
:10BD500003F47043BF0102F0200207F040071A43CA
:10BD600042EA50034FEAC91247EA5909D2B249EAF6
:10BD7000010113434FEA0812D2B242F420621A437F
:10BD800013E7013708F10408042FBFD14B462A46B8
:10BD90004849494803F02CFE636A18603AE1B9F15A
:10BDA000000F10D140F245439F4205D14FF43F416F
:10BDB0002046FCF787FE2DE140F211539F42E5D16A
:10BDC0004BF63071F4E7B9F1010F40F0038140F216
:10BDD0005D32974212D1014632682046FFF78CFD52
:10BDE00001462046FCF7FCFE002840F01381646AFF
:10BDF0003249314803F072FD20600BE1B7F5597FFD
:10BE000009D1014632682046FFF776FD01462046FB
:10BE1000FCF73AFFE8E740F26B32974209D101465E
:10BE20000F2332682046FFF7CBFDC00040F48E415F
:10BE3000BEE7622B48D1059B032B0CD0052B40F0AD
:10BE40008D80C3785F2B40F0898003796E2B02D000
:10BE5000772B40F0838069780022194B4FF0FF3731
:10BE60005878884205D195F802C09878844508BF73
:10BE70001F78013203330E2AF2D17B1C86D0326840
:10BE800029462046FFF738FD059B0246052B09D1C0
:10BE90002B79A3F177056B426B4139462046FCF7BD
:10BEA000BDFEA1E70023F8E7D6350560E035056063
:10BEB0004837056006360560004C05603B36056076
:10BEC000B436056049370560692B47D14378742B38
:10BED00044D13068FFF738FDB74B017800221F4688
:10BEE0005E788E4228D190F801C09E78B44523D167
:10BEF00086780EBBAE1C31460B46013118780028FF
:10BF0000FAD1691D8B423FF641AF02EB4202013B81
:10BF10000821BA5C12F0010F4FEAC2000CBF4FF0CB
:10BF2000080C4FF0000C00F00800B34209D241EABF
:10BF3000021141F43F413BE7013203330E2ACFD1D6
:10BF400024E713F801794908742F01D10143ECE784
:10BF5000652F7FF41BAF4CEA0101E6E740F287331F
:10BF60009F4202D14BF2726122E7B7F5627F02D1A4
:10BF70004BF262611CE740F26D439F4213D132687D
:10BF800029462046FFF758FD10F43F4F024607D1DF
:10BF900050044ABFD1B242F4344141F4354107E77D
:10BFA0004EF62D1101E6782F7FF4F0AE3268294667
:10BFB0002046FFF741FD10F4FE4F024607D1010471
:10BFC0004ABFC1B240F43C4141F43D41F0E64EF677
:10BFD000BD01EAE5B9F1020F40F0AE81736803F0EC
:10BFE0000F03022B40F2394340F09E809F4214D150
:10BFF00001460F2332682046FFF7E2FC07467268CD
:10C0000029460F232046FFF7DBFC3946024620462F
:10C01000FCF7C2FD08B0BDE8F08740F279339F42DB
:10C020001CD14FF6B0294FF280070F233268294602
:10C030002046FFF7C5FC7268804629460F2320463C
:10C04000FFF7BEFC47EA000249EA000142EA082283
:10C05000ABE54FF690294FF2A007E6E740F27743B1
:10C060009F42F6D040F23D439F422BD101460C2324
:10C0700032682046FFF7A4FC07467068FFF764FCAF
:10C08000014603904D481CF0F2FF98B103994C48CB
:10C090001CF0EDFFA0B12A464A494B4803F0A8FC2A
:10C0A000636A0022186042EA07224FF2EF3142F43D
:10C0B00000427AE50023454A02EBC302D25CF2E774
:10C0C0000123F8E740F252339F4215D14FF48047E5
:10C0D0003268294607232046FFF772FC80467268C3
:10C0E000294607232046FFF76BFC424603463946A4
:10C0F0002046FCF74CFD8DE7DFF8D88000270322AF
:10C10000414628461CF0C9FF40B9EB7833B9304BA3
:10C1100013F827703F0147F48047D9E7013708F14A
:10C1200004080F2FEBD131E69F421CD14FF400578A
:10C130000723326829462046FFF742FC29468046FD
:10C14000FF2372682046FFF7C7FC47EA000141EA77
:10C1500008212DE64FF42057EAE74FF44057E7E770
:10C160004FF46057E4E740F27B339F42F2D0B7F5DB
:10C17000537FF2D040F2C6439F42F1D040F23B439E
:10C180009F4229D14FF240280F233268294620468A
:10C19000FFF716FC07464FF6FF73726829462046E4
:10C1A000FFF79AFC3A46034641462046FCF706FD57
:10C1B00030E74FF2C028E7E7B4360560AD370560D9
:10C1C000B6370560E6350560004C0560AC370560A4
:10C1D000F4360560F536056040F23A439F42E8D0F8
:10C1E00040F23C439F421AD101460F233268204659
:10C1F000FFF7E6FB294607464FF0FF3372682046FB
:10C20000FFF76AFC054683B23A464FF240212046CA
:10C21000FCF7D4FC3A462B0C4FF2C021C5E740F2A4
:10C2200007439F4228D101460F2332682046FFF77B
:10C23000C7FB07AB074629460093204606AB72684A
:10C24000FFF7FEFA00283FF4E5AE0F23069A2946D1
:10C250002046FFF7B5FBFF230646079A29462046EE
:10C26000FFF73AFC46F46841830841F0500143EA85
:10C27000073242F4706298E440F205439F4240D096
:10C2800040F206439F423ED0B7F5816F3DD0972FD5
:10C290003DD040F2C2439F423BD040F2C4439F4254
:10C2A0007FF474AD0523874A2946204632F823706F
:10C2B00007233268FFF784FB07AB804629460093CB
:10C2C000204606AB7268FFF7BBFA00283FF45EAD6C
:10C2D000069A072329462046FFF772FBFA04064612
:10C2E00019D51F23079A29462046FFF7F5FB034679
:10C2F00047EA08079B0147EAC60103F4F8631943BC
:10C3000056E50023CFE70123CDE70223CBE7032344
:10C31000C9E70423C7E73B04079A06D53E2329460D
:10C320002046FFF7D9FB4308E2E77C232946204655
:10C33000FFF7D2FB8308DBE7B9F1030F7FF426ADEB
:10C3400040F217439F4221D1002707233268294634
:10C350002046FFF735FB81460723726829462046B1
:10C3600047EA0907FFF72CFB294680461F23B268DE
:10C370002046FFF7B1FB47EA801747EAC80117E5F7
:10C380004FF40067E1E74FF48057DEE7B7F5836FBE
:10C39000F6D040F259339F42F5D0B7F5537F2BD1F9
:10C3A0004FF4C0580723326829462046FFF708FBA0
:10C3B00007237268074629462046FFF701FBB2684B
:10C3C000814602F00F03022B0ED107232946204697
:10C3D000FFF7F6FA47EAC90747EA080141EA801180
:10C3E000E6E44FF4D058DDE707232946204648F419
:10C3F0008068FFF771FBEDE740F299439F4222D13D
:10C400004FF690380F23326829462046FFF7D8FAB6
:10C410000F238146726829462046FFF7D1FAB26899
:10C42000074629460F232046FFF7CAFA48EA0701C4
:10C4300040EA092040F4704242F0F002FFF7B5BB39
:10C440004FF6B038DEE740F2E5439F42F8D040F2C5
:10C45000C6439F42C5D040F2C3439F427FF496AC8F
:10C4600001460F2332682046FFF7AAFA0F237268AD
:10C47000294607462046FFF7A3FA07AB8046294620
:10C480000093204606ABB268FFF7DAF900283FF4C4
:10C49000C1AD0F23069A29462046FFF791FAFF23E4
:10C4A0000646079A29462046FFF716FB46F46841E0
:10C4B0003B0241F0400143EA083343EA9002FFF7B0
:10C4C00074BB00BF3037056004292DE9F0410646F2
:10C4D0000C46904625D9446A1349144803F0FEF9E6
:10C4E000206000242046BDE8F0810009F6F73DF900
:10C4F00007461CF0B5FD022810D13B78722B0DD1F8
:10C500007A7805F130039A4208D10135A542E9D085
:10C5100058F8250000F00F03022BE6D0746A044996
:10C52000DBE70025F2E700BF4F360560004C0560F1
:10C530008236056038B505463020F5F7ADFF044674
:10C54000202200211CF058FD29462046FCF767FAFE
:10C55000A562A800F5F7A0FFE062204638BD10B53F
:10C560000446C06AF5F7C0FF00212046FCF75FFAD9
:10C570002046BDE81040F5F7B7BF000000000000FE
:10C5800007292DE9F74F9DF8305010D8012905D91A
:10C590003F2300F8013B0023037001E00029FAD19A
:10C5A000012994BF0020012003B0BDE8F08F10EEF8
:10C5B000904A002C044622DAB4EE400BF1EE10FA59
:10C5C0001DD6B1EE400B2D2504F8015BB0EEC07B0B
:10C5D00002F020089FEDCE6BB4EE467BF1EE10FA30
:10C5E00012DD88F0490388F04605E11C237088F0CD
:10C5F0004E03A57063700023081A0B70D4E7002D5A
:10C60000E4D004F8015BE1E7B4EE400BF1EE10FA80
:10C6100008D748F04E0388F04105E11C237065708F
:10C62000A370E8E7002BA4EB000542F02002B8BF9E
:10C630000623491B672A01F1FF3662D1B5EE400B94
:10C64000002B08BF0123F1EE10FA00F0A580B7EE31
:10C65000007BB4EEC70BF1EE10FA40F1CB8000275F
:10C66000DFF8C4E24FF4807CDFF8C0A23D469FEDC6
:10C67000AA6BB4EEC60BF1EE10FAACBF4FF0310965
:10C680004FF03009BEEC025BB4EEC05BF1EE10FA85
:10C6900006DD0AEB070B65449BED005B20EE050B06
:10C6A00008374FEA6C0C482FECD1B4EEC70BF1EE13
:10C6B00010FA40F18380B4EEC60BF1EE10FA78DB8D
:10C6C000002DB7EE000B14BF2D272B27662A05D0AF
:10C6D000672A40F08480042D00F38180672A84F863
:10C6E000009004BF05F1FF37DB195F1CB742A8BFFC
:10C6F000CB1E002B64D101341E461F464FF0FF3C79
:10C70000B0E0B5EE400BF1EE10FAA0D1662A43D1AD
:10C710005D1C0027B542BC463D46A8BFCB1E662126
:10C720005E1C652923EAE37E40F0C1800EF101061C
:10C73000B2EE046B00234FF02E0B0193019B9E423F
:10C7400000F3BE80662A40F0F380B54240F3448196
:10C75000F7B1632D4FF00A0148F045086770CABF72
:10C760006423A61CE61C84F80080C2BF95FBF3F38B
:10C770003033A370344695FBF1F393FBF1F201FBE8
:10C78000135501FB12323035303204F8022B75702C
:10C790000023201A237007E75D1DB5424FF0000605
:10C7A000A8BFCB1F652A11467BD12B27B44635463F
:10C7B000B7E7B2EE047B013520EE070B2D2785E7A6
:10C7C0002E211E46023404F8011C3021013D6AD09E
:10C7D0000EB9374692E7013E04F8011BF6E7CE1F7B
:10C7E0009E4203DC672A60D0A1F1080311460026AF
:10C7F000B44696E70027DFF834E14FF4807CDFF899
:10C8000028913D46BEEC027BB4EEC07BF1EE10FAFF
:10C8100006D809EB070A65449AED007B20EE070B6A
:10C8200008374FEA6C0C482FECD1FDEEC07B17EEB9
:10C83000907A092F04DD01359FED397B20EE070B3F
:10C84000662A11D1B54217DA59190131B14205DB17
:10C85000761B012EA6F1020308BF0023EE18AC469A
:10C860000027013666215CE7652A05D0672A0DD0CE
:10C87000114600262B27BBE7CE1F9E4201DCA1F10B
:10C88000080300262B276521B4464AE75F1DB742FF
:10C8900000DBCB1F9D4201DB6721EAE7691C5B1AC5
:10C8A000DCE7374682E72F4628E733469EE76729CD
:10C8B0007FF43EAF002BD6BF01267646B64637E75B
:10C8C000BDEEC07B04F1010A17EE103A002BA8BFA1
:10C8D00003F13009019BB4BF4FF030095FFA89F9C9
:10C8E0009C4584F8009006D1BEF1000F03D004F1FE
:10C8F000020A84F801B0B8EEC77B019B54460133AD
:10C9000030EE470B019320EE060B17E7AFF30080E4
:10C91000FFFFFFFFFFFFEF7F1450FFFFFFFFEF3F21
:10C920009A9999999999B93FC03705600838056077
:10C93000B1EE047BB4EEC70BF1EE10FA24DB631EFC
:10C940004FF030091E7803F1FF3C2E2E2ED0A6F1B9
:10C95000300ABAF1090F2BD901331E78302E13D1CA
:10C9600093F801C0BCF12E0F2FD166292DD02D2FA9
:10C9700083F800C05E7026D1013D08BF2B272146F9
:10C980008B4224D331211970672A7FF4E1AEBEF1C6
:10C99000000F3FF4DDAE23461C46013B14F8012C8A
:10C9A000302AF9D02E2A08BF1C46D1E66346C9E7D3
:10C9B000392E02D001361E70CFE798428CF80190D4
:10C9C000F4D10346C9E70135D9E70134D7E711F8B7
:10C9D000016C01F80169D3E7B1EE047BB4EEC70B3B
:10C9E000F1EE10FAABDAB3E6012910B5146827D9D5
:10C9F00034F01001037814D1302B1DD14178831C01
:10CA000041F02001782903D110211160181A10BDBE
:10CA1000CCB96F2901D10821F7E7622911D1022190
:10CA2000F3E7082C11D1302B0DD1437843F02003CC
:10CA30006F2B08D1831CE9E7082C04D0022C02D00C
:10CA40000CB90A2313600346E0E7022CFBD1302B1C
:10CA5000F9D1437843F02003622BEAE7044608B596
:10CA600031B1054B4A6C03600023096802F0FCFFFA
:10CA70002046F5F7EDFC00BF004C05602DE9FF47AF
:10CA80001E464518019212B1023A222A34D80446B1
:10CA9000AC42274639D214F8010BF6F7F7FB804673
:10CAA0000028F5D13B782B2B29D12746E91B3846A6
:10CAB00001AA0024FFF798FF0744B946A9454B4651
:10CAC00026D3B8F1000F00D06442640044F00104A2
:10CAD000BB4209D01F46AF423B4641D218780137CE
:10CAE000F6F7D4FB0028F6D12049019A204802F03D
:10CAF0007FFF3146FFF7B2FF1E4840F03DFC2D2B73
:10CB000004BF27464FF00108D0E74FF00008CDE7FB
:10CB100019F8012BA2F1300ABAF1090F09D95F2ADD
:10CB2000CCD042F02002A2F161011929C9D8A2F1AA
:10CB3000570A01995145C4D920460CF011FA28B979
:10CB4000019B03FB04A494EA4403B7D5019B42462E
:10CB5000E91B03A8039704F045F9039B0446B7E7D4
:10CB6000C2D1204604B0BDE8F08700BF733805602D
:10CB7000F04C0560503805602DE9F04F2DED048B29
:10CB800083B0044691464618DDF840800193B442D4
:10CB9000254680F0318128780134F6F777FB074687
:10CBA0000028F4D12B782B2B09D125468246B4429C
:10CBB0000CD300239FED949B1F4618468AE02D2B33
:10CBC00003D125464FF0010AF1E782462B7843F066
:10CBD0002003692B31D1AB1C9E4240F205816B785A
:10CBE00043F020036E2B40F0FF80AB7843F020032E
:10CBF000662B40F0F980EB1DEC1C9E421AD9EB78B5
:10CC000043F02003692B15D12B7943F020036E2BC1
:10CC100010D16B7943F02003692B0BD1AB7943F032
:10CC20002003742B06D1EB7943F02003792B01D13B
:10CC300005F108049FED768B14E06E2B2AD1AB1C16
:10CC40009E4240F2D1806B7843F02003612B40F08C
:10CC5000CB80AB7843F020036E2B40F0C580EC1CFA
:10CC60009FED6D8BBAF1000F01D0B1EE488BA5425C
:10CC700009D0B442234680F0998018780134F6F741
:10CC800005FB0028F5D16A496A4802F027FE4146B3
:10CC9000FFF7E4FE0023B2EE045BAC4618461946EB
:10CCA00000939FED599B9FED5E6B644614F801EB7A
:10CCB000AEF1300BBBF1090F39D8022923D15E4AFE
:10CCC000904202DC0A2202FB00B0A6425FD8009A22
:10CCD00002B14042034413F59A7F05DC03F233139B
:10CCE0009FED517B29EE079B13F1160F53D35B4247
:10CCF000B2EE040B01EE103AB8EEC11B16F018F8B4
:10CD000089EE008BAEE7B4EEC69BF1EE10FA0BD5C0
:10CD100007EE90BA0129B8EEE77B09EE057BB0EE8D
:10CD2000479B31D1013BD0E729B90133CDE721B988
:10CD3000BEF12E0F03D10121C7E7022917D04EF013
:10CD4000200BBBF1650F12D1A64258D99CF80110F7
:10CD50002B2905D10CF10204B44294D00221B4E78E
:10CD60002D2913D101220CF102040092F4E7B9F14C
:10CD7000000F04D04EF0200BBBF16A0F09D0BEF1BA
:10CD80005F0FA2D06446A2E700219EE70221A446DD
:10CD90008BE74F469BE707EE903AB2EE040BB8EEF6
:10CDA000E71B15F0C5FF29EE008B5BE77FF46BAF47
:10CDB00057B1B0EE481B9FED140B03B0BDEC048BD4
:10CDC000BDE8F04F01F074BE019B23B1B0EE480BFB
:10CDD0009FED0D1BF1E7B0EE480B03B0BDEC048BEB
:10CDE000BDE8F04F02F04CBFBAF1000F3FF44BAF7B
:10CDF0002C469FED058B38E74FF0000AD9E63FF44B
:10CE000042AF64E7AFF300800000000000000000C4
:10CE1000000000000000F07F000000000000F87F2C
:10CE20005A62D7D718E774690DC6402C18FA31003A
:10CE30009B380560F04C05606466660608B51020F6
:10CE4000F5F743FB0121027861F30202027008BD8D
:10CE500003F07F0310B50488DB0024F47F7443F0F3
:10CE6000020324F003042343C0E90112038010BD30
:10CE700070B503F11F0422F01F05144424F01F04B1
:10CE8000631B002B0CDDBFF34F8F174EC6F86852A3
:10CE90002035631B002BF9DCBFF34F8FBFF36F8F7F
:10CEA000BFF34F8FBFF36F8F0F4B0024C3F8504277
:10CEB000BFF34F8FBFF36F8F049B01F007014260F8
:10CEC0008360059B094ADB0003F47E730B430699DC
:10CED00002EA812213430268520D52051343036094
:10CEE000079BC36070BD00BF00ED00E000FC1F00A9
:10CEF00038B504460D4610462378616803F00703F1
:10CF0000042B0BD8022B0BD9A3682A4603F07EFA18
:10CF100023881A0701D50B4B036038BD052B08D0B9
:10CF2000A3682A4603F044FA23881B07F5D5064B6D
:10CF3000F2E72068E268C0F38A20BDE8384003F0D9
:10CF40006DBA00BFA05105606451056038B5144644
:10CF500012F480721D4618BF1A46FFF7C9FF620916
:10CF6000E1B202F008022A44BDE8384001F026BDD3
:10CF7000D0E90003184770B505460C468E18B44238
:10CF800000D170BDD5E90003984704F8010BF6E71E
:10CF900038B504460025D4E90003984700F07F0324
:10CFA00043EAC5150306F6D4284638BD2DE9F041FD
:10CFB00086B00546FFF7DCFF10F0FF0453D0012CCC
:10CFC00053D0022C53D0032C53D0042C53D02846DA
:10CFD000FFF7DEFF064648B9062C07D1274C284646
:10CFE000FFF7C6FF204606B0BDE8F0810A2C10D13D
:10CFF0000021304607F0C2FE0027044600F1080871
:10D00000B742EFD028460137FFF7D0FF48F8040BAE
:10D01000F6E7314602A8F5F779FC3246049928462E
:10D02000FFF7A9FF631F012B0CD82846FFF7A0FFCD
:10D030001348144B02A9052C18BF184605F05AFED8
:10D040000446CFE7072C4FF00003DDE9031003D1BE
:10D050000A22FFF713FDF3E7093C009362426241A5
:10D06000FFF78AFDECE7084CBCE70624BAE70E247C
:10D07000B8E71E24B6E7054CB4E700BF5060056072
:10D08000EC62056060600560643B0560705B056094
:10D090002DE9F84305460E4617460024DFF8A08028
:10D0A0002868FFF765FF5FFA80F9B9F1FF0F01D13A
:10D0B000BDE8F883C2070CD52868FFF769FF10F0B8
:10D0C000010F4FEA500016BFAC6806EB800404EB7A
:10D0D0008004B9F10B0F4FEA590311D8DB070DD5C6
:10D0E0002868FFF755FF5FEA990927D0B9F1010FCA
:10D0F0000CBFAB68EB68024621461AE00120F2E75C
:10D10000062B03D16B689B680120F4E7072B02D143
:10D110006B68DB68F8E7082B17BF03F180434346D1
:10D12000093B58F82330EFE751F804CB9C4441F811
:10D1300004CC013AF8D204EB8004B1E73B46DAE7CD
:10D14000643B05602DE9F04F91B007460A91FFF767
:10D150001FFF00F003034FEAD0099A1C069200F06B
:10D16000040248460792002B3ED14FF0000AF5F723
:10D1700093F94A4601465546D04656460446384637
:10D18000FFF7F9FECDE908AA079B002B00F0998074
:10D190003846FFF7FDFE069A03460790032A08BFAC
:10D1A00001339800F5F778F9079A8346059000EB6C
:10D1B000820293457CD1FFF741FE069B8346022BFA
:10D1C00040F0898022460023E64312F8011B09063D
:10D1D00002EB060578D4059A21465846FFF738FE3B
:10D1E000584611B0BDE8F08FF5F756F94A460146AA
:10D1F00004463846FFF7BFFE069B3846032B1BD17B
:10D20000FFF7C6FE23180646225C591C4FF00008A3
:10D21000DB43100601EB030506D44FF0000A554628
:10D220000023CDE90833AFE711F8012BC2F38010DA
:10D23000A84048EA0008ECE7FFF7AAFE069B8046F4
:10D24000052B09D138460026FFF7A2FE05463846D1
:10D25000FFF79EFE8246E3E710F0200521D0384616
:10D26000FFF796FE824618F0400002D03846FFF7DE
:10D270008FFE1AEB000616D0033020F003060AEBEF
:10D280000600F5F722F903460890334409932DB1BF
:10D290000025524619463846FFF76DFEAA462E462F
:10D2A00072E7AA46DFE7B2463546CDE908666BE786
:10D2B0000A9938460B92FFF745FF0B9A4BF8040B7F
:10D2C00077E7089B059376E712F8011BC1F38010FE
:10D2D000A84003437BE70A9B18F0100F0C970D93AF
:10D2E000099B0E93089B0F9312D0164FD7F8D010BE
:10D2F00021B9084604F072F9C7F8D0002146D7F8E2
:10D30000D00003F014FF224621460CA8FFF7C0FE10
:10D31000069B032B06D1079B264483B1059B079AE6
:10D3200043F82260059B22460699584600934B46D7
:10D33000CDF80480CDE9025AFFF79AFD50E7059633
:10D34000F0E700BFB02700202DE9F74F0D46164645
:10D350000422074628460DEB0201FFF70CFE9DF85C
:10D3600004304D2B0BD19DF80530062B07D19DF8CD
:10D3700006309A0703D19DF807201F2A02D92F48AB
:10D380003FF0FAFF9B0804D0043B042B01D92C4842
:10D39000F6E728464FF0000AFFF7FAFD81462846D7
:10D3A0004FEA4904FFF7F4FD8046033400EB940094
:10D3B00024F003048000F5F76FF8B0602044F060BB
:10D3C000CA4510D1002444452FD131462846FFF7E5
:10D3D000B9FEAB680446286898473846C7E9006438
:10D3E00003B0BDE8F08F2846FFF7D2FD10F0010F23
:10D3F0004FEA500413D12046F5F74EF82246014675
:10D4000083462846FFF7B7FD2846FFF7B1FD2146C2
:10D410005846F5F7EBF804465846F5F765F8B36853
:10D4200023F81A400AF1010ACAE7D6F80C902846F8
:10D43000FFF7BCFD49F824000134C4E7B5380560A6
:10D44000CC38056010B586B0044603A8019211F0EF
:10D4500095FF2046019A03A9FFF776FF204606B004
:10D4600010BD0000054B9861B3F8502312B2012A99
:10D4700002D10022A3F85023704700BFB02700203C
:10D48000024800233C308360FFF7ECBFB027002048
:10D49000EFF3108172B6084AB2F850331B0408D576
:10D4A000B2F85033013B1BB2A2F8503381F310881D
:10D4B00070474FF6FF73F7E7B0270020EFF31081B6
:10D4C00072B60C4BB3F850231846013212B2A3F8CF
:10D4D00050233AB99A6912B993F852232AB100231A
:10D4E000A0F8503381F3108870470122A3F850232D
:10D4F000F8E700BFB0270020114B4FF6FF7270B560
:10D5000093F852530446A3F85023B5B193F853232C
:10D51000013DD10001325C3102F00702CE18C8583B
:10D52000716883F8532383F8525384F3108840F0D2
:10D5300067F8BDE87040FFF7C1BF80F31088F8E7D7
:10D54000B0270020114BB3F8502312B210B5E2B946
:10D55000EFF3108172B6B3F8502312B29AB99C69F6
:10D5600064B19A6193F8522312B90122A3F85023AF
:10D5700020B181F310882046F4F76AFF0846BDE821
:10D580001040FFF7B9BF81F3108810BDB02700200D
:10D5900070B5EFF3108572B60F4B93F85223082A3B
:10D5A00018D0B3F8504324B2012C02D10024A3F8C0
:10D5B000504393F85343561C224483F8526302F0BD
:10D5C00007020B3203EBC203C3E90101012085F31B
:10D5D000108870BD0020FAE7B027002038B1044A57
:10D5E0001369984202D010611846704700207047B6
:10D5F000B027002001F00F01012903D0022906D035
:10D6000039B97047002814BF1E200E20704703F060
:10D6100059BB03F0DDBB00F087BA08B500F084FA0F
:10D62000B7EEC00B08BD02F02BBBB7EEC00A02F08C
:10D6300027BB0000F0B593B005460F461446684678
:10D640001668F4F7EDFE78B9002E234632462846D8
:10D650000CBF394600213FF0E7FE0546F4F7D8FE3F
:10D66000012D0BD1284611E0019B23601049206851
:10D6700002F0E9F960B92068F4F7EAFE2368002DAA
:10D68000F4D10BB9062323603EB9002013B0F0BDDE
:10D69000206802F0F9F82060F6E70649304602F00B
:10D6A000D2F90028F1D030463FF0A2FFE4E700BFF6
:10D6B000C44B05607C480560036803B940683FF0CF
:10D6C0007FBF1346C1F30722C9B23FF035BF1FB574
:10D6D00001F00F030446012B11D011F00E0F08D1F9
:10D6E0007BB1012201A9204600F011FC58B101983C
:10D6F00007E0023B012BF4D800F0B8F901E000F09C
:10D7000025FB04B010BD2046F6E708B528B1062871
:10D7100003D03FF06DFFF4F79BFE08BD10B50C463B
:10D7200019B9BDE810403FF09FBE3FF09DFE844216
:10D730001CBF0023C4E90030002010BD40F26B4341
:10D74000984217D8B0F58D6F09D25E281DD0752884
:10D750001DD03E2814BF4FF0FF30012070476FF4FA
:10D760008D631844022803D8DFE800F00B0D130086
:10D7700004207047B0F59D6F14BF4FF0FF300320B9
:10D78000704706207047072070470220704700202E
:10D7900070470520704738B5034615460C4609B951
:10D7A0002C460BE052B111462046984758B16368A9
:10D7B00033B9656044F00103A560EB60204638BDD5
:10D7C000A368DD60F6E76B68E3606C60002BE7D16F
:10D7D00045F00103AC60E360E2E7F8B5064631B11D
:10D7E000002511F0010304D000232946EB60084610
:10D7F000F8BDCC68CB6014F0010307D1E76822467E
:10D80000E3603046FFF7C7FF3C4601460A46304614
:10D810002946FFF7C0FF21460546E2E78A428446D3
:10D820002DE9F0410E4606D100235168BDE8F041D4
:10D830005360FFF7D2BFD2F80C80B8F1000F12D0BE
:10D840001446E468E307FCD524F00104516808F0AD
:10D8500001076368934216D1002339B99F4208BF7C
:10D8600041466160D3603046BDE8F0816046536058
:10D87000D360FFF7B2FF05466060C5F80C80002F4B
:10D88000F1D0A560EFE71D46DB689342FBD1002293
:10D8900060465A60DA60FFF7A0FF0028EDD0E8602C
:10D8A0000546EAE7014B1860704700BFB02700202B
:10D8B00082B0034B186801ABC01A02B0704700BFBA
:10D8C000B0270020014B5860704700BFB0270020F0
:10D8D00007B5064A01A9136852685B1A9A4201D833
:10D8E0003FF07AFD03B05DF804FB00BFB0270020D5
:10D8F000704710B50C46F4F7CFFD046010BD000072
:10D9000083070FBF006800F00F00024B53F82000A0
:10D91000704700BF0C40056008B5FFF7F1FFC088F5
:10D92000BDE80840F4F721BF37B50D460446019223
:10D93000FFF7CEFF2846FFF7E3FF836833B1019A74
:10D940002946204603B0BDE830401847C28820462B
:10D95000024903B0BDE83040F5F748BC423E0560DF
:10D960000A4601460148FFF7DFBF00BF04780560A3
:10D970002DE9F347044608460E4602F05DF898B1DB
:10D9800001AA6946304602F0AFF8009B63B11A491C
:10D990002046F5F7AFF8009D184F033DDFF864808F
:10D9A000DFF85C90002D0BDA022231462046FFF7AB
:10D9B000BBFF13492046F5F79DF802B0BDE8F0879C
:10D9C000019A394620464FEA850A02EB850352F850
:10D9D00025205B68F5F70AFC019B53449A682AB935
:10D9E00049462046F5F786F8033DDBE741462046E9
:10D9F000F5F7FCFBF8E700BF473E05606B3E0560AE
:10DA0000583D0660803E056008B50246FFF778FF86
:10DA100006490069884203D0003818BF012008BDBC
:10DA20001046BDE8084008F023B800BF99580160CF
:10DA30000E28014608B513D01E2813D0C20701D501
:10DA4000401008BD830707D10268074B9A4203D1F3
:10DA5000BDE8084003F0E6B908203FF0A5FCF7E771
:10DA60000020EEE70120ECE79C520560C20705D4D8
:10DA7000830705D10268034B9A4201D103F0CAB96A
:10DA8000FFF7D6BF9C5205600E2810B50C4603D197
:10DA900000230B60012203E01E2803D101220A604B
:10DAA000104610BD10F0010202D043100B60F7E7E2
:10DAB0008107F5D10168034B9942F1D103F0B2F926
:10DAC0002060E7E79C5205600E2810B50C461DD07B
:10DAD0001E281ED010F0010209D0431000EE103AAB
:10DAE000B8EEC00B012284ED000B104610BD81077B
:10DAF000FBD103680A498B4202D103F0D1FAF1E766
:10DB000008498B42F1D102F022F9EBE79FED020BBD
:10DB1000E8E7B7EE000BE5E70000000000000000BA
:10DB20009C520560004E056013B569460446FFF738
:10DB3000CBFF38B92046FFF7EFFE04490246044800
:10DB40003FF012FD9DED000B02B010BD893E056057
:10DB5000784C05600E28F8B50D46144607D1002212
:10DB60000023C1E90023C4E90023012616E01E2892
:10DB700006D10022164BC1E9002300220023F2E760
:10DB800010F001060CD04310002207EE903A00235B
:10DB9000B8EEE77B81ED007BC4E900233046F8BD99
:10DBA0008707FBD103680B4FBB4204D103F078FA1F
:10DBB00085ED000BE1E7084FBB4202D102F0C7F848
:10DBC000F6E7064CA342E9D101F03EF8CDE700BFED
:10DBD0000000F03F9C520560004E05609C430560CC
:10DBE00010B50446FFF7B6FF38B92046FFF794FE9C
:10DBF0000249024602483FF0B7FC10BDA33E056053
:10DC0000784C056038B5840703460ED104680B4D87
:10DC1000AC4203D1BDE8384007F0B8B9084DAC427A
:10DC200003D1BDE8384003F0EFBC1846FFF774FE9F
:10DC30000449024604483FF097FC00BF7065056048
:10DC400034540560BF3E0560784C056013B50C4642
:10DC500001A9FFF7D7FF019BA34204D02246034945
:10DC600003483FF081FC02B010BD00BFE13E0560FB
:10DC7000F04C0560F0B51F46D30785B006460D464B
:10DC800014460FD554100394039A002ABCBF5219AE
:10DC90000392039ADFB1002A15DA00230393039855
:10DCA00005B0F0BD03A91046FFF7EEFE0028EBD14A
:10DCB000F28820460192FFF72FFE019A0346084999
:10DCC00008483FF051FCAA42E9D90395E7E7002A4A
:10DCD00001DBAA42E3D3F288034904483FF044FC45
:10DCE0000E3F0560784C0560323F056030490560A5
:10DCF000820701D002F0E6BF002803DB400040F0BD
:10DD00000100704703F064B88307014610B510D1D5
:10DD100002680D4B9A420CD100F00703022B06D18A
:10DD2000C008F4F717FD400040F0010010BD806806
:10DD3000F9E70846FFF7E4FD43691BB10520BDE89C
:10DD4000104018471846F1E7606005600E2810B5CE
:10DD500004461FD01E2801D1012010BD062819D06D
:10DD6000C20703D5013818BF0120F6E7FFF7C8FD49
:10DD7000436943B121460420984720B1A0F11E0316
:10DD800058425841E9E72046FFF7BEFF0028E3D09C
:10DD90000138E8E70020E0E705282DE9F84F15BF36
:10DDA0001E260E264FF00E094FF01E09914207461F
:10DDB0000C46154607D1C80720D40846FFF7A0FD3A
:10DDC000838859071AD504F00703022B05D0A20750
:10DDD00017D122682A4B9A4213D105F00703022B70
:10DDE00005D0AB0712D12A68254B9A420ED129469D
:10DDF000204605F05DFC002808BF4E463046BDE8D1
:10DE0000F88F14F0010A06D0E80734D423464FF007
:10DE1000010A2C461D462046FFF772FDD0F818B0C7
:10DE20008046BBF1000F10D08288110704D4284629
:10DE3000FFF766FD804508D1052F0DD0D8F81830C2
:10DE40002A4621460220984780B9BAF1000FDDD05A
:10DE5000AC4218BF4E46D1E7D306EFD52A4621463D
:10DE60003846D8470028E9D00646C7E7022F04D035
:10DE7000FFF76CFFBFE74E46C0E70646BEE700BFB0
:10DE8000EC6205600A460146022008B5FFF784FFF0
:10DE9000BDE80840FFF75ABF10B50446FFF734FF4E
:10DEA00038B92046FFF738FD0249024602483FF0E4
:10DEB0005BFB10BD483F0560784C056038B50446F3
:10DEC0001546FFF71DFD036A13B120469847A0B918
:10DED000204635B9FFF720FD0849024608483FF0C3
:10DEE00043FB042D04D1FFF717FD06490246F5E771
:10DEF000FFF712FD04490246F0E738BD693F0560AF
:10DF0000784C0560933F0560B33F0560704710B5DE
:10DF10000446FFF7F5FCC36A2BB120469847B0FAD8
:10DF200080F0400910BD1846FCE7000008B5FFF777
:10DF3000EEFF10B901483FF01FFB08BDDF3F056051
:10DF4000062806BF480040F0010000207047042862
:10DF500003D0052807D0002070478B68002B14BF22
:10DF60001E200E2070478868400040F00100704776
:10DF7000084B0268C1E900300023C1E90233064BB7
:10DF80009A4208BF4368084604BFC3F317238B6057
:10DF9000704700BF54410560CC410560F8B50D469F
:10DFA00001790446164601F07F010022402008F066
:10DFB00019FBA368E268434327682A606B602379F2
:10DFC00003F07F01A96008498F4209D1190601D4E5
:10DFD000B30707D46368C3F3172300FB032028604B
:10DFE0000020F8BD0120FCE7CC410560F8B5002217
:10DFF00005460E460146402008F0F4FA0746102078
:10E00000F4F74AFA094A0A4B04460571012D18BF74
:10E010001346036043686FF31F23C0E9013606FB14
:10E0200007F0F4F739FAE0602046F8BD18410560C2
:10E03000904105607FB504460122084601A9FFF71B
:10E0400075FF00222179402008F0CCFA029D636818
:10E050000646B5FBF0F5B5EB132FC3F3172219D91C
:10E06000A16829444143E068F4F731FA6368E0604D
:10E070006FF31F23636005FB06F20199D4E90203E5
:10E0800000FB06301AF078FFA36806201D44A56047
:10E0900004B070BD521B62F31F23EBE7F7B546686F
:10E0A00004460B4636F0FF061FD132460191017936
:10E0B000402008F097FA62680821054661F31F22A4
:10E0C000A168083162604143E068F4F700FA6268D1
:10E0D000A168C2F31722E06001FB05573146013AFF
:10E0E00038446A431AF088FF019B2079D4E9022161
:10E0F00008F036FDA36806200133A3606368A3F52A
:10E100008073636003B0F0BD4268C36891688B425E
:10E1100030B40AD214795D1CD1688268C56004F0FD
:10E120007F001A4430BC08F0FDBA002030BC7047B4
:10E130002DE9F04F044687B00D4616460AB9002572
:10E14000C6E011F003078068DFF8149240F0D68033
:10E150000B687D4A934240F0D1806A4607F0BEFECC
:10E1600010B97A483FF044F92179042E3A464FF02D
:10E17000400001F07F0100F0948008F033FA16F0BF
:10E180000302054659D133687149186A884247D15C
:10E190003179402001F07F0108F024FAA84202D032
:10E1A0006C483FF0E9F833684B45D6E9028B04D15F
:10E1B0007368C3F3172305FB03BB2368E6684B456D
:10E1C000DDE90002A2EB000AA8EB0A0737D194F9B7
:10E1D0000430002BB3DA002FE2D16368C3F31723B6
:10E1E00005FB036605FB08F2594605FB00601AF0C3
:10E1F000EBFE0199A2680098521A05FB01614044A8
:10E200006A4305FB00601AF0DFFEA068AAEB080273
:10E21000002138446A4305FB00601AF0EDFE35E04A
:10E220004D4A934209D1012DBAD12A4603A930465D
:10E23000FFF77CFEDDE903B8BFE7484892E7002F0F
:10E24000D0DD6368B7EB132F0BD9A1683046394492
:10E250006943F4F73CF963680646E06067F31F23FF
:10E2600063600098A268404401993A4401FB05614B
:10E27000121A05FB00606A431AF0A6FE009805FB1F
:10E2800008F2594600FB05601AF09EFE6368C7EB72
:10E29000132262F31F236360A3681F44A76006254F
:10E2A00016E008F09FF9236806464B4514D110206C
:10E2B000F4F7F2F8054694E80F0085E80F00009A9D
:10E2C00002EB112363F31F216960019B9B1AAB6072
:10E2D000284607B0BDE8F08FDDE900312079C91A82
:10E2E000FFF784FEE1680546C068DDE90032D21A16
:10E2F00006FB031172431AF03FFEE9E700232A46AA
:10E3000001462068FFF7B6FC236802464B4511D151
:10E310006368042E00EB13220ED094F90430002B16
:10E32000BFF60DAF20793346E16800F07F0008F0BA
:10E3300017FCB4E7042EF5D12079E16800F07F00E6
:10E3400008F0F0F90546C3E7D45B05604C40056072
:10E3500031E100607D400560606005609E400560C1
:10E36000CC41056001282DE9F043074685B00E46F3
:10E3700008D08B0724D10B68254A934202D0254A46
:10E3800093421DD1012201A93046FFF7C0FDB8B16B
:10E3900000223946402008F025F9029E0546B6FBCA
:10E3A000F0F638463146FFF721FE06FB05F204463B
:10E3B0000199C0681AF0E0FD204605B0BDE8F08381
:10E3C0003046FFF7A1FC054600B145102946384606
:10E3D000FFF70CFE0021044630463FF045F84FF0B1
:10E3E0000008064630463FF0EBF803460028E3D02D
:10E3F00025B919462046FFF751FEF3E708F1010958
:10E400004246E1683846C84608F0AAFBEAE700BF82
:10E41000606005609041056038B50D461C461146A8
:10E42000094A28463FF02CF8206805F0A1F9012D93
:10E43000007804D10021BDE83840FFF7D7BD6168FE
:10E44000BDE83840FFF78EBF040002000B79012BB6
:10E45000F7B505460C4610D11B490193F4F74AFB6A
:10E46000019B2846D4E9022104F09CFA174928466A
:10E4700003B0BDE8F040F4F73DBB1A461449F4F789
:10E48000B5FEA368002BF1D00026124F1249284692
:10E49000F4F730FBA368B34204D810492846F4F7D8
:10E4A00029FBE3E71EB139462846F4F723FB324641
:10E4B000E1682079013608F035F901220146284645
:10E4C000FFF732FAE6E700BFC1400560673F05602D
:10E4D000CD400560DC400560D84005600411066051
:10E4E00037B50C46114606221D4620463EF0C8FFB1
:10E4F00034B92146012003B0BDE83040FFF776BDB6
:10E500002968CA070BD48B0703D10A680C4B9A42BF
:10E5100005D0012003B0BDE83040FFF723BF084617
:10E52000FFF786FA014601900120FFF75FFD0446E0
:10E53000019A0021C0681AF05FFD204603B030BD8B
:10E540009C5205601B2870B506468CB00C461546DB
:10E5500026D005D8042867D90E284CD0002447E0DF
:10E560002428FBD1012203A92846FFF7D0FC00286C
:10E570004AD0A10756D12268454B9A4252D1012276
:10E5800009A92046FFF70AFD0123DDE909010093EF
:10E59000DDE9032304F0DCFA002843D01E2427E041
:10E5A000012206A92046FFF7F9FC2846012209A905
:10E5B000FFF7BCFC00229DF82010402008F012F864
:10E5C0000A9EA1680546B6FBF0F69DF8200031448E
:10E5D000FFF70CFD0446C068DDE906121AF0CCFC1A
:10E5E000E068079B06FB05F2099918441AF0C4FC81
:10E5F00020460CB070BD0A68264B9A42AED0294620
:10E600002046FFF717FDF3E7EA0702D500203EF0AA
:10E61000EFFEAB0706D12B681F4A9342F6D01F4A84
:10E620009342F3D00E24E3E7012206A92046FFF728
:10E63000B5FC012209A92846FFF769FC0028F1D0A2
:10E64000089A012A1DD05A2A1DDC203201460B9B54
:10E65000012B1AD05A2B01DC203301469342D5D12D
:10E6600023F00203642BD1D0022E01D00029CDD09B
:10E670000A9B30460093099BDDE9061207F06DFC0A
:10E680008AE74222E1E70021E1E74223E4E700BF15
:10E6900090410560CC4105609C520560004E0560CC
:10E6A00070B50646102014460D46F3F7F5FE054AF0
:10E6B000067102604268C4606FF31F22C0E9012541
:10E6C00070BD00BFCC4105607FB51D4608461146B0
:10E6D0004FF002123EF0D4FE012201A92868FFF794
:10E6E00025FC9DF80C40029E00222146402007F0A8
:10E6F00079FF019AB6FBF0F12046FFF7D1FF0446FF
:10E700002868FFF7FDF80D4B834209D12A6861683C
:10E710005368C3F3172363F31F216160D368E36079
:10E72000032201A92868FFF7F2FB18B1237963F0EF
:10E730007F032371204604B070BD00BFCC4105604B
:10E7400038B505460C4610200349FFF7D2F80122E0
:10E75000C460C0E9012538BD90410560136870B5FB
:10E760006BB94468A51C50F825509C4207D055F859
:10E770002360B14204D1023350F82330136070BDDE
:10E780000133F2E72DE9F04716460025DFF85490F3
:10E790000F4606F10808DFF850A010490446F4F7C8
:10E7A000A9F97368AB4205D820460D49BDE8F0478A
:10E7B000F4F7A0B91DB149462046F4F79BF957F884
:10E7C0002520514620460135F4F710FD012258F866
:10E7D000041B2046FFF7A8F8E3E700BFB95B05601C
:10E7E000673F0560DC400560084205604B680A46EB
:10E7F000023351F82310FFF7C5BF0E2914BF0321C0
:10E8000001213EF005BE052805D00E2914BF0321C5
:10E8100001213EF0C9BD0020704738B50C461146B5
:10E8200002221D4620463EF02BFE1CB12868FFF751
:10E830008DFA08B90E2038BD1E20FCE7032A05D149
:10E840000E2914BF04490549F4F754B90E2914BF21
:10E8500003490449F8E700BF042405600924056062
:10E86000232505601D250560136813B940683EF037
:10E87000E3BD70472DE9F84F984602EB430300AF24
:10E8800082465D1C042B8B4616464FEA85051FD831
:10E89000EB1D4FF0000923F00703ADEB030D6C46B1
:10E8A00020462A1FB96A40F804BB1AF065FB2346CC
:10E8B0004246711C50463EF03FFE0446B9F1000F3F
:10E8C00002D04846F3F710FE2046BD46BDE8F88F5B
:10E8D0002846F3F7ECFD04460028D9D08146DFE74F
:10E8E00007B5009313460A46D0E90101FFF7C2FFBE
:10E8F00003B05DF804FB000038B505460C460C205B
:10E900000249FEF7F6FFC0E9015438BD84420560B4
:10E91000406870474160704710B5044602490820BE
:10E92000FEF7E7FF446010BDC04205602DE9F047E7
:10E93000866804460F4688B006EB010A154607EBC9
:10E94000420998460AEB420004F10C014FEA89099A
:10E95000052815D8B60003A832461AF00DFB03AB04
:10E960004A46414698191AF007FB606803AB2A46ED
:10E9700051463EF0E1FD0446204608B0BDE8F08770
:10E9800080000191F3F788FDA26801990646920084
:10E990001AF0F2FAA0684A46414606EB80001AF0E7
:10E9A000EBFAA16833462A46394460683EF0C4FD5C
:10E9B00004463046F3F798FDDEE700002DE9F0410C
:10E9C000CD1C174680460E46AD0008492846FEF786
:10E9D00090FF0446A5F10C023946C0E901860C30CF
:10E9E0001AF0CAFA2046BDE8F08100BFFC4205607B
:10E9F00091ED020B30B5B5EE400B8BB00023044611
:10EA00000D466722F1EE10FA00934FF020014FF00F
:10EA1000100302A80AD195ED040BFDF7B1FD02AA7F
:10EA200014492046F4F7E2FB0BB030BDFDF7A8FD1A
:10EA300002AA11492046F4F7D9FB95ED047BB5EE07
:10EA4000C07BF1EE10FA04DAB4EE477BF1EE10FA77
:10EA500003D70A492046F4F74DF800236722202106
:10EA600002A80093102395ED040BFDF789FD02AA7F
:10EA70000349D6E7384305603C430560E94006603A
:10EA800040430560136810B5144643B940F2834310
:10EA9000994205D190ED020B01F0F2F8206010BD13
:10EAA00040F2EA339942FAD190ED040BF4E700000A
:10EAB00008B52DED048BB0EE409B0649B0EE418BBE
:10EAC0001820FEF716FF80ED029B80ED048BBDEC55
:10EAD000048B08BD9C43056008B5072805D8DFE80E
:10EAE00000F005290404070418350021084608BD74
:10EAF00091ED027BB5EE407BF1EE10FA34D191ED51
:10EB0000047BB5EE407BF1EE10FA14BF1E210E21FE
:10EB1000ECE791ED047B91ED026BBDEEC77BFDEE62
:10EB2000C67B17EE103A17EE901A4B40590041F091
:10EB30000101DBE791ED041B91ED020BBDE80840FC
:10EB4000B1EE411BB1EE400BFFF7B2BF91ED040BEC
:10EB500091ED027B20EE000B07EE070B14F0A8FFEF
:10EB6000BDE8084001F08CB81E21BFE7000000009E
:10EB700030B50C46114604221D4620462DED048B6F
:10EB800085B03EF07DFCF4B1012C2A6822D09107BB
:10EB900043D111682A4B99423FD192ED028B92EDFD
:10EBA000049B6868830740D10268254B9A423CD198
:10EBB00090ED047B90ED021B38EE478B39EE011B84
:10EBC000B0EE480B03E09FED1C1BB0EE410BFFF7CE
:10EBD0006FFF15E002F007031046022B05D09407E3
:10EBE00015D1136817498B420ED103A9104604F0C2
:10EBF000D9FD00230399009301231A46FDF7BCFFBA
:10EC000005B0BDEC048B30BD0D498B42F8D01046E9
:10EC1000FEF78AFF9FED081BD9E71046FEF784FF39
:10EC2000B0EE408B9FED049BBBE7FEF77DFF30EE1F
:10EC3000091BC5E7AFF300800000000000000000E2
:10EC40009C430560EC62056030B5D0E90245C1E93E
:10EC50000045D0E90401C2E9000130BD0000000018
:10EC600010B52DED068B84B004460846B0EE40ABDF
:10EC700002AA6946B0EE418BFEF76CFF002800F057
:10EC8000CD80A01E202800F2CD80DFE800F0B7CBB9
:10EC9000CBCBCBCBCBCBCBCBCBCB11205BCB292CDA
:10ECA000CB6ACBCBCBCBCB11205BCB292CCB6A0057
:10ECB0009DED009B9DED027B3AEE099B38EE078BA4
:10ECC000B0EE481BB0EE490BFFF7F2FEA6E09DED5B
:10ECD000009B9DED027B3AEE499B38EE478BEFE7B8
:10ECE00055483EF049FC9DED027B9DED006BB5EE75
:10ECF000407BF1EE10FAB5EE406B0BD1F1EE10FA5D
:10ED000003D14E494E483EF047FC8AEE069B88EE02
:10ED1000068BD5E7F1EE10FA06D1B1EE4AAB88EEDC
:10ED2000079B8AEE078BCBE727EE075BB1EE477BAD
:10ED300006EE065B86EE054B87EE056B8DED004B10
:10ED40008DED026B9DED027B9DED006B27EE089B28
:10ED500016EE0A9B27EE0AAB06EE08ABB0EE4A8B26
:10ED6000AEE728EE080B0AEE0A0B14F0A1FEB5EE92
:10ED7000400BF1EE10FA1AD19DED027BB5EE407B0F
:10ED8000F1EE10FA11D19DED007BB5EEC07BF1EEF6
:10ED900010FA0ADBB5EE407BB7EE009BF1EE10FAFD
:10EDA0009FED230B09FE009B8AE72649AAE713F093
:10EDB000B7FDB0EE4A1BB0EE409BB0EE480B12F030
:10EDC000FBFD9DED006B9DED027B26EE008B27EE9B
:10EDD000000B07EE098B16EE090B13F075FAB0EE77
:10EDE00040ABB0EE480B12F0D3FE20EE0A9BB0EE23
:10EDF000480B14F00DFB20EE0A8B61E79DED007BC4
:10EE0000B4EE4A7BF1EE10FA0ED19DED027BB4EE2A
:10EE1000487BF1EE10FA14BF0E201E2004B0BDECAA
:10EE2000068B10BD0020F9E70E20F7E7AFF3008056
:10EE30000000000000000000454305606C430560D1
:10EE4000684D0560834305600B46114693ED041B36
:10EE500093ED020BFFF704BFF8B50F461E461146AF
:10EE60000446134A38463EF00BFB3268114B9A4277
:10EE700002D000203EF080FA7068FEF7D9FD051E32
:10EE8000F7DB21461820FEF734FD00230446681CFA
:10EE9000C4E9023360608000F3F717FB022F2061A2
:10EEA00003D9B068FEF7C4FD60612046F8BD00BF1D
:10EEB0000600040068650560042803D0052808D012
:10EEC00000207047D1E90203984214BF1E200E2093
:10EED0007047D1E90230C01A44BF4B68C0184000E7
:10EEE00040F0010070470000D0E9023102468B4239
:10EEF00010B503D1084909483EF04EFB01690024D2
:10EF000051F8230041F82340013351688B4208BF78
:10EF10002346936010BD00BF8944056030490560F9
:10EF200070B5C56842686B1C466984689A4208BF20
:10EF30000023F60705D5A34203D1084908483EF04F
:10EF40002BFB0669A34246F82510C36004D10133A8
:10EF50009A4208BF00238360062070BD7475056067
:10EF600030490560044B0B60037A0B714368084617
:10EF70008B600023CB60704740460560044B88607F
:10EF800008460B6001230B710023CB60704700BF64
:10EF90004046056008B503799B0702D500203EF086
:10EFA000EBFA08BD10B5044904460C20FEF7A1FC9D
:10EFB00002224460027210BD0446056010B504468A
:10EFC000FFF7E8FF201D3EF063FA062010BD04287D
:10EFD00003D0052808D0002070474B6833F00703A2
:10EFE00014BF1E200E2070474868C0F3DC004000AC
:10EFF00040F0010070470000F8B506460D460F6866
:10F00000144612B13846FFF7C5FF22466968381D1D
:10F010003EF052FA034608B1406870B9022E05D19D
:10F02000022C08D1696807483EF002FAA868012C52
:10F0300000D15860F8BD0620F9E7022C04BF002279
:10F040005A60F7E76C4905600122FFF7D5BF02223D
:10F05000FFF7D2BF0022FFF7CFBF30B50B6885683E
:10F06000AB4201D300220AE0C46804EBC30254F8A7
:10F0700033400133002CF3D0042CF1D00B60104648
:10F0800030BD00002DE9F3470C68164607460D46D3
:10F090002046FFF77FFF3168314A3846C9083EF005
:10F0A000EFF9022F14D1686810F003031BD1026836
:10F0B000D1682C4A914216D12A68904208D004F1B6
:10F0C0000408019301A96868FFF7C7FF074610B954
:10F0D000002504343CE00122396840463EF0ECF95A
:10F0E0007B684360EEE7002104F1040A3EF0BCF9BE
:10F0F000814648463EF064FA0028E9D000213EF0FF
:10F10000B3F980463EF05CFA074640463EF058FAB6
:10F11000054640463EF054FA0FB105B110B1124811
:10F120003EF02AF90122394650463EF0C5F94560C5
:10F13000DFE7B36853F8351003EBC50739B104298D
:10F1400005D0012220463EF0B7F97B6843600135C7
:10F150007368AB42EDD8062002B0BDE8F08700BF6F
:10F1600005000200E5F400604444056013B5044660
:10F1700000F10C018068FFF770FF60B12379012B6B
:10F180000BD0022B0BD00368694600934368022022
:10F19000019305F0F3FD02B010BD0068FBE7406885
:10F1A000F9E70000F0B5174B04460A7A85B00D4622
:10F1B000012653F82210F3F79DFC13492046134F04
:10F1C000F3F798FC124B00932B7A8DF804306B68A0
:10F1D0000293002303936846FFF7C8FF054628B94A
:10F1E0000C492046F3F786FC05B0F0BD1EB9394640
:10F1F0002046F3F77FFC0122294620460026FEF731
:10F2000093FBE8E7BC4505606A440560DC400560A7
:10F21000404605606D4405601FB50446FFF7BAFE21
:10F22000636833F0070203D1114912483EF0B4F984
:10F230000022204601922279510701A942BFC3F35F
:10F24000DC0303F1FF330193FFF707FF6368042238
:10F2500002A9083B63600368029343680393002399
:10F26000C0E90023022005F089FD04B010BD00BFF5
:10F27000704405606C4905600228F7B50E461446D7
:10F280000BD0242857D100222146301D3EF014F91E
:10F29000002840D10E2003B0F0BD02F003038A071E
:10F2A00025D10A6826498A4221D1002BF2D1216852
:10F2B00091421ED1CDE9003369463046FFF7CDFEBD
:10F2C000074601A92046FFF7C8FE0546002F34D0A7
:10F2D0000028DFD029683868FEF7D4FD0028D9D08F
:10F2E00069687868FEF7CEFD0028E5D1D2E7002BEB
:10F2F000D0D12268134B9A42CCD1736862685340D4
:10F3000033F00703C6D10434019301A93046FFF757
:10F31000A4FE054608B91E20BDE700222968204644
:10F320003EF0CAF80028B5D041686868FEF7AAFD2B
:10F330000028EAD1AEE70020ADE70028AAD1EAE72D
:10F340007C460560C845056010B40C7A012C06D1D6
:10F35000242804D149685DF8044BFFF78DBF0020D5
:10F360005DF8044B704700002DE9F04F032A154665
:10F370000B6885B0344A1CBF0125DFF8E4900446D1
:10F3800018BFDFF8E0800F46934608BFD0E9028936
:10F39000934205D0032D03D0DA882C49F3F726FFDA
:10F3A0002B492046F3F7A6FB0023DFF8BCA003930C
:10F3B000012303A938460193FFF74FFE019B064640
:10F3C00078B924492046F3F795FB3B685B4505D0A7
:10F3D000032D03D020492046F3F78CFB05B0BDE890
:10F3E000F08F1BB941462046F3F784FB032D28D14B
:10F3F000326802F00703022B23D012F0030304D17A
:10F400001268164992698A4204D051462046F3F7A1
:10F4100071FB01232A46316820460193FEF784FAE6
:10F42000019B1BB151462046F3F764FB4946204639
:10F43000F3F760FB2A4671682046FEF775FA002351
:10F44000B7E70023E6E700BFC84505608F440560C5
:10F450009344056091350560673F0560E1370160C1
:10F46000E09D0560DC4005609544056010B50449E9
:10F4700004460C20FEF73DFA00224460027210BDE3
:10F480000446056010B5044904460C20FEF731FA25
:10F4900001224460027210BD0446056010B50022CE
:10F4A00004300C463EF008F818B9214602483DF0F9
:10F4B000BFFF406810BD00BF6C490560024B40F8BB
:10F4C000043B3EF005B800BFC845056013B5019088
:10F4D0001020F2F7E1FF04460199FFF7EFFF204605
:10F4E00002B010BD2DE9F041804686B000200D46E7
:10F4F00016461F46FFF7EAFF0F4B0446C0F8008090
:10F50000984502BF037943F00403037155EA0603EB
:10F510000DD03B6807EB85023146019003A80293AA
:10F520003EF046F803AA01A9681CFFF7ABFD204690
:10F5300006B0BDE8F08100BF7C46056038B50446E2
:10F540008068FFF7C3FF054623686268036023797C
:10F5500022F0070203F0050313434360A268E16849
:10F56000D200C06819F008FD284638BDF8B50C4631
:10F570000646002160683DF077FF022E0546606870
:10F580008CBFA6680626FEF7BFFB50B9FFF79EFFAB
:10F590000446071D28463EF013F8014618B92046D8
:10F5A000F8BD4010F2E7012238463DF085FF466085
:10F5B000F0E74068C008704737B50446154601912A
:10F5C000FFF7E8FC01220199201D3DF075FF456021
:10F5D000204603B030BD022213B50446CDE9000138
:10F5E00069461046FFF708FD204602B010BD000036
:10F5F00038B50C461AB9FFF7EEFF06200BE0042AD7
:10F600000AD1002204303DF057FF18B921460448C2
:10F610003DF00EFF406838BDFFF7CEFFEDE700BFBD
:10F620006C49056013B5044640683DF0C9FF58B108
:10F63000A36869465A1C5B0043F00103A260CDE950
:10F640000030022005F09AFB02B010BD1FB5044641
:10F65000084611461A4602AB01930A4B0093022357
:10F660003DF05AFF21460C20FEF743F904460021E5
:10F6700002983DF0F9FE039B60602046A36004B051
:10F6800010BD00BFB8460560F8B5164602F07F070A
:10F6900004460D4632061AD47B1E012B17D80B6880
:10F6A000D888F3F762F801462046F3F723FA022FD1
:10F6B00011D122492046F3F71DFAEB680BB15A68C5
:10F6C00082B920461E49BDE8F840F3F713BA022F6D
:10F6D000EFD0002FF1D03246E9682046BDE8F8406F
:10F6E00005F0D2BA2868174988421FD1022A1DD8CE
:10F6F0009868C3071AD509F037F80346B0B1EA682D
:10F700002046114992685210F3F770FDEB685B6870
:10F71000012B12D909492046F3F7ECF9EB680022D6
:10F72000D9682046BDE8F840FEF7FEB8EB685A6895
:10F73000012AD0D100229968F3E7F8BDE09D056069
:10F74000CC3B0660D44A0560044705602DE9F843C8
:10F750000E4604461146DFF87480194A3046994631
:10F760003DF08EFE1020F2F7A2FE0023002814BF09
:10F77000054645462C60AB60E6B1B71CBF00384675
:10F78000F2F795FE044650B9D8F8242307F1180380
:10F79000A8F128089A420DDBD8F838401834094BF4
:10F7A000A7F10802494604F10800C4E9003619F03F
:10F7B000E3FB00E0044C2846EC60BDE8F88300BFA2
:10F7C000FEFF01007065056068650560D8270020B0
:10F7D00010B50446FEF794F8034BC2689A4218BF6E
:10F7E0002469204610BD00BF4DF70060F8B51546EE
:10F7F0000F460446D0E90123591991420FD30178ED
:10F80000D9B105F11006C068164401223146F2F75D
:10F8100069FE78B96568A268013D2070AD1A2A4674
:10F820003946D4E90230184419F0A6FBA2682A44EC
:10F83000A260F8BD6660E060F1E7013AD51AEEE734
:10F84000024B0022C3F84C239A637047B027002074
:10F8500010B5FEF7EDF8041E11DDF2F71DFE094BA1
:10F860009A6BEFF3108172B6C3F84C43986381F33F
:10F87000108812B11046F2F737FE062010BD0020A6
:10F88000EDE700BFB027002008B5FFF7A1FFC36870
:10F890005A680AB1986808BD0620FCE7136810B5DD
:10F8A000144643B1E02905D15368062B02D1002349
:10F8B000C380236010BD3D2901D1C368F9E7A229A7
:10F8C00003D040F2B6339942F4D1FFF7DDFF206058
:10F8D000F0E700231A461946FFF738BF73B506460E
:10F8E00010200D46F2F7E3FD044630B90F4BD3F874
:10F8F0004C23332A12DD9C6B24340D4B28462360A5
:10F9000019F0AEFB0146C4E902052846F2F724FED1
:10F9100001AB002201216060019402E0034602462F
:10F9200001463046FFF712FF02B070BDB02700203D
:10F93000EC6205602DE9F0410E4688B007461020C4
:10F940000192F2F7B4FD0446304619F089FB00F14C
:10F95000010805464046F2F7AAFD019A03460CB19C
:10F9600000283DD11F48D0F84C1343291FDD836B7D
:10F97000A1F13408012503F12404343385F0010595
:10F98000314602A8CDF814808DF810500025CDE93D
:10F99000065304AB0293144B0393F3F7D7FADDE954
:10F9A0000632D554069BA360079BE3600CE044B984
:10F9B0002346224621463846FFF7C8FE08B0BDE878
:10F9C000F0816BB9C4E90256084BD4E902102360F8
:10F9D000F2F7C2FD04AB6060002201210494EAE763
:10F9E0000025CBE7B0270020EDF70060EC62056052
:10F9F0000EB403B503AA52F8041B0192FFF79AFF55
:10FA000002B05DF804EB03B070470000830707D134
:10FA10000268064B9A4203D1C268054B9A4202D053
:10FA2000044906F037B90120704700BF5C680560E3
:10FA30004DF70060C847056008B5FDF761FFBDE8F8
:10FA40000840FFF7E3BF38B504460D46FFF7F4FF63
:10FA500018B12046FDF754FF044629462046BDE86C
:10FA6000384006F017B900002DE9F04188461746E6
:10FA70001E46FFF7ADFE04468068E8B90C20F2F799
:10FA800016FDA060B0B9174BD3F84C23172A0FDD31
:10FA90009B6BA3600623A3800023E380E388A16817
:10FAA000D81C01EB8302E08041F82380C2E9017693
:10FAB000BDE8F0810323EEE7E388A5880233AB427B
:10FAC000ECDB084B9B6B9842F2D003350122A90076
:10FAD000F2F708FD0028EBD0A388A0600333A380D1
:10FAE000DCE700BFB027002038B50D461446FFF70D
:10FAF0006FFE836813B92B60236038BDC2882A600B
:10FB0000FAE737B50446A0683DF05AFD019068B1A8
:10FB10006568062D05D001AB0022012128463DF085
:10FB20000BFDFEF713F90028EDD0019803B030BDAE
:10FB300038B504461D46084611464FF004123DF004
:10FB40009FFC21460C20FDF7D4FE2B6804460021C3
:10FB5000436068683DF088FCA060204638BD000026
:10FB600030B500238BB00D46044600936722102366
:10FB7000202102A895ED020BFCF702FD02A9204608
:10FB8000F2F7B8FF2E2102A819F0C0FA68B9652172
:10FB900002A819F0BBFA40B96E2102A819F0B6FA12
:10FBA00018B903492046F2F7A5FF0BB030BD00BFDE
:10FBB000778E05600000000038B505460C4691EDD3
:10FBC000001B90ED000B12F09BFDB5EE400B95ED88
:10FBD000005B94ED007BF1EE10FA35EE404B84EEC5
:10FBE000076B1DD117EE903A002B9FED210B9FED77
:10FBF000224B20FE040BB5EE406BF1EE10FA26D13D
:10FC000085EE077B9FED1C6B53EC172B9FED187B4C
:10FC1000002B27FE067B85ED007B84ED000B38BDB5
:10FC2000B5EEC00BF1EE10FAB5EEC07B4CBF012271
:10FC30000022F1EE10FA4CBF012300239A42DAD0E1
:10FC4000B7EE004B30EE070B36EE446BD3E7B6EE63
:10FC5000005BBBFE467B36EE476BB4EEC56BF1EE48
:10FC600010FAD8DDB7EE006B37EE067BD3E700BFA6
:10FC70000000000000000000000000000000008004
:10FC800008B52DED028BB0EE408B1020F2F704FC8E
:10FC9000034A80ED028BBDEC028B026008BD00BF01
:10FCA000004E05600000000030B50D4687B01146DB
:10FCB000022228461C463DF0E3FB25B99FED0E0BC2
:10FCC000FFF7DEFF0CE0012203A92068FEF71FF911
:10FCD00040B10023DDE903011A460093FCF74CFF15
:10FCE00007B030BD2068830703D10268044B9A42F5
:10FCF000F6D0FDF719FFE3E7000000000000000068
:10FD0000004E056091ED020B072805D8DFE800F0F2
:10FD1000051B040407040F17002108467047B5EEC1
:10FD2000400BF1EE10FA14BF1E210E21F5E7BDEED7
:10FD3000C00B10EE103A590041F00101EDE710EE52
:10FD4000903A002BE9DAB1EE400BFFF799BF90ED46
:10FD5000020B70470000000030B50C4687B0054626
:10FD600002A920468DED000BFDF7AEFE002800F045
:10FD7000C280232D00F21B81DFE815F0DD00E900D1
:10FD8000F50001010D0119011901190119011901EC
:10FD90001901190119011901240031003800190154
:10FDA0003F004F005D008F00190119011901190171
:10FDB000190124003100380019013F004F005D0097
:10FDC0008F00C2009DED007B9DED026B37EE067B40
:10FDD0008DED007B9DED000BFFF752FF8BE09DED5D
:10FDE000007B9DED026B37EE467BF1E79DED007BDE
:10FDF0009DED026B27EE067BEAE79DED027BB5EEFB
:10FE0000407BF1EE10FA03D1714972483DF0C4FB1A
:10FE100002A96846FFF7D0FEDCE79DED027BB5EE58
:10FE2000407BF1EE10FAEFD09DED005B85EE076BA5
:10FE30008DED006BCEE79DED021BB5EE401BF1EEA4
:10FE400010FAE1D09DED000B12F05AFCB5EE400B1C
:10FE50008DED000BF1EE10FA08D1039B9FED567B60
:10FE60009FED576B002B27FE067BB1E7B5EEC00B6D
:10FE70009DED027BF1EE10FAB5EEC07B4CBF012286
:10FE80000022F1EE10FA4CBF012300239A42A1D0C8
:10FE900030EE070B8DED000B9CE79DED000B9DED0B
:10FEA000021BB5EE400BF1EE10FA0DD1B5EEC01B02
:10FEB000F1EE10FA08D5B0EEC17B9FED436BB4EEC6
:10FEC000467BF1EE10FA9FDDB5EEC00BF1EE10FAB5
:10FED00013D5BBFE417BB4EE417BF1EE10FA0CD0A2
:10FEE000B4EE411BF1EE10FA07D6214622209FED19
:10FEF000321BFEF7B5FE07B030BD12F019FFC9E79F
:10FF00009DED027BB5EE407BF1EE10FA3FF47CAF45
:10FF100002A96846FFF750FE9DED000BFFF7B0FE0B
:10FF200004909DED020BFFF7ABFE04A905900220A3
:10FF300004F024FFDFE79DED006B9DED027BB4EE46
:10FF4000C76BF1EE10FA4CBF1E200E20D3E79DEDDB
:10FF5000006B9DED027BB4EEC76BF1EE10FACCBFE7
:10FF60001E200E20C7E79DED006B9DED027BB4EED9
:10FF7000476BF1EE10FA14BF0E201E20BBE79DED7B
:10FF8000006B9DED027BB4EEC76BF1EE10FA94BFEF
:10FF90001E200E20AFE79DED006B9DED027BB4EEC1
:10FFA000C76BF1EE10FAACBF1E200E20A3E70020B5
:10FFB000A1E700BFAFF300800000000000000000D8
:10FFC0000000000000000080FFFFFFFFFFFFEF7F49
:10FFD00074430560684D056091ED020B910703467F
:10FFE00010B40AD114680A498C4206D19FED061B51
:10FFF00011465DF8044BFEF733BE114618465DF816
:02000004600199
:10000000044BFFF7A9BE00BF000000000000000085
:100010009C43056010B504460846114600223DF099
:100020002FFA6368BDE81040184770B51C460546B6
:10003000084611464FF002123DF022FA6B68206824
:10004000BDE87040184770B51C4605460846114685
:100050004FF004123DF014FA6B68D4E90001BDE8DA
:100060007040184770B51C460546084611464FF0CB
:1000700006123DF005FA6B682068D4E90112BDE86C
:100080007040184730B5044685B0CDE90221019390
:10009000FDF71EFCE068039940F001052046DDE90C
:1000A0000132AC4605B0BDE8304060472DE9F04F65
:1000B00083B006468846914600AF9A46FDF708FC95
:1000C000F268002112F8013BC3F3C30BC3F38004B1
:1000D0001B0638D40BF1010B04EB44045C44A40070
:1000E0002C2C04F114033CD80733002423F007031D
:1000F000ADEB030D6D464146DFF8888053464A4616
:1001000028462E60A5F80CB008F01EFDD8F8103077
:10011000002128462B6173685B68C8F810303DF0F9
:10012000FFF92B690646C8F8103018BBAB68D3F846
:1001300000801CB12846F2F7D7F9FEB940460C37CB
:10014000BD46BDE8F08F12F8013B4D0003F03000D2
:10015000A8404BEA000B03F0020088400131044341
:10016000B6E718467B60F2F7A2F97B6805460028DF
:10017000C1D1B9E7D5F81480002CDBD14046F2F7A5
:1001800067F900BFB027002070B50C4686B0114655
:100190000546426820461E4601913DF071F96B68A4
:1001A000019913F0010F0BD006EB840203A83DF078
:1001B000FFF9AB6803AA31462046984706B070BDE8
:1001C000AB68314620469847F8E700001FB510F0AD
:1001D0000103044602D0401004B010BD06283FD0F1
:1001E0000E283DD01E283DD010F0030306D1016833
:1001F0001D4A914202D100F00DFEEDE704F0070226
:10020000022A04D043B92268184B9A4204D101A9AA
:10021000204603F0C7FADFE72046FDF771FB144BD9
:10022000984207D12046FFF792FDFDEEC07B17EE06
:10023000900AD1E70F4B984202D00F4B984206D15B
:1002400001AA69462046FDF7DDFC0198C4E70122BA
:1002500001A92046FDF75BFE0028F6D12046BBE74A
:100260001846B9E70120B7E79C520560EC620560CB
:10027000004E05607065056034540560F7B51C4696
:1002800043680F4611465A000546384642EA434243
:100290003DF0F6F8AE6846F0010637B9B047E968B8
:1002A00003B0BDE8F040FDF7A5B9012F206803D1E8
:1002B000FFF78CFFB047F2E7022F09D1FFF786FF67
:1002C00007466068FFF782FF01463846B047E6E719
:1002D000032F0ED1FFF77AFF07466068FFF776FF1E
:1002E0000090A068FFF772FF009902463846B047B9
:1002F000D5E7FFF76BFF07466068FFF767FF0190E0
:10030000A068FFF763FF0090E068FFF75FFF034618
:100310003846DDE90021B047C1E7000003680F4A15
:10032000934210B5044616D00D4A934213D0C368C9
:1003300013F8012B51B2184613F8012B0029F9DBF1
:1003400010F9013B002BFBDB08F049FA63689B685E
:1003500033F8100010BD0120FCE700BFF84F056026
:10036000A051056010B51446126803463AB9172922
:1003700006D1FFF7D3FFC00040F00200206010BD9F
:10038000BB2902BF43685B682360F8E713B50446E6
:1003900008460191FFF7C2FF019B02460349204630
:1003A00002B0BDE81040F2F721BF00BF3C4E05602F
:1003B0002DE9F047884691469A460446F8B1076809
:1003C00007B37E6864680CB9304600E0701C0430E6
:1003D0000D498000FDF78DFA0546C0F80C80C0E994
:1003E000019A2FB1B20007F10801103018F0C4FDD6
:1003F00014B1043645F826402846BDE8F087074684
:100400000646E4E73E46DDE7904E056008B5FFF797
:10041000CFFF014B036008BDF84F056070B506467D
:100420000D46144603491020FDF763FAC460C0E985
:10043000016570BD544E05602DE9F3410646C06864
:100440000F464FF0000C10F8011BC1F3C305C1F3B8
:100450008004090619D4013504EB440414492C44E2
:100460000734A000CDE90023FDF743FA0621044636
:100470008582C0E90116DDE900233946083008F01D
:1004800063FB204602B0BDE8F08110F8011B4FEA83
:100490004C0801F0300E0EFA08FE45EA0E0501F098
:1004A000020E0EFA0CFE0CF1010C44EA0E04D0E729
:1004B000285105602DE9F3418846C16805468768E3
:1004C000096809B157F821703C46002114F8010B66
:1004D000C0F3C306000624D406F10800164901360D
:1004E0008000CDE90023FDF704FA06210446C76029
:1004F0008682C0E9011500F118010830DDE900230A
:100500008160414608F02AFB4FF6FF732046E382E4
:10051000EB685A68134443F00103E36002B0BDE89E
:10052000F08114F8010B00F0300C0CFA01FC0231E0
:1005300046EA0C06CEE700BF2851056008B54368BF
:1005400013B903483CF018FF4160184608BD00BFCE
:100550003450056070B50C4605468868FFF7DEFE2E
:100560002346024602492846BDE87040F2F73EBEE7
:10057000505005602DE9F04104460D4617461E46D1
:10058000FDF7A6F9E06828B906230546336028463A
:10059000BDE8F081636813B929483CF0EDFE062BF5
:1005A00018BF1F4604F118022369B4F816C093421D
:1005B00004D1062D03D023483CF0DEFF1D6000234C
:1005C00020466360204B1A699846A26150F8082FB4
:1005D0005168496819614FF6FF718C4516D1D3688F
:1005E0003946083343F001039847C5B2A369012D8A
:1005F000C8F810304FF0060363600CD00023022DC2
:10060000E3600ED023691B683360C0E739463CF0D5
:1006100087FF0546EAE722691268326022691360A3
:10062000B5E7E0693060FDF76BF9084905F032FB8A
:100630000028ACD006490748FFF750F93060A6E71C
:10064000345005606E500560B0270020C44B056033
:10065000BF3905604C4B056013B51C4601ABFFF775
:1006600089FF01280FD002280FD0019B062B04BF61
:100670000023019301980CB13CF096FF044BD86124
:10068000204602B010BD0198FBE70198F1F7E0FEAB
:10069000B027002002284A6810B40C4603D98B68A2
:1006A000062B18BF1A462068012306215DF8044B6B
:1006B000FFF7D2BF01230022FFF7CEBF00230621A0
:1006C0001A46FFF7C9BF000007B50E4A01AB062165
:1006D000FFF750FF012805D0022807D0062003B0FD
:1006E0005DF804FB084909483CF056FF0198FDF706
:1006F00007F9074905F0CEFA0028EFD10198F1F784
:10070000A7FE00BF18510560A45005604C4B056062
:100710007C48056030B593B005466846F1F780FE29
:10072000014680B92A1D01203CF0CAFEEB68044650
:1007300023F00103023343F00103EB60F1F768FE9D
:10074000204613B030BD0198054A0368934204D097
:10075000044A934201D0F1F77BFE0024F0E700BF8A
:10076000C44B056030490560044B0B6003684B6067
:10077000436808468B600123CB607047DC510560FD
:100780002DE9F041486886B00C46FDF751F9021E8C
:1007900002DA00203CF0F0FDD4F8088040F26A371D
:1007A000114602A8B8EB0706019218BF0126F2F71E
:1007B000ADF8049D0021019A284618F01DFC206820
:1007C000019A10F0010F0AD12B46314600F019FAB8
:1007D00002A90A4802F08EFA06B0BDE8F081042AA8
:1007E0004FEA60031046314628BF0420B84514BFC5
:1007F000121A00222A4406F0A9F8E9E760600560B1
:10080000F0B50C4685B00122606801A9FDF78EFBAA
:1008100040F26A33A568002002999D42019A0C4675
:1008200007BF01F1FF334FF0FF361346012608BF23
:100830009B1814B900F0CCFA0BE0B0F5800F04F16E
:10084000FF3408D340F26A30281A18BF012000F0A4
:10085000C8F905B0F0BD1F78334447EA0020E8E747
:1008600010B52DED028BB0EE408B47F6F07110EE17
:10087000102A18EE903A31EA13410DD110EE100A09
:10088000C3F3130150EA010303D1174917483CF0A1
:1008900083FE17483CF070FD002B19DA002A18BFC0
:1008A00043F0010333F0004215D003F1FF4303F599
:1008B000E003104A93420ED900F05CF9B0EE480B09
:1008C00004460430F2F7CCFE2046BDEC028B10BD8E
:1008D0001B0D1B05EDE7FDEEC87B17EE900A4000EF
:1008E00040F00104F0E700BF18520560104B0560AE
:1008F000315205600000C04130B50D4685B011464B
:10090000042228461C463CF0BBFD002D3BD0012DA7
:100910002AD12068C30720D410F0030303D1016853
:100920001A4A914219D000F00702022A05D0B3B941
:100930000368174A9969914208D103A902F032FF6E
:10094000002303991A46FCF799F806E0114A9342EE
:1009500005D1FFF7FCF9FFF783FF05B030BD014675
:1009600008203CF021FDF8E703A9206802F01AFFF7
:100970000399054660680191FDF75AF80023024685
:1009800001992846DFE70120E7E700BF9C52056098
:10099000E1370160004E056038B50A4C214411F87A
:1009A000015CB0FBF5F55BB16C1C0320B4FBF0F40B
:1009B00010460AB118F054FB03352C44204438BDCE
:1009C0001C46F5E78C52056013F0010F2DE9F74F37
:1009D00007468B469DF838409DF83CA00092DDE923
:1009E0000C863FD05D1044D44FF000095346414679
:1009F00032462020FFF7D0FFDBF80030014683426B
:100A000006D20190F1F748FD01993860CBF800104B
:100A1000D7F800B000230BEB010202F8013C65B3EC
:100A2000013AA4F10A0E1046AC46441EB5FBF8F597
:100A300008FB15C3092B8CBF7344303300F8013C0D
:100A4000BAF1000F30D0C4451BD3A34519D2131BF4
:100A5000032B05D1841E00F802ACA34511D2224617
:100A60002046E1E7CDE90E4A03B0BDE8F04F00F0C3
:100A70008FB86D424FF02D09B8E73023941E02F86D
:100A8000023CCEB13046019118F0EAFA201A0199E1
:100A9000834511D2013E024616F8013F4BB9044688
:100AA000B9F1000F0DD10FE0A345EAD2C445D7D26A
:100AB000E7E702F8013BEFE7B9F1000F04D05C452E
:100AC00002D904F8019C013C3868009B014420468F
:100AD000091B0139196003B0BDE8F08F30B5102251
:100AE0008DB004460B460692002208AD06A901927D
:100AF00005A80595CDE902220A22009207AAFFF770
:100B000063FF01462046F1F7F5FF0598A84201D0A2
:100B1000F1F7EAFC0DB030BD0E2A134630B40C4696
:100B200003D1012230BC3CF073BC1E2A01D1032248
:100B3000F8E71D2814D102F00702022A0CD09A0708
:100B40000ED11A6808499069884205D007498A423F
:100B500002D007498A4203D1224619461D20E1E707
:100B6000002030BC704700BFE13701607065056050
:100B70003454056010B505491020FCF7BAFE044650
:100B80000430F2F7FEFC204610BD00BF9C52056009
:100B90002DE9F74F05469DF83CB098680E46904603
:100BA0001C4600015B46DDE90C9A52464946FFF7B8
:100BB000F3FE33680746834203D2F1F76DFC2860E9
:100BC00037602D6852469DF838304946201DCDE9E2
:100BD00000B5F3F749FCC8F80000284603B0BDE8AB
:100BE000F08F73B50E4605460192FFF7C3FF04462A
:100BF000019B324629460430F2F700FE204602B03F
:100C000070BD0430F3F7B9BBC30706D54010002808
:100C10000DDB14BF012000207047836853B10379B6
:100C200013F0010F14BF4FF0FF30012070474FF059
:100C3000FF3070471846704738B50C46072805D86E
:100C4000DFE800F005141D0407040D2500242046EC
:100C500038BD8B68002B14BF1E240E24F7E7081D37
:100C6000F3F75FFB400040F00104F0E7FFF782FF7D
:100C7000211D05460430F2F71FFE2C46E7E7FFF77B
:100C800079FF211D05460430F2F727FEF5E70B79C1
:100C9000DB07DCD5FFF76EFF211D05460430F2F7B8
:100CA00000FEEAE71FB502910390FFF763FF012101
:100CB000044604300091DDE90232F2F7A2FC20463E
:100CC00004B010BD90EA40024FEA400302D443F062
:100CD00001007047C117FFF7E5BF1FB502910390F0
:100CE000FFF748FF0021044604300091DDE902329D
:100CF000F2F787FC204604B010BD00002DE9F04F4C
:100D000010F001098BB006460D46144605D1810747
:100D100015D102682C4B9A4211D115F0010805D16A
:100D2000AA070CD12A68284B9A4208D114F0010B6B
:100D300008D1A30703D12268234B9A4202D023484B
:100D40003CF01AFC00200021FFF7C7FF0DF1040A58
:100D50000746B9F1000F31D0711056465046F2F7F0
:100D60003CFC0DF11009B8F1000F29D069104D4677
:100D70004846F2F732FC0DF11C08BBF1000F21D000
:100D8000611044464046F2F728FC23462A46314685
:100D9000381DF3F76BFA564502D13046F2F7F6FBF1
:100DA0004D4502D12846F2F7F1FB444502D12046D9
:100DB000F2F7ECFB38460BB0BDE8F08F0436D0E715
:100DC0000435D8E70434E0E79C520560D85205604A
:100DD00010F0404F03D1400040F001007047002167
:100DE000FFF77BBF2DE9F34104460E4617469846B0
:100DF000FFF7C0FE324605463B4621680430CDF879
:100E00000080F2F7B0FC236818442060284602B046
:100E1000BDE8F081C30701D5401070470430F3F7F7
:100E200080BA0000C30707B503D5401003B05DF8D2
:100E300004FB01A90430F3F787FA08B10198F5E73C
:100E4000014902483CF0A8FB01530560104B0560C6
:100E50002DE9F0410646C8070C4617462DED028BDA
:100E60008AB025D504AD4B10022203A904A8F2F7DD
:100E7000BBFBF9071ED502227B1003A904A8F2F7D9
:100E8000B3FB04AA202E01D0132E3FD15368019248
:100E9000002B6AD02846F3F7C3FA019AB0EE408BD4
:100EA0001046F3F7BDFA88EE000BFEF7E9FE20E0EE
:100EB0000D1DDEE7BA0723D13B68734A934201D187
:100EC0003A1DDFE7714A934207D12846F3F7A8FAA3
:100ED00039463046FEF740FF0BE06D4A93420FD192
:100EE0002846F3F79DFA394630469FED651BFDF71E
:100EF000B7FE044620460AB0BDEC028BBDE8F08187
:100F00003A4621463046FFF707FEF2E7A6F1090808
:100F10005FFA88F31A2B00F28A800192FFF72AFE0B
:100F2000019A0446B8F1190F6CD8DFE808F043487D
:100F30003E4D4D0D12176B1C6B316243483E4D4DBB
:100F40000D12176B1C6B316229460430F2F7AEFDAF
:100F5000D0E729460430F2F7E9FDCBE72946043013
:100F6000F2F776FFC6E753681BB94A494A483CF096
:100F700013FB07A80192F2F704FB019A07A9201DB1
:100F800013462A46F3F723F807A8F2F7FFFAB1E76A
:100F900053680192002BE8D007A8F2F7F2FA019A01
:100FA000211D07A813462A46ECE729460430F2F72C
:100FB00001FE9FE729460430F2F772FE9AE72946C0
:100FC0000430F2F7DBFE95E73846FFF72BFF021EF1
:100FD00002DA32483CF0D0F9192E04F10400294617
:100FE00001D00C2E02D1F2F7B1FC83E7F2F708FD35
:100FF00080E71378DB073FF568AF29460430F2F746
:10100000A3FF77E753680192002BAED0FFF7B2FD44
:10101000019A0646211D134604302A46F2F7D7FFEF
:1010200007A90220CDE9076403F0A8FE61E7114695
:101030002846F2F719FC042E1DD8DFE806F0030855
:10104000170D12000028ACBF0E241E2452E7002802
:10105000D4BF0E241E244DE70028CCBF0E241E242E
:1010600048E70028B4BF0E241E2443E7002814BF1D
:101070000E241E243EE700243CE700BFAFF30080AF
:1010800000000000000000009C520560004E05605A
:101090009C43056074430560684D0560CE3A056069
:1010A0000430F3F7BDB9042803D0052807D0002089
:1010B00070478B68002B14BF1E200E207047886875
:1010C000400040F001007047044B0B60044BC1E945
:1010D000013000230846CB60704700BFE85605602A
:1010E000131101608368002203EBD3719B00491048
:1010F00070B59142A3F1040301DC062070BDC46801
:10110000E65854F8225044F822600132C468E55091
:10111000EFE7D0E9022391688B4237BFD268002203
:1011200052F82320013338BFC3601046704738B5EA
:101130000D460446D0E901138B4211D3C900C068A3
:10114000F1F7C5F96268A36800215200E0606260AF
:10115000D21A0133013A00EB8300920017F04CFFE2
:101160000620D4E90232591CA16042F8235038BD50
:101170008368491048BFC91870B521EAE174054673
:10118000062116469C4228BF1C46FFF7D0FFAB68DD
:10119000013BE9689C4203DB062041F8246070BDF6
:1011A00001EB830252F8042C41F82320F0E738B514
:1011B0000025044610218560C068F1F788F90423F2
:1011C00010222946E060636017F016FF062038BD44
:1011D0002DE9F84F81460F4690469A46FCF778FB7A
:1011E000B94501D3BDE8F88FA9F1040B3D68B8F10A
:1011F000000F04D0294640463CF0F2F805463E4632
:101200000BF10404A64209D92168B8F1000F18D1E6
:101210002A4600203CF0FCF8824510D0043EB4423F
:1012200024D2B8F1000F11D13268294600203CF0D9
:10123000EFF88245F2D02368326822603360A3461B
:10124000DEE740463CF0CCF80146E1E73168404635
:101250003CF0C6F80246E8E731463E465346424671
:101260004846FFF7B5FF3746D946B9E73A680BF16C
:10127000080B236822603C1B3B60A6EB0903A4100B
:10128000013CB4EBA30FE7DC5846534642463946CF
:10129000CB46FFF79DFFE6E71FB502AB0C460138D2
:1012A000043101930F4B009302233CF015F923689E
:1012B0009968012912D9029A01F18041D868062A59
:1012C0009DF80C3001F1FF3108BF0022002B00EB2C
:1012D000810114BF0E231E23FFF77AFF062004B0FE
:1012E00010BD00BF5853056010B40C6802460B4691
:1012F000D4E902105DF8044B04F0AEBE38B50C68BA
:101300000346A5681DB91A491A483CF045F9012B56
:1013100020684FF0000314BF4A684FF0FF3229469F
:10132000FCF7A8FCA268E368013A53F8205003EBED
:101330008001A260121A043103EB8000920017F0C2
:1013400043FE0021D4E9023242F8231061680429E7
:101350000BD9B1EB430F08D94908E0688900F1F7D0
:10136000B6F86368E0605B086360284638BD00BF7C
:10137000445305603049056007B5CDE90001694671
:101380000220FFF7B1FF694601900220FFF7B6FF88
:10139000062003B05DF804FB38B50446084600217A
:1013A0003CF062F8054628463CF00AF90146204622
:1013B00001B938BDFFF7BBFEF5E70A46D0E90210D8
:1013C00004F07EBE2DE9F041032A4FF000050F46E0
:1013D0001049164604460EBFD0F808800126DFF8F3
:1013E0003C80F1F787FBBB68AB4205D820460A4931
:1013F000BDE8F041F1F77EBB1DB141462046F1F753
:1014000079FBFB683246204653F825100135FCF77E
:101410008BFAE8E7DA40056004110660DC400560FD
:1014200070B511F0030604460D4629D10A68174B22
:101430009A4225D1AB68816819444368994210D912
:101440000431C0688900F1F742F8AA68A368314600
:10145000E06013441A1D00EB83006260102217F055
:10146000CBFDAA68E9689200D4E9020303EB80008F
:1014700017F082FDA368AA681344A360062070BD1C
:1014800029462046FFF788FFF8E700BF345405607F
:1014900038B504290B4B04460D460360084638BF97
:1014A0000420C4E901018000F0F7F6FF6268E06003
:1014B0000021521B00EB85009200BDE8384017F078
:1014C0009BBD00BF3454056013B501901020F0F7A8
:1014D000E3FF04460199FFF7DBFF204602B010BD91
:1014E0001B287FB503460E46154622D005D8042892
:1014F00044D90E283CD0002437E01D28FBD103A995
:101500001046FCF7C1FA0028F5D0039B002BBCBFA6
:1015100000230393B36803985843FFF7D5FFC368CC
:101520000446B26800930421039BF06804F0C3FCF6
:101530001BE012F00304DED112681B4B9A4214D157
:10154000AB6888681844FFF7BFFFB2680446F168CB
:101550009200C06817F010FDB068E368AA68E968F7
:1015600003EB8000920017F007FD204604B070BD29
:10157000114630463446FFF753FFF6E7AA0703D17A
:101580002968094A914203D0022BB4D10E24ECE71A
:10159000AB68D6E902210093EB6804F012FD002845
:1015A000F4D01E24E1E700BF3454056013B50846AB
:1015B000114602221C4601903BF062FF019820B9BF
:1015C00002B0BDE81040FFF77FBF0020FFF77CFFAF
:1015D000216802B0BDE81040FFF7DEBE38B50C460A
:1015E0000546FFF771FF4CB938BD54F82310C268A7
:1015F00042F823100133AB42F7D1F5E70023FAE7B5
:10160000D0E90201FFF7EABF83680B60C36813608B
:1016100070478160704738B50446154600230A4676
:1016200081680068FCF726FBE36843F8205038BD6A
:10163000F0B5044689B00D4601F0030610466ABBBA
:1016400026BB0A685B4B9A4220D102AAA06804F02C
:1016500045FC10B900203BF0CBFEDDE90257D4E990
:101660000220D21B00EB870100EB8500ED1B9200EE
:1016700017F0AAFCA0686FF00302E3683146284423
:101680006A4303EB800017F0B7FC73E005A9022062
:10169000CDE90545FFF732FE062511E0042A2CD1DD
:1016A000A06806BB0A68434B9A421CD105AA04F005
:1016B00015FC40B905AAD4E9020104F02CFC05464A
:1016C000284609B0F0BDDDE90530C01AFFF7FCFE81
:1016D000E3688268054605999200C06803EB8101C2
:1016E00017F04AFCECE700232A4601462068FCF785
:1016F000C1FAE36853F82050E2E7002E53D10A689C
:101700002C4B9A424FD101AA6946FCF77BFA05AAF5
:101710002946A06804F0E2FB00289BD0009AE0680C
:10172000DDE90535ED1A551B002D27DDA16863683D
:101730002944994206D98900F0F7C9FEA368E06000
:101740002B446360009A059BE0681344A2680699E5
:101750002A4400EB8101D21A00EB8300920017F0BB
:1017600033FCE368009A05989200019903EB80002E
:1017700017F02AFCA3681D44A5608DE7019992002B
:1017800000EB830017F020FC0699A268059B009FE0
:10179000521AE0683B44920000EB810100EB8300A9
:1017A00017F012FC66E7024629462046FFF733FF92
:1017B00072E700BFD45B056070B5054648680E4609
:1017C0000022BA2104303BF077FEB0B1406801F04E
:1017D000CFFF04467068002240F2BA5104303BF05B
:1017E0006BFE60B1406801F0C3FF22460346074923
:1017F0002846BDE87040F1F7F9BC054CEAE72246FF
:1018000028460449BDE87040F1F7F0BCAC540560CF
:10181000CC3B0660C4540560F8B51546126807460F
:101820000C464068CAB9CE00043046F00206314684
:101830003BF042FE024610B143682B600CE00E2CD8
:101840000AD07868722104303BF036FE20B1314670
:1018500040683BF0C5FD2860F8BD03799B070DD5B6
:101860000C4B9842F8D10C4ED6F8CC3023B901205D
:10187000FDF72CFEC6F8CC00D6F8CC00E1006A6873
:1018800041F002011AB9FDF7A6FE0023D5E7FDF7E6
:1018900093FEFAE7E86C0560B0270020C000012243
:1018A00070B540F002050C4829463BF005FE44683F
:1018B000064674B91020F0F7EFFD084B04460360AC
:1018C0000120FDF703FE2A46BA216060FDF774FE91
:1018D0007460204670BD00BF00280020F0550560F0
:1018E00073B5C000002240F002050E4829463BF0C7
:1018F000E3FD044698B146686A46112130463BF044
:101900009BFD009B53B100216A4608463BF0D8FD81
:101910000122294604483BF0CFFD4660646820461A
:1019200002B070BDD454056000280020C100002220
:1019300010B541F00201044605483BF0BDFD20B959
:101940002046BDE81040FFF7CBBF406810BD00BF88
:10195000002800200620704770B5154606460C4644
:10196000FBF7CEFF0D4BC2689A4202D00C483BF009
:1019700003FE04F00703022B07D0A30703D122685C
:10198000084B9A4201D00020F1E701222146301D88
:101990003BF092FD4560062070BD00BF31590160EB
:1019A0002C560560EC62056007B5820707D1016817
:1019B000074A914203D1C268064B9A4202D00648B8
:1019C0003BF0DAFD01A903F09DFF03B05DF804FBD5
:1019D0005C680560315901602C56056010B50446FD
:1019E0000846114600223BF04BFD21460420BDE88D
:1019F0001040FBF77EBF000038B505460C46FBF7EC
:101A00007FFF0F4BC2689A4202D00E483BF0B4FDF4
:101A100004F00703022B07D0A30703D122680A4B67
:101A20009A4201D00020F1E702222146281D3BF016
:101A300043FD18B9054906483BF0AEFD062038BD08
:101A4000315901602C560560EC6205604256056014
:101A50008C4705604368184770B5054610200E4650
:101A6000F0F71AFD044695E80F0084E80F002046C1
:101A7000E66070BD70B5054610200E46F0F70CFD0F
:101A8000044695E80F0084E80F002046A66070BD6C
:101A900070B5054610200E46F0F7FEFC044695E8AA
:101AA0000F0084E80F002046666070BD10B586B058
:101AB0000446084611461A4602AB0193084B0093B0
:101AC00004233BF029FD21461020FBF712FF029A68
:101AD0004260039A8260049AC26006B010BD00BFE3
:101AE0002457056004307047032A0CBF014902499E
:101AF000F1F700B8C0570560F3EE046038B50B6825
:101B00000C4606490546DA88F1F770FB2168224643
:101B100028464031BDE83840FCF734BE0F47056029
:101B2000C26B00F14003002010B5824202D14FF099
:101B3000FF3010BD53F8044B8C42FAD00130F4E76B
:101B400038B51368054614464BB90068FFF7E8FF3F
:101B5000431C03D0831C55F82330236038BD024951
:101B600002483BF019FD00BF045805608C47056032
:101B70002DE9F3471746C26B80460C46CD199946AE
:101B8000954204D02B461E491E483BF0EDFC4FEA1F
:101B9000840A0021284603F0F1F8524606464946D9
:101BA00040F8088B17F0E8F90AF10800BA0009F1CB
:101BB000040A2F440021304417F01EFAA74203D82C
:101BC000304602B0BDE8F08759F8240001F0B8FDB6
:101BD000014601904046FFF7A3FF431C019A03D141
:101BE000094908483BF0C0FC06EB8005AB680BB127
:101BF0000649F6E75AF824300234AB60DEE700BF4E
:101C0000CC3C0560784C0560185805603958056073
:101C1000F8B500F1100407460D46A4002046403CEC
:101C2000F0F73AFC06463C22002117F0E5F92C4477
:101C3000F76306F14007A54201D13046F8BD55F8DB
:101C4000040B01F07DFD47F8040BF4E71FB501918B
:101C500001F076FD019B044603F00702022A05D03D
:101C60009A0708D11A68144B9A4204D101A901209D
:101C700002F06EF8019003AA02A90198FBF7C2FFD7
:101C8000DDE90201FFF7C4FF0C4AC48002600822AC
:101C900082800B4A82600B4AC2600B4A42610B4A47
:101CA00082610B4AC2610B4A02620B4A42620B4AD2
:101CB000426304B010BD00BFEC6205605C68056063
:101CC000FD1A0160711B0160294D0160B54D016075
:101CD000411B0160A14E01606D4C016070650560A3
:101CE000C268002A05DDD0E90113994206DB002312
:101CF0000AE0FCD0D0E901139942F8DD41684B00BD
:101D00000A4443F00103426018467047C36810B5A7
:101D1000D0E901420348C1E90223C1E900040846B1
:101D200010BD00BFCC58056070B50E460446114684
:101D3000134A30461D463BF0A3FB21461020FBF71B
:101D4000D8FD00230446436001239E42C3602868F7
:101D500004D1FBF76DFEA060204670BDFBF768FE66
:101D600060606868FBF764FE032EA060F4D1A86889
:101D7000FBF75EFEE0600028EED102483BF0FCFA83
:101D8000060002007058056038B50C460546D1E9DA
:101D900001230949F1F72AFAE268012A05D1284608
:101DA0000649BDE83840F0F7A5BE28460449BDE81D
:101DB0003840F1F71BBA00BF7A580560673F0560ED
:101DC00087580560042A1FB504463DD16268D0E9F2
:101DD00002309B1A00280344CCBF03F1FF330133C8
:101DE00093FBF0F08B0720EAE0701FD10A68174BD5
:101DF0009A421BD101AA04F071F815491020FBF793
:101E000078FDE2686168019B03FB02134360029B5B
:101E1000616803FB021303994A4300298360C2608F
:101E200002DAE2689B1A836004B010BD0A46002300
:101E300001462068FBF71EFFE268636802FB003082
:101E4000400040F00100EFE70020EDE7D45B0560C3
:101E500090580560136810B514462BB9922904D127
:101E60004068FEF72FFF206010BD962901D18068E1
:101E7000F7E79529F8D1C068F3E7D1E9023249685C
:101E8000002AA3EB01031344CCBF03F1FF3301335A
:101E9000042893FBF2F303D0052806D000207047F6
:101EA000002BCCBF1E200E20704723EAE3704000B9
:101EB00040F0010070470346806840B1411E042293
:101EC00058689960490041F00101FBF7F7BF70477E
:101ED00037B51D460446084611464FF002123BF046
:101EE000CFFA6A46D02128683BF0A6FA009B43B19E
:101EF00000216A4608463BF0E3FA0446204603B058
:101F000030BD21460C20FBF7F4FC044628686060D5
:101F1000FBF7C2FFFBF78CFDA060EFE7820708D15B
:101F20000068064B984206D0054BC31A58425841E8
:101F30007047002070470120704700BF005A0560BD
:101F4000C4590560044B0B60044BC1E90130002308
:101F50000846CB60704700BFE8560560D521016098
:101F60000122043008B53BF00FFA062008BD02221A
:101F7000043008B53BF008FA062008BD38B5044621
:101F8000084600213BF070FA0434054628463BF031
:101F900017FB014600B938BD012220463BF0F4F999
:101FA000F4E770B506460D460124B44201D306207D
:101FB00070BD55F8241001342868FFF7DFFFF4E7FF
:101FC00038B50446084600213BF04EFA0434054675
:101FD00028463BF0F5FA014608B9062038BD032231
:101FE00020463BF0D1F9F3E730B585B0044608460A
:101FF000694604343BF038FA054628463BF0E0FADF
:10200000014610B91E2005B030BD002220463BF02D
:10201000BBF90028F1D00E20F5E738B50446016879
:102020001020FBF766FC6168054604303BF05CFA63
:10203000A3686268E1689200E868AB6016F09CFFF4
:10204000284638BD13B50191FFF7E7FF0446019913
:10205000FFF794FF204602B010BD13B50191FFF7C2
:10206000DCFF04460199FFF7ABFF204602B010BD2C
:1020700010B5022204300C463BF086F918B921460F
:1020800002483BF0D5F9062010BD00BF6C49056041
:10209000043008B53BF0B8FA062008BD2DE9F84336
:1020A00007460E460C681AB92046FFF7B6FF0446ED
:1020B000012504F10409BD4202D32046BDE8F8839E
:1020C00056F82500844204D148463BF09DFA01357C
:1020D000F1E700213BF0C8F9804640463BF070FA3A
:1020E00001460028F3D0022248463BF04DF9F4E7C0
:1020F000012208B5FFF7D2FF062008BD0022FFF736
:10210000CDBF00008A072DE9F84304460D4611D1E2
:102110000E68214BF31A5E425E41AB6863B91EB193
:102120001E492046F0F7E6FC1D492046BDE8F8436D
:10213000F0F7E0BC0026F0E71EB11A492046F0F7A0
:10214000D9FC19492046F0F7D5FC00270123DFF818
:1021500064806A68BA4206D814492046F0F7CAFC7F
:10216000C6B11349E1E7EA684FEA870952F8272028
:1021700072B1042A0CD01BB941462046F0F7BAFCD4
:10218000EB680122204653F80910FBF7CDFB002332
:102190000137DEE7BDE8F883C4590560C0DD04609F
:1021A000445905604A5905609344056091350560BE
:1021B000673F0560DC40056008B504303BF0E8F996
:1021C00018B9024902483BF0E7F908BD55590560C6
:1021D0006C4905608168C36810B54C68A34201D39F
:1021E000002208E0CA6852F823200133002AF5D003
:1021F000042AF3D0C360104610BD00000528F8B5CE
:102200000D4609D006280CD0042824D18B68002B59
:1022100014BF1E200E20F8BD8868400040F0010069
:10222000F9E711F0030016D10E680C4B9E42F2D173
:102230004F680446A74201D17000EFE7EB6853F8FE
:10224000241031B1042904D006203BF0ADF806EB90
:1022500060060134EEE70020DDE700BFC4590560E9
:10226000F8B505460C4610200A49FBF742FB071D4E
:10227000294604EB8505064638463BF035F9AC4265
:1022800001D13046F8BD012254F8041B38463BF01A
:102290007BF8F4E7005A05602DE9F3410F46002171
:1022A000054616460846FFF7DBFF00210446384680
:1022B0003BF0DAF805F10408074638463BF080F9B0
:1022C000014670B94EB1E868F0F70EF963686B60CB
:1022D000A368AB60E3680624EB60204602B0BDE86B
:1022E000F0810022404601913BF04EF80199002810
:1022F000E3D02046FFF734FEDFE7814202D001221F
:10230000FFF7CABF06207047814201D1FFF785BEA3
:102310000022FFF7C1BF012204303BF035B870B591
:102320000C4605461146022220461E463BF0A8F800
:102330003CB921462046FFF793FF0446204625601E
:1023400070BD00210846FFF78BFF0021044630686E
:102350003BF08AF8064630463BF032F90146002849
:10236000ECD02046FFF7D7FFF5E700002DE9F0415C
:1023700086B016460446CDE90010FFF7CFFD0246B1
:10238000002835D101AB012120480127FFF7C7FF05
:102390000446009D2846FFF7C1FD024650BB6B4630
:1023A00001211A484FF00108FFF7B9FF05461EB199
:1023B000A268AB689A4226D0154B2E1D0293154B8E
:1023C000CDE903340023059302A8FFF703FF01467C
:1023D00098B91E2617B1201D3BF016F9B8F1000F71
:1023E00002D0281D3BF010F9304606B0BDE8F08160
:1023F0000027CEE74FF00008D9E7002230463AF038
:10240000C3FF0028E0D10E26E4E700BF005A0560B4
:10241000E8560560D52101600B46002201461846AA
:10242000FFF7A4BF0022FFF7A1BF0000F0B585B001
:10243000174606460C46CDE902128A0720D10D68E0
:102440003F4BEB1A5D425D41242E01956BD038461F
:10245000FFF764FD00286ED0019A1C2E6BD8DFE8D0
:1024600006F04A5054585D6A6A6A6A212E356A6AD3
:102470006A456A6A6A6A6A6A2911166A6A6A1C0087
:102480000025E1E739462046FFF7E7FD03E039463E
:102490002046FFF739FF044609E002A90220FFF7B2
:1024A0002DFEF8E735B102A90220FFF77AFD20469C
:1024B00005B0F0BD39462046FFF7C4FDEBE73946CD
:1024C0002046002DE0D0FFF77BFDF0E7BC4205D1B0
:1024D000002DECD12046FFF7A0FDDCE72046394671
:1024E000FFF7DAFE002D08BF0446E0E702A902204C
:1024F000FFF7D4FDCFE7012239462046FFF736FF2C
:10250000C9E7012221463846F8E7A268BB689A422B
:102510000FD139462046FFF785FFBCE739462046F4
:10252000FFF77AFFB7E700223946201D3AF02CFF6B
:1025300018B90E24BBE70024B9E71E24B7E700BF93
:10254000005A05604A680149F0F750BE0F47056020
:1025500070B504460D46104E1049F0F7CBFA012233
:1025600069682046FBF7E0F931462046F0F7C2FAE9
:102570000122A9682046FBF7D7F931462046F0F73B
:10258000B9FAE96820460122FBF7CEF92046044952
:10259000BDE87040F0F7AEBADC400560B45B0560A2
:1025A000673F0560136893B9922902D143681360AD
:1025B0007047962901D18368F9E7952901D1C3684D
:1025C000F5E7B1F57B7F04BF014BC2E900307047EE
:1025D000105C056070B506460D4614460349102090
:1025E000FBF787F9C460C0E9016570BDD45B056085
:1025F0002DE9F0418046C0680D46164606281BD0DE
:10260000FBF716FA071E02D125483AF0B5FE14DC96
:10261000D8F80400062833D16C1ED8F80800062824
:1026200038D0FBF705FA0028B8BF401940EAE0703F
:10263000A84232DB013D1CE00127D8F8040006283F
:102640001CD0FBF7F5F9041EB8BF641924EAE47442
:10265000AC42A8BF2C46D8F80800062809D0FBF7E2
:10266000E7F90028B8BF401920EAE0708542A8BF0A
:102670000546B760C6E90045BDE8F0810024EAE7F9
:10268000FBF7D6F9041EB8BF641944EAE474AC42FF
:10269000C2DAC2E74FF0FF35EBE70546E9E700BFD6
:1026A000BB5B056010B5044686B00846FEF7BAFB72
:1026B0006A4601462046FFF79BFF009B03A90320C3
:1026C0005B0043F001030393019B5B0043F00103B4
:1026D0000493029B5B0043F00103059302F04EFB61
:1026E00006B010BD0E280CD01E280AD010F0010331
:1026F00007D1820707D10068044BC31A58425841DA
:102700007047012070471846704700BF9C52056013
:1027100008B50146FFF7E6FF38B98A0704D1086813
:10272000034BC31A5842584108BD0120FCE700BFC3
:10273000004E0560044B0B60044BC1E901300023DF
:102740000846CB60704700BFE8560560512701601E
:1027500013B50446806800F00703022B11D101A9CC
:10276000C008F0F70EF8E268019B9A4237BF835C1D
:10277000002001325B003CBFE26043F0010002B088
:1027800010BD8368C0680193EDE7000008B5FBF752
:10279000B7F8C2880349972A03480CBF42239723FE
:1027A0003AF0E2FE185C0560784C05602DE9FF47C1
:1027B0000C4682460868FBF7A3F881466068FBF781
:1027C0009FF8814502D06068FFF7E0FF206800F0C5
:1027D0000703022B39D102A9C008EFF7D2FF064642
:1027E000606800F00703022B33D103A9C008EFF79C
:1027F000C8FF8046029ABAF1020F06EB02072FD9F2
:10280000A368062B2AD0012148460091314602F0E8
:102810002FF80546BAF1030F0AD0E368062B07D05C
:102820000122314648460092029A02F021F80746FA
:10283000039B4BBB791B2846F0F718FD0130400085
:1028400040F0010004B0BDE8F0878368C6680293D9
:10285000C6E78368D0F80C800393CBE73546D9E709
:102860003546E5E74146284616F0E8FB38B901341D
:102870003546039AAE18BE42F4D96000E0E7284618
:10288000F0F7DEFC0646F3E70024F2E701F0070369
:10289000022BF7B5074608460FD101A9C008EFF78C
:1028A00070FF0646019B23B3144B9F4223D0144B69
:1028B00000249F4209D1254616E08B68CE6801931B
:1028C000F0E7305DB847A0B10134019BA342F8D8CE
:1028D0001E2003B0F0BD305DF0F7E2FC18B1305DB2
:1028E000B847054628B10134019BA342F3D8002D17
:1028F000EED10E20EDE70024DDE700BF01330060DC
:102900001533006001460148FFF7C0BF8D320060FB
:1029100001460148FFF7BABFA132006001460148F5
:10292000FFF7B4BFB532006001460148FFF7AEBF04
:102930000133006001460148FFF7A8BF153300606E
:10294000884230B513D20378303B092B0FD80023CF
:102950000A25136010F8014B1368303C814205FBD7
:102960000343136003D00378303B092BF2D930BD09
:10297000012A13B50C4613D100F00703022B0BD12B
:1029800001A9C008EFF7FDFE019B206000206360F5
:102990004223A36002B010BD8368C0680193F3E7CF
:1029A0000120F7E72DE9F84F98468F1804460D46A9
:1029B0000B4600229F4217D8002A0CBF272622264A
:1029C000DFF89C903246DFF89CA02046DFF898B0F4
:1029D0001F49F0F70BFCBD4210D3324620461C497C
:1029E000BDE8F84FF0F702BC13F8011B272903D00C
:1029F0002229DFD12726E3E70122DBE715F8012BA7
:102A0000B24205D1324613492046F0F7EFFBE2E728
:102A10005C2A04D110492046F0F76CF8DBE71F2A46
:102A200008D97F2A12D0B8F1000F01D013060DD4B7
:102A30000749E9E70A2A01D10849ECE70D2A01D143
:102A40005946E8E7092A01D15146E4E74946DBE760
:102A50000D870560435C0560475C05604A5C056066
:102A6000535C0560505C05604D5C05602DE9F843E2
:102A70000D461646184F04462E44DFF87080DFF8E6
:102A800070901649F0F736F8AE4205D82046134943
:102A9000BDE8F843F0F72EB815F8012B222A01D033
:102AA0005C2A04D139462046F0F7A0FBECE71F2A48
:102AB00001D90B49F7E70A2A04D10A492046F0F761
:102AC00019F8E1E70D2A01D10749F7E7092A01D1F1
:102AD0004946F3E74146E6E7435C056095440560F7
:102AE0000D8705604A5C05604D5C05605A5C0560B9
:102AF000505C056001F00703022B73B504461646CF
:102B000008460DD101A9C008EFF73BFE0546032E8C
:102B10000AD1019A29462046FFF7A8FF02B070BDEE
:102B20008B68CD680193F2E7042ED4E9000303D14A
:102B3000019A29469847F1E7012204499847012361
:102B4000019A29462046FFF72DFFE7E7CB400560B5
:102B500099422DE9F047DDF820A0804691461E46B7
:102B600013D3BAF1000FA1EB0304CEBF0025254615
:102B7000002408EB050732464946384616F05EFA4F
:102B800020B1A54201D05544F3E700273846BDE8FF
:102B9000F08700002DE9F04F87B00D4682460868A7
:102BA00093460393FAF7ACFE07466868FAF7A8FE67
:102BB000874202D06868FFF7E9FD286800F0070344
:102BC000022B3ED104A9C008EFF7DBFD044668687C
:102BD00000F00703022B38D105A9C008EFF7D1FD9B
:102BE0008146049ABAF1020F04EB020834D9AB68AB
:102BF000062B2FD0012138460091214601F038FEE6
:102C00000646BAF1030F0AD0EB68062B07D0012263
:102C1000214638460092049A01F02AFE8046B045CB
:102C20000AD3A8EB0601059B4A463046CDF800B012
:102C3000FFF78EFF014688B9039BEBB110483AF0CD
:102C40009BFB8368C4680493C1E78368D0F80C9049
:102C50000593C6E72646D4E72646E0E7094B9F42A0
:102C600008D12046F0F7F5FA400040F0010007B027
:102C7000BDE8F08F001BF7E74FF0FF30F7E700BF2C
:102C8000615C0560EC62056000230122FFF782BFF2
:102C900000234FF0FF32FFF77DBF01231A46FFF7F5
:102CA00079BF01234FF0FF32FFF774BFF8B5144628
:102CB0000E4601461020FAF71CFE054684607EB1E0
:102CC00021463046EFF748FC6860601CEFF7E4FBF4
:102CD00022463146E860074616F04EF900233B5580
:102CE0002846F8BD08B5EFF781FCC00040F00200AF
:102CF00008BD0000194B984270B506460D460FD12D
:102D0000D1E90110EFF744FC044648B1E40028463D
:102D1000EFF71AFE002344F002042B60204670BD3A
:102D200031461020FAF7E5FD696804468160A8681D
:102D3000EFF712FC69682B6801316060994208D195
:102D4000AB68E3600023D4E902218B54AB602B60B5
:102D5000E4E7A868EFF7BBFBE060F3E7EC6205602F
:102D60002DE9F04104468AB00191FAF7C9FD04F05B
:102D700007030646022B30D102A9E008EFF701FD58
:102D80000746019A364B12F0030F05D112689A429A
:102D900009D034498A4206D0DC68002201AB012107
:102DA0002F48A0470190002404AA03A901982546B2
:102DB000FAF728FF039BA34213D8294606A8EFF78A
:102DC000A5FD0025089C039BAB4228D806A93046E8
:102DD000FFF790FF0AB0BDE8F081A368E7680293AF
:102DE000CFE7049B4FEA840853F82400FAF788FDE4
:102DF000864202D01C483AF0BFFB0CB1029B1D4436
:102E0000049B53F8080000F00703022B05D1C0080B
:102E1000EFF7A0FC05440134CCE78068FAE735B150
:102E20002046029A394616F0A7F8029B1C44049BE0
:102E300053F8250000F00703022B0CD105A9C008A8
:102E4000EFF79FFC01462046059A16F095F8059B82
:102E500001351C44B7E78368C1680593F3E700BFF9
:102E60003454056070650560755C056000F007030B
:102E7000022B70B5044686B00D4626D101A9C008C4
:102E8000EFF77FFC06462846FAF7D2FD019B054680
:102E9000834217D2014602A8EFF738FD2A462021C7
:102EA000049816F0A9F8019A04983146AD1A00EB7F
:102EB000550016F061F82046FAF722FD02A9FFF747
:102EC00019FF0446204606B070BD8368C6680193AA
:102ED000D9E704282DE9F04F0C4691B018D1C86805
:102EE000FAF7A6FD18B9206811B0BDE8F08F40EAE6
:102EF000E07320680493FAF703FD06906068FAF720
:102F0000FFFC069B0546984205D06068FFF73EFC33
:102F10004FF0FF33EDE7A068FAF7F2FC854201D0ED
:102F2000A068F3E7206800F00703022B4DD109A940
:102F3000C008EFF726FC0390606800F00703022B3F
:102F400048D10AA9C008EFF71CFC0590A06800F062
:102F50000703022B43D10BA9C008EFF712FC8346ED
:102F6000DDE909329A42BED80026DDE90953002B7B
:102F70003AD126B10B9A5946304615F0FDFF0B9F0A
:102F80004FF0010ADDF80C80049B9A450CD05DB12E
:102F900001220A9B294640460092059A0793FFF7B3
:102FA000D7FD079B814618BB26B12A464146F0193A
:102FB00015F0E2FFE919002E39D1BAF1000F92D0D5
:102FC0000CA8EFF7A3FC0E9ECFE783680993C368B4
:102FD0000393B1E783680A93C3680593B6E78368F0
:102FE000D0F80CB00B93BBE74FF0000A5746C9E787
:102FF0000BB909F10109A9EB080526B12A4641469A
:10300000F01915F0B9FF2F4426B10B9A5946F01963
:1030100015F0B2FF0A9B0AF1010A099D09EB0308AA
:10302000039B0B991D440F44A5EB0805ACE70CA9C5
:103030000698FFF75FFE57E701F00703022B2DE923
:10304000F041074686B00C4617D101A9E008EFF71A
:1030500098FB0646019902A8EFF758FC0025DDF819
:103060001080019BAB420CD82046FAF749FC02A91C
:10307000FFF740FE06B0BDE8F0818B68CE68019393
:10308000E8E7705DB84708F805000135E9E700009A
:1030900001460148FFF7D0BF2933006001460148CF
:1030A000FFF7CABF3933006013B504460191EFF74B
:1030B0006FFA019A20B1C00040F0020002B010BDCA
:1030C0002146034802B0BDE81040FFF7EFBD00BF46
:1030D000EC620560F0B5064687B00F461C46154603
:1030E0000AB13AF095FA0622294638463AF0C8F96C
:1030F000002F60D0012F0FD16A46102102A8EFF7F0
:1031000017FC216868462A46FAF70EFC02A93046E9
:10311000FFF7F0FD07B0F0BD206883073CD10268DF
:10312000264B9A4238D100F00703022B1CD1694686
:10313000C008EFF726FB0546206800F00703022BC6
:1031400016D1C008EFF7FAFA044624B900992846C8
:10315000EFF702FA044600992846F0F7FCF848B960
:10316000002117483AF018FA8368C5680093E3E72E
:103170004468EAE700992846EFF70AFA18B1C00058
:1031800040F00200C6E7009F31461020FAF7B1FB7D
:103190004460C0E90275BDE702A90122FAF7C6FE44
:1031A000DDE90201F0F7D7F80028D9D0DDE9020106
:1031B000FFF77AFFAEE70A20ACE700BF606005606A
:1031C000B44C056001280B4607B506D10B680220F8
:1031D000009340F20A5301936B46014600220348D4
:1031E000FFF778FF03B05DF804FB00BFEC620560F9
:1031F0000A4601460148FFF759BD00BF60600560FF
:103200000346086870B50C4610F003018EB003D178
:1032100005683D4A954229D000F00702022A04D0F1
:1032200061BB056839498D4228D1023B012B67D823
:10323000022A1DD10AA9C008EFF7A3FA05462068A3
:1032400000F00702022A17D1C008EFF777FA044608
:1032500024B90A992846EFF77FF904460A9E102000
:103260002949FAF746FB4460C0E902650EB070BD1B
:103270008368C5680A93E2E74468E9E7012B3FD811
:10328000C30713D5421002D500203AF075F8114655
:103290000AA80192EFF73AFB0021019A0C9815F069
:1032A000ABFE0AA91848FFF725FDDFE7012203A9B5
:1032B000FAF72DFE20B1DDE90301FFF799FFD5E70D
:1032C0002068FAF721FD70B9102106A8EFF70DFB71
:1032D00020680AA93AF0C8F8044620463AF070F986
:1032E00018B906A9DEE74110EFE7FAF7A1FBFF28BE
:1032F00001D90748C9E7C1B206A8EFF77DFBECE7A3
:1033000004483AF039F900BF60600560EC6205607E
:10331000BA5C0560D35C05600846194608B50AB179
:103320003AF076F918B1BDE80840FFF769BF0148E7
:1033300008BD00BF50600560012807B50BD10B68C0
:1033400002206946009340F20A530193FFF758FFA9
:1033500003B05DF804FB0028F8D10148F8E700BF8E
:1033600050600560034608461146034A9A4201D15F
:10337000FFF79ABEFFF73CBFEC6205602DE9FF4105
:1033800002AB0C46013804310193234B0093012317
:103390003AF0A2F82068FAF7B3FA0021804608460E
:1033A000FEF71CF90546206800F00703022B0CD13C
:1033B00003A9C008EFF7E5F90146039E0E44B142A8
:1033C00007D3284604B0BDE8F0818368C168039341
:1033D000F3E70B461A781C4601330A2A19D00D2A46
:1033E00012D163780A2B0CBF022701279DF8083001
:1033F000621A03B13A444046FFF7B4FF014628463B
:10340000FDF795FEE119DAE79E421C46E2D100275E
:10341000ECE70127EAE700BF3C6005602DE9F04FCB
:103420008BB00C46164605901068FAF769FA012C25
:10343000074641D07068FAF763FA8742706801D096
:10344000FFF7A4F900F00703022B30D109A9C00847
:10345000EFF797F98346099B0693306800F007035E
:10346000022B2ED109A9C008EFF78BF90390059B19
:103470000024DDF82490012BA246A046CDF8109040
:103480000BBF4FF0FF33012309F1FF3500250CBFBF
:1034900007930793049BCBB9BAF1000F27D1234BB5
:1034A00023489F4208BF0A200BB0BDE8F08F836815
:1034B000D0F80CB00993CEE70623DFF878B0069376
:1034C000CBE783680993C3680393D0E70123039A8A
:1034D000069958462A440093FFF73AFBA8B9BAF177
:1034E000000F18D1059B4BB909F1FF34A846621CA7
:1034F000A2EB08024A4512D13068D5E7059B2C465D
:10350000012B0AD0A8464FF0010A079B1D44049BDB
:10351000013B0493BEE72C46F7E7D046E7E7039B61
:10352000384643441946FFF71DFFBDE7EC620560CE
:10353000506005609C6205600A4601460220FFF764
:103540006DBF0A4601460020FFF768BF0A460146E4
:103550000120FFF763BF00002DE9F0410C4688B061
:1035600090460546FAF7CCF907462046FAF7C8F91F
:10357000874202D02046FFF709F905F00703022B26
:1035800011D103A9E808EFF7FCF8064604F0070399
:10359000022B0CD104A9E008EFF7F3F8049B53B910
:1035A0001C4839F0E9FEAB68EE680393EEE7A368C8
:1035B000E0680493F2E7184A03999742CDF8008037
:1035C0000CBF0A22154AB8F1010F079218BF0795E0
:1035D000CDE905220246304608BF0595FFF7B8FA47
:1035E00088B1851B314638462A46FFF7BBFEDDE928
:1035F0000321CDE90504521A29443846521B3144AF
:10360000FFF7B0FE079005A9032001F0B7FB08B053
:10361000BDE8F081ED5C0560EC620560506005601E
:103620000122FFF799BF4FF0FF32FFF795BF00006F
:10363000F0B5054685B00C461746FAF761F905F076
:1036400007030646022B15D1E8086946EFF799F8FB
:103650000546042F26D1A307009818D12268124BE3
:103660009A4214D101AA214602F038FC30B90F4821
:1036700039F0BEFEAB68ED680093EAE7DDE90112C0
:103680003046521A2944FFF76DFE05B0F0BD0146E1
:10369000002322463046FAF7EDFA285C400040F05D
:1036A0000100F2E70020F0E7D45B05604C400560C4
:1036B0002DE9F34100F0070804460D4601F0070725
:1036C000B8F1020F12D1022F05D1431A58425841C6
:1036D00002B0BDE8F081C008EFF730F80646686830
:1036E00086B178B1B0420DD00020F1E7022F4668D4
:1036F000F5D1C808EFF722F8002EF2D1A368E468EC
:10370000009307E0B8F1020FF8D1E0086946EFF73F
:1037100038F80446022F0FD101A9E808EFF731F875
:103720000146DDE900239A42DED1204615F086FCF1
:10373000B0FA80F04009CBE7AB68E9680193F0E7A5
:1037400008B500F00703022B01D1C00808BD8307AC
:1037500009D10268054B9A4205D1D0E90210BDE8B3
:103760000840EEF743BFFFF711F800BFEC620560B9
:1037700000F00703022B07B508D0830704D10368C4
:103780009A69074B9A4208D0FFF700F801A9C008D0
:10379000EEF7F7FF03B05DF804FBC068FAE700BF7F
:1037A000E137016000F00703022B13B50C4608D087
:1037B000830704D103689A69084B9A4209D0FEF73F
:1037C000E5FF01A9C008EEF7DCFF019B236002B012
:1037D00010BD8368C0680193F7E700BFE13701605F
:1037E0002DE9F04F21289DB004460D4601F0070752
:1037F000099240F0088209AB12F0030491460B9342
:103800004FF001030C9308D11368B44A934207D1D7
:103810000BAA0CA9484601F0B9FB4FF0000904E0DF
:10382000AF4A934218BF4FF000090C9B022F04933C
:103830000B9B06931FD10DA9E808EEF7A2FF059098
:10384000AC071DD1A74B2A68D01A4342434110AAA6
:10385000102114A80793EFF76BF8059A0D9B00272A
:10386000144602EB0308A0450CD8049BBB4200F0B1
:10387000C0819D4822E0AB680D93EB680593DFE7BC
:103880000023E4E72178252904D014A8EFF7B4F841
:103890000134E8E7661CB04502D8944839F06CFD65
:1038A0006178252904D114A83446EFF7A5F8EFE78D
:1038B000282930D1B9F1000F02D18D4839F05CFED2
:1038C000A01C01460E4616F8013B292B1DD1091AF2
:1038D0000127FFF707FA01464846FBF7DFFD0546DB
:1038E0004FF0000B33464FF0200A5E4698451C46C9
:1038F00013D80023A0450E9336D923782A2B6DD1F7
:10390000049BBB4225D87B48D8E7884501D17A483B
:10391000C4E73146D6E70025E2E713F8012B2D2A4C
:1039200002D146F00106E1E72B2A02D146F0020659
:10393000DCE7202A02D146F00406D7E7232A05D087
:10394000302AD6D146F040069246CFE74FF0100B12
:10395000CCE77B1C01340893069B53F82700FAF749
:1039600067F8089B0E901F464FF0FF33A0450F935A
:1039700093D923782E2B16D1601C80458DD963787E
:103980002A2B32D1049BBB42BDD97B1C0234089345
:10399000069B53F82700FAF74BF8089B0F901F4639
:1039A000A0457FF67AAF35B9049BBB42ABD9069BE5
:1039B00053F8275001372378472B65D8442B68D913
:1039C0002846FAF7B1F80F9B21783246019310A8E8
